:200000000C94FB010C9418020C9418020C9418020C9418020C9418020C9418020C941155E2
:200020000C9418020C94415A0C9418020C9418020C9418020C94825A0C94595A0C94180214
:200040000C9418020C9418020C94A66F0C9418020C94AE6C0C94DA6C0C9418020C941802A9
:200060000C9418020C9418020C9418020C941802571E5D1E721E771E7C1E811E861E8B1EFD
:20008000901EA51EC31EC81ECD1ED21ED71EDC1EE11EF11EAC1FB21F1E1F231F281F2D1FA2
:2000A000321F371F501F551FAF1E5F1F641F691FA01F461E521E3C1F411F461F4B1F631EC2
:2000C000681E6D1EA01EFB1E5A1F951E9A1EE61EEB1EAA1EF61E441E441E441E001F441EC4
:2000E000441E441E141F191F6E1F731F781F7D1F821F871F8C1F911F961F9B1FB41EB91EC5
:20010000BE1E051F0A1F0F1F441E441E441E441E441E441E441E441E441E441E441E441EF0
:20012000441E441E441E441E441E441E441E441E441E441E441E441E441E441E441E441E9F
:20014000441E441E441E441E441E441E441E441E441E441E441E441E441E441E441E441E7F
:20016000441E441EB81FBC1FC11FC61FD71FDB1F441EE71FEF1FFA1FFF1F04200920132027
:200180001D20441E212025202F20332037203B2043204D20512055205D2067203F20592054
:2001A000EB1F6C207020DF1FE31FCB1FCF1FD31F441E441E441E441E441E441E441E441E3F
:2001C000441E441E441E441E441E441E441E441E441E441E441E441E441E441E441E441EFF
:2001E000441E441E441E441E441E441E441E441E441E441E742079207E20832029294C2FF0
:200200008833EB27D228623073308C309030A630BB30CF300D3228323C324F327832A232A0
:200220001B281D28272829282B2834283D283F284128432845284B284D284F285128532887
:200240005528572859285D286128642867286928742876287B28822887288C2895289E28FA
:20026000A728B228BE28C028D02886299429CC29DA29E829F629042A122A202A4A2AAE2A7B
:20028000BC2ACA2AD82AE62AF42A022B2C2B402D4E2DAA2BB82BC62BD42BE22BF02B3E2CAE
:2002A0004C2C742A682C782C882C322D6A297829FE2B0E2C1E2C2E2CA229B029BE29662A87
:2002C000482B5A2C2E2A3C2A102B1E2B582A3A2B883388338833562B8833883388338E2B60
:2002E0009C2B982CA62CB42CC42CD42CE42CF22C022D122D222D842A922AA02A642B722B86
:20030000802B8833883388338833883388338833883388338833883388338833883388333D
:2003200088338833883388338833883388338833883388338833883388338833883388330D
:200340008833883388338833883388338833883388338833883388338833883388335C2D1F
:20036000682D782D882DBC2DC82D8833F02D082E162E242E322E422E4E2E5A2E8833662EE9
:20038000722E7E2E8A2E962EA22EBC2EC82ED42EE22EFA2E062FB02EEE2EFC2D142F202FC1
:2003A000D42DE22D982DA42DB02D88338833883388338833883388338833883388338833B1
:2003C00088338833883388338833883388338833883388338833883388338833883388336D
:2003E00088338833883388338833883388332C2F372F3A2F3F2F11241FBECFEFD0E1DEBF2A
:20040000CDBF12E0A0E0B1E0E0EEFBEE02C005900D92A03DB107D9F71CE0A0EDB2E001C05F
:200420001D92AB36B107E1F70E943D160C94EE750C94000090E08091DC028D3208F491E079
:20044000892F08951198099A1092EC071092D0021092D1021092D2021092D3020895109251
:20046000840A1092D8021092D9021092DA021092DB021092D4021092D5021092D6021092EB
:20048000D7020E94220281E00895DC01009711F480E00895E091B708F091B808E85BFE4F48
:2004A00080818C9381E00895982F807E11F080E00895E091B708F091B808E85BFE4F908347
:2004C00081E00895DC01009711F480E00895E091B708F091B808E75BFE4F80818C9381E027
:2004E00008958A3010F080E00895E091B708F091B808E75BFE4F808381E00895FC01009713
:2005000011F480E008958091210984FF03C080E69BE002C080EB95E09183808381E00895C0
:20052000EF92FF920F931F93009779F10E94EB15882359F12091D0023091D1024091D20201
:200540005091D3028091210984FF06C0E12CF12C92E0092F112D05C0E12CF12C81E0082FC8
:20056000112D2F5F3F4F4F4F5F4FCA01B901A80197010E9427756093D0027093D102809323
:20058000D2029093D30281E001C080E01F910F91FF90EF900895EF92FF920F931F93DF933A
:2005A000CF930F92CDB7DEB7982F8091EC07813079F5992369F1CE0101960E94EB15209166
:2005C000D0023091D1024091D2025091D3022F5F3F4F4F4F5F4F8091210984FF06C0E12C61
:2005E000F12C72E0072F112D05C0E12CF12C61E0062F112DCA01B901A80197010E94277571
:200600006093D0027093D1028093D2029093D3020E9491151092EC0781E00F90CF91DF91B3
:200620001F910F91FF90EF9008958091EC07882311F00E9491151092EC0781E00895682F9D
:200640001092DC022091D4023091D5024091D6025091D7028091210984FF05C083ED9FEF17
:20066000A1E0B0E004C083ED9FEFA0E0B0E082179307A407B50778F41092D4021092D502A0
:200680001092D6021092D702662329F40E9415031092840A03C082E08093840A81E0089511
:2006A000EF92FF920F931F937B018C018091EC07813019F40E94CB0204C0823011F40E947D
:2006C00015030E945915882351F40E9491150E945915882321F40E945915882399F1809194
:2006E000210984FF05C08FEF9FEFA0E0B0E004C08FEF9FE7A0E0B0E08E159F05A007B107EE
:2007000010F080EA01C082EA0E9495158823D1F0BB27A12F902F8F2D0E949515882391F0E5
:200720008E2D0E949515882369F0E092D002F092D1020093D2021093D30282E08093EC07CE
:2007400081E001C080E01F910F91FF90EF900895EF92FF920F931F937B018C010E945003B8
:20076000882379F10E948E15882331F40E9491150E948E15882329F18091210984FF05C07A
:200780008FEF9FEFA0E0B0E004C08FEF9FE7A0E0B0E08E159F05A007B10710F081EA01C093
:2007A00083EA0E949515882361F0E092D002F092D1020093D2021093D30281E08093EC07A5
:2007C00001C080E01F910F91FF90EF900895EF92FF920F931F93CF93DF93009709F45CC013
:2007E0000E94CC15882309F457C02091D0023091D1024091D2025091D3028091210990E09A
:20080000EC01C071D07084FF06C0E12CF12CA2E00A2F112D05C0E12CF12CF1E00F2F112DD2
:200820002F5F3F4F4F4F5F4FCA01B901A80197010E9427759B01AC012093D0023093D102E8
:200840004093D2025093D302CD2B41F5211531054105510529F02050304840405040F1F40D
:2008600081E00E94CB026091D0027091D1028091D2029091D3026150704080409040609352
:20088000D0027093D1028093D2029093D3020E94A803882321F002C080E001C081E0DF9114
:2008A000CF911F910F91FF90EF9008950F931F93CF93DF93EC01162F042F0097D1F41DC017
:2008C000123010F4002349F4CE010E94E703882371F4CE010E94E70308C0CE010E949002E1
:2008E000882329F4CE010E949002882331F011502196112329F781E001C080E0DF91CF91A3
:200900001F910F910895482F8FEE97E06DE20E9456048823A1F08091D8029091D902A091E0
:20092000DA02B091DB028D96A11DB11D8093D8029093D902A093DA02B093DB0281E00895F6
:200940002091D8023091D9024091DA025091DB028091D0029091D102A091D202B091D30213
:20096000281739074A075B0721F48091EC07813091F08091EC07813011F40E94CB026091E0
:20098000D8027091D9028091DA029091DB020E94A803882319F081E08093840A0895109274
:2009A000D8021092D9021092DA021092DB020E94A0040895EF92FF920F931F93CF93DF93C6
:2009C0000E949515882309F449C02091D0023091D1024091D2025091D3028091210990E0FD
:2009E000EC01C071D07084FF06C0E12CF12C82E0082F112D05C0E12CF12CB1E00B2F112D57
:200A00002F5F3F4F4F4F5F4FCA01B901A80197010E9427759B01AC012093D0023093D10206
:200A20004093D2025093D302CD2BB9F4211531054105510529F0205030484040504069F43C
:200A40000E9415036091D0027091D1028091D2029091D3020E94500301C081E0DF91CF9183
:200A60001F910F91FF90EF9008951F93CF93DF93EC01162F009769F410C088810E94DA0476
:200A8000882329F488810E94DA04882331F021961150112391F781E001C080E0DF91CF9113
:200AA0001F9108951F938091840A8230E1F0813009F04AC02091DC028091D4029091D502F3
:200AC000A091D602B091D702821B9109A109B1098093D4029093D502A093D602B093D7024E
:200AE0001092840A31C02091DC022D3258F5822F90E009968E9710F419E002C01DE2121BCA
:200B0000822F90E08151984F612F0E9435058823D9F08091DC02810F8093DC028091D402C4
:200B20009091D502A091D602B091D702810F911DA11DB11D8093D4029093D502A093D602E2
:200B4000B093D70281E001C080E01F9108950F931F93DF93CF9300D000D000D0CDB7DEB7F9
:200B60002091D4023091D5024091D6025091D7028091D0029091D102A091D202B091D30201
:200B8000281739074A075B0721F48091EC07823039F0CA01B9010E945003882309F4B7C195
:200BA00000910A0110910B0120919C0A30919D0A200F311F54E0220F331F5A95E1F730936D
:200BC000F4078091E10A9091E20AA801481B590BCA019F70292B2093F5078093F60782E052
:200BE00061E041E00E94EA589801281B390B44E0220F331F4A95E1F73093F70780917808DF
:200C000090917908800F911F9F70292B2093F8078093F907CE010196BE016D5F7F4FAE015D
:200C20004B5F5F4F0E94FA5E8091600C682F80FF07C089819A81909581959F4F9A83898391
:200C400049815A814150584F34E0440F551F3A95E1F75093EF0761FF07C08B819C819095E7
:200C600081959F4F9C838B838FEF97E02B813C81821B930B9F70292F242B2093F007809337
:200C8000F10762FF07C08D819E81909581959F4F9E838D838D819E818150984F24E0880F2D
:200CA000991F2A95E1F79093F20720917F0A282B2093F3072091C90A3091CA0A200F311FF7
:200CC00094E0220F331F9A95E1F73093FA078091CB0A9091CC0A800F911F9F70292B209320
:200CE000FB078093FC072091CD0A3091CE0A200F311F84E0220F331F8A95E1F73093FD0797
:200D00008091D30A9091D40A800F911F9F70292B2093FE078093FF0780910E0B90910F0B0E
:200D20009801281B390BB4E0220F331FBA95E1F7309300088091100B9091110BA801481B15
:200D4000590BCA019F70292B20930108809302088091120B9091130B9801281B390BA4E017
:200D6000220F331FAA95E1F7309303088091180B9091190BA801481B590BCA019F70292BF4
:200D800020930408809305082091A3083091A408200F311FF4E0220F331FFA95E1F73093AB
:200DA00006088091A5089091A608800F911F9F70292B20930708809308082091A7083091F0
:200DC000A808200F311FE4E0220F331FEA95E1F7309309088091AB089091AC08800F911F9A
:200DE0009F70292B20930A0880930B082091D70A3091D80A200F311F74E0220F331F7A950B
:200E0000E1F730930C088091B1089091B208800F911F9F70292B20930D0880930E088091DA
:200E2000AD089091AE089801281B390B64E0220F331F6A95E1F730930F088091AF089091A5
:200E4000B008800F911F9F70292B20931008809311082091D50A3091D60A200F311F54E05D
:200E6000220F331F5A95E1F73093120880911A0B90911B0BA801481B590BCA019F70292B30
:200E8000209313088093140880910D0B992787FD9095800F911F44E0880F991F4A95E1F75A
:200EA0009093150880931608CE010196BE016D5F7F4FAE014B5F5F4F0E94105F49815A8145
:200EC0004150584F34E0440F551F3A95E1F7509317088FEF97E02B813C81821B930B9F70AE
:200EE000292F242B20931808809319088D819E818150984F24E0880F991F2A95E1F7909352
:200F00001A0880931B0882E08093840A81E026960FB6F894DEBF0FBECDBFCF91DF911F9192
:200F20000F9108951092DC020E94A70508954091360B5091370B2091380B3091390B421782
:200F400053074CF44817590714F020E00EC08217930754F407C02817390734F420E08417E2
:200F600095071CF421E001C022E0822F0895CF93DF93FC0181E090E0A0E0B0E08093C7081F
:200F80009093C808A093C908B093CA08309709F491C282E090E0A0E0B0E08093C708909347
:200FA000C808A093C908B093CA0861817281DF01119620E030E0AF01485B5E4F12968C9117
:200FC00012972827822F82958227082E869586958025082E869580258770022E232F86950D
:200FE00007948795302D282706948795302528271196A417B50711F76217730709F05AC206
:2010000083E090E0A0E0B0E08093C7089093C808A093C908B093CA088381883008F04AC23F
:2010200084E090E0A0E0B0E08093C7089093C808A093C908B093CA08DF0190E014968C91C7
:20104000149783588B3F28F085E090E0A0E0B0E0DCC018968C91189783588B3F28F086E00A
:2010600090E0A0E0B0E0D1C01C968C911C9783588B3F28F087E090E0A0E0B0E0C6C09F5FB5
:2010800011969430D9F688E090E0A0E0B0E08093C7089093C808A093C908B093CA08808937
:2010A000813808F007C289E090E0A0E0B0E08093C7089093C808A093C908B093CA088189D5
:2010C000813808F0F7C18AE090E0A0E0B0E08093C7089093C808A093C908B093CA088289C4
:2010E000813808F0E7C18BE090E0A0E0B0E08093C7089093C808A093C908B093CA088389B2
:20110000887F09F0D7C18CE090E0A0E0B0E08093C7089093C808A093C908B093CA08848950
:20112000813808F0C7C18DE090E0A0E0B0E08093C7089093C808A093C908B093CA0885898D
:20114000807709F0B7C18EE090E0A0E0B0E08093C7089093C808A093C908B093CA0886893C
:201160009789865E994F85539C4008F0A3C18FE090E0A0E0B0E08093C7089093C808A0937C
:20118000C908B093CA08808D918D865E994F85539C4008F08FC180E190E0A0E0B0E0809382
:2011A000C7089093C808A093C908B093CA08828D938D23EC8035920731F4DF015D96EF01E0
:2011C000A59620E005C0885A914609F073C1F5CF8C918E3728F081E190E0A0E0B0E015C0B4
:2011E00014968C9114978E3728F082E190E0A0E0B0E00BC0888199818C509E4F895E93404C
:2012000068F083E190E0A0E0B0E08093C7089093C808A093C908B093CA084CC12F5F119662
:2012200022962430A9F684E190E0A0E0B0E08093C7089093C808A093C908B093CA0886A505
:2012400097A523EC8035920781F031E6883A930761F027E28031920741F032E282349307D8
:2012600021F08C549D4109F025C185E190E0A0E0B0E08093C7089093C808A093C908B093BE
:20128000CA0883A994A93EE0863A930741F029E08830920721F08C56974009F00BC186E11A
:2012A00090E0A0E0B0E08093C7089093C808A093C908B093CA0881A98E3708F0FBC087E1B6
:2012C00090E0A0E0B0E08093C7089093C808A093C908B093CA0882A98E3708F0EBC088E1A4
:2012E00090E0A0E0B0E08093C7089093C808A093C908B093CA0885A996A98C509E4F895E63
:20130000934008F0D7C089E190E0A0E0B0E08093C7089093C808A093C908B093CA0887A963
:20132000823008F0C7C08AE190E0A0E0B0E08093C7089093C808A093C908B093CA08DF01C3
:20134000D89620E08D919C9111978552964008F0B1C02F5F12962438A9F78DE190E0A0E086
:20136000B0E08093C7089093C808A093C908B093CA08E05CFE4F8081E054F140887F09F000
:2013800099C08EE190E0A0E0B0E08093C7089093C808A093C908B093CA08EA5BFE4F808184
:2013A000E654F140807F09F085C08FE190E0A0E0B0E08093C7089093C808A093C908B09379
:2013C000CA08EE5BFE4F80819181E254F140865E994F85539C4008F06DC080E290E0A0E034
:2013E000B0E08093C7089093C808A093C908B093CA08EF5BFE4F8081E154F140823008F0C7
:2014000059C081E290E0A0E0B0E08093C7089093C808A093C908B093CA08EC5BFE4F80814D
:201420009181E454F140885E9340815A9F4008F041C082E290E0A0E0B0E08093C7089093DC
:20144000C808A093C908B093CA08E95BFE4F8081E754F140887F71F584E290E0A0E0B0E052
:201460008093C7089093C808A093C908B093CA08E85BFE4F8081E854F140807ED9F485E24E
:2014800090E0A0E0B0E08093C7089093C808A093C908B093CA08E75BFE4F80818A3050F450
:2014A0001092C7081092C8081092C9081092CA0881E001C080E0DF91CF910895CF93DF939F
:2014C000FC0185E690E0A0E0B0E08093C7089093C808A093C908B093CA08309709F485C528
:2014E00086E690E0A0E0B0E08093C7089093C808A093C908B093CA0861817281DF011196B6
:2015000020E030E0AF014F585F4F12968C9112972827822F82958227082E86958695802577
:20152000082E869580258770022E232F869507948795302D282706948795302528271196BD
:20154000A417B50711F76217730709F04EC58AE690E0A0E0B0E08093C7089093C808A09315
:20156000C908B093CA088381823008F03EC58BE690E0A0E0B0E08093C7089093C808A093DB
:20158000C908B093CA088481813808F02EC58CE690E0A0E0B0E08093C7089093C808A093C2
:2015A000C908B093CA08EF01DF0190E015968C911597853008F019C59F5F11969830B1F7F1
:2015C0008DE690E0A0E0B0E08093C7089093C808A093C908B093CA08DF0190E01D968C910A
:2015E0001D97813808F001C59F5F11969830B1F78EE690E0A0E0B0E08093C7089093C808E2
:20160000A093C908B093CA088589813808F0EDC48FE690E0A0E0B0E08093C7089093C80877
:20162000A093C908B093CA088689813808F0DDC480E790E0A0E0B0E08093C7089093C80874
:20164000A093C908B093CA088789813808F0CDC481E790E0A0E0B0E08093C7089093C80862
:20166000A093C908B093CA08808D813808F0BDC482E790E0A0E0B0E08093C7089093C80854
:20168000A093C908B093CA08818D813808F0ADC483E790E0A0E0B0E08093C7089093C80842
:2016A000A093C908B093CA08828D813808F09DC484E790E0A0E0B0E08093C7089093C80830
:2016C000A093C908B093CA08838D813808F08DC485E790E0A0E0B0E08093C7089093C8081E
:2016E000A093C908B093CA08848D813808F07DC486E790E0A0E0B0E08093C7089093C8080C
:20170000A093C908B093CA08858D813808F06DC487E790E0A0E0B0E08093C7089093C808F9
:20172000A093C908B093CA08868D813808F05DC488E790E0A0E0B0E08093C7089093C808E7
:20174000A093C908B093CA08878D823008F04DC489E790E0A0E0B0E08093C7089093C808DC
:20176000A093C908B093CA0890E088A1813808F03CC49F5F21969930C1F78AE790E0A0E06F
:20178000B0E08093C7089093C808A093C908B093CA0881A5813808F028C48BE790E0A0E0A6
:2017A000B0E08093C7089093C808A093C908B093CA0882A5813208F018C48CE790E0A0E09A
:2017C000B0E08093C7089093C808A093C908B093CA0883A5813808F008C48DE790E0A0E082
:2017E000B0E08093C7089093C808A093C908B093CA0884A5813808F0F8C38EE790E0A0E071
:20180000B0E08093C7089093C808A093C908B093CA0885A5813808F0E8C38FE790E0A0E05E
:20182000B0E08093C7089093C808A093C908B093CA0886A5813808F0D8C380E890E0A0E05B
:20184000B0E08093C7089093C808A093C908B093CA0887A583588B3F08F0C7C381E890E0DE
:20186000A0E0B0E08093C7089093C808A093C908B093CA0880A9813808F0B7C382E890E03C
:20188000A0E0B0E08093C7089093C808A093C908B093CA0881A9813808F0A7C383E890E02A
:2018A000A0E0B0E08093C7089093C808A093C908B093CA0882A9813808F097C384E890E018
:2018C000A0E0B0E08093C7089093C808A093C908B093CA0883A9813808F087C385E890E006
:2018E000A0E0B0E08093C7089093C808A093C908B093CA0884A9813808F077C386E890E0F4
:20190000A0E0B0E08093C7089093C808A093C908B093CA0885A9813808F067C387E890E0E1
:20192000A0E0B0E08093C7089093C808A093C908B093CA0886A9813808F057C388E890E0CF
:20194000A0E0B0E08093C7089093C808A093C908B093CA0887A9823008F047C389E890E0C4
:20196000A0E0B0E08093C7089093C808A093C908B093CA08DF01D89690E08C91813808F0DD
:2019800034C39F5F11969930C1F78AE890E0A0E0B0E08093C7089093C808A093C908B0931C
:2019A000CA08EF5BFF4F8081E154F040813808F01CC38BE890E0A0E0B0E08093C7089093CF
:2019C000C808A093C908B093CA08EE5BFF4F8081E254F040813208F008C38CE890E0A0E046
:2019E000B0E08093C7089093C808A093C908B093CA08ED5BFF4F8081E354F040813808F0BA
:201A0000F4C28DE890E0A0E0B0E08093C7089093C808A093C908B093CA08EC5BFF4F808197
:201A2000E454F040813808F0E0C28EE890E0A0E0B0E08093C7089093C808A093C908B093D9
:201A4000CA08EB5BFF4F8081E554F040813808F0CCC28FE890E0A0E0B0E08093C70890937B
:201A6000C808A093C908B093CA08EA5BFF4F8081E654F040813808F0B8C280E990E0A0E0FB
:201A8000B0E08093C7089093C808A093C908B093CA08E95BFF4F8081E754F040813808F019
:201AA000A4C281E990E0A0E0B0E08093C7089093C808A093C908B093CA08E75AFF4F808158
:201AC000E955F040813808F090C282E990E0A0E0B0E08093C7089093C808A093C908B0938E
:201AE000CA08E65AFF4F8081EA55F040813208F07CC283E990E0A0E0B0E08093C70890933C
:201B0000C808A093C908B093CA08E85BFF4F8081E854F040813808F068C284E990E0A0E0A6
:201B2000B0E08093C7089093C808A093C908B093CA08E75BFF4F8081E954F040813808F078
:201B400054C285E990E0A0E0B0E08093C7089093C808A093C908B093CA08E65BFF4F808103
:201B6000EA54F040813808F040C286E990E0A0E0B0E08093C7089093C808A093C908B09339
:201B8000CA08E55BFF4F8081EB54F040813808F02CC287E990E0A0E0B0E08093C7089093E1
:201BA000C808A093C908B093CA08E45BFF4F8081EC54F040813808F018C288E990E0A0E052
:201BC000B0E08093C7089093C808A093C908B093CA08E35BFF4F8081ED54F040813808F0D8
:201BE00004C289E990E0A0E0B0E08093C7089093C808A093C908B093CA08E25BFF4F8081B3
:201C0000EE54F040805F813208F0EFC18AE990E0A0E0B0E08093C7089093C808A093C9084C
:201C2000B093CA08E15BFF4F8081EF54F040805F813208F0DAC18BE990E0A0E0B0E0809365
:201C4000C7089093C808A093C908B093CA08E05BFF4F8081E055F040805F813208F0C5C1AA
:201C60008CE990E0A0E0B0E08093C7089093C808A093C908B093CA08EF5AFF4F8081E155B3
:201C8000F040805F813208F0B0C18DE990E0A0E0B0E08093C7089093C808A093C908B09307
:201CA000CA08EE5AFF4F8081E255F040813808F09CC18EE990E0A0E0B0E08093C70890934A
:201CC000C808A093C908B093CA08ED5AFF4F8081E355F040813808F088C18FE990E0A0E0BB
:201CE000B0E08093C7089093C808A093C908B093CA08EC5AFF4F8081E455F040813208F0BD
:201D000074C180EA90E0A0E0B0E08093C7089093C808A093C908B093CA08EB5AFF4F808122
:201D2000E555F04083588B3F08F05FC181EA90E0A0E0B0E08093C7089093C808A093C908B8
:201D4000B093CA08EA5AFF4F8081E655F04083588B3F08F04AC182EA90E0A0E0B0E08093C9
:201D6000C7089093C808A093C908B093CA08E95AFF4F8081E755F04083588B3F08F035C1F7
:201D800083EA90E0A0E0B0E08093C7089093C808A093C908B093CA08E85AFF4F8081E8559A
:201DA000F040823008F021C184EA90E0A0E0B0E08093C7089093C808A093C908B093CA088B
:201DC000E55AFF4F8081EB55F0408E7F09F00DC185EA90E0A0E0B0E08093C7089093C8086D
:201DE000A093C908B093CA08E45AFF4F80819181EC55F040815D974008F0F7C086EA90E076
:201E0000A0E0B0E08093C7089093C808A093C908B093CA08E25AFF4F80819181EE55F040B4
:201E20008058934F8150994108F0DFC087EA90E0A0E0B0E08093C7089093C808A093C908DC
:201E4000B093CA08E05AFF4F80819181E056F0408058934F8150994108F0C7C088EA90E0A6
:201E6000A0E0B0E08093C7089093C808A093C908B093CA08EE59FF4F80819181E256F04054
:201E8000805C904E81589E4308F0AFC089EA90E0A0E0B0E08093C7089093C808A093C9089B
:201EA000B093CA08EC59FF4F8081E456F0408E7F09F09BC08AEA90E0A0E0B0E08093C708D8
:201EC0009093C808A093C908B093CA08EB59FF4F80819181E556F0408050914F81509E4186
:201EE00008F083C08BEA90E0A0E0B0E08093C7089093C808A093C908B093CA08E959FF4F34
:201F000080819181E756F0408050914F81509E4108F06BC08CEA90E0A0E0B0E08093C708E6
:201F20009093C808A093C908B093CA08E759FF4F80819181E956F0408050914F81509E4125
:201F400008F053C08DEA90E0A0E0B0E08093C7089093C808A093C908B093CA08E559FF4F05
:201F600080819181EB56F0408050914F81509E41E0F58EEA90E0A0E0B0E08093C7089093AB
:201F8000C808A093C908B093CA08E359FF4F8081ED56F040813848F5E259FF4F8081EE5696
:201FA000F040813810F58FEA90E0A0E0B0E08093C7089093C808A093C908B093CA08E05913
:201FC000FF4F8081E057F040883078F4EF58FF4F8081883050F41092C7081092C808109210
:201FE000C9081092CA0881E001C080E0DF91CF9108956F708295807F860F0895FB01DA01AF
:20200000982F92959F7090838F708C930895682F83E090E00E94C9750895682F80E090E0A7
:202020000E94C975089583EB92E060E00E94C975089584EB92E060E00E94C975089584EB79
:2020400092E060E00E94C97583EB92E060E00E94C975089583E090E00E94AB75089580E0BF
:2020600090E00E94AB75089584EB92E00E94AB75089583EB92E00E94AB7508950F931F93BE
:2020800004EB12E0C8010E94AB75682F6F5FC8010E94C9751F910F91089583EB92E00E9457
:2020A000AB75882311F46FEF02C0682F615083EB92E00E94C975089583EB92E00E94AB75E9
:2020C0008F3F11F460E002C0682F6F5F83EB92E00E94C9750895BC0181E090E00E94D775ED
:2020E000089581E090E00E94B37508950F931F93CF93DF930E942C6F0E94416F40918F0AEA
:202100005091900A8091210990E0BC016870707083FF03C020E030E002C020EF33E0CA0120
:20212000821B930B9C0197FF03C0309521953F4F283731050CF44BC04091910A5091920ADC
:202140006115710519F020E030E002C020EF33E0CA01821B930B9C0197FF03C0309521951F
:202160003F4F283731059CF14091930A5091940A6115710519F020E030E002C020EF33E0D9
:20218000CA01821B930B9C0197FF03C0309521953F4F28373105DCF0672B19F080E090E06E
:2021A00002C080EF93E09093940A8093930A9093920A8093910A9093900A80938F0A8FE8BD
:2021C0009AE06DEA72E046E050E00E94BF7583E00E94B86A80E06CE64FE32DE70E94396B4B
:2021E00081E060E043E82DE70E94396B82E064E94FE32DE70E94396B83E060E040E020E0BB
:202200000E94396B87E30E94546B87E30E94796B87E30E94016C80E00E94715882E00E9475
:202220008A588FE89DEF0E94A35881E792E00E94C25880E00E945F5880E593EC0E946F5B7D
:2022400080E060E00E942F5B81E060E00E942F5B82E060E00E942F5B83E060E00E942F5B48
:2022600080E060E070E00E94D25B80E064E60E94905B80E064E60E94B15B81E060E070E01F
:202280000E94D25B81E064E60E94905B81E064E60E94B15B82E060E070E00E94D25B82E0BB
:2022A00064E60E94905B82E064E60E94B15B83E060E070E00E94D25B83E064E60E94905BF1
:2022C00083E064E60E94B15B82E00E94D95D8CE49DE10E94385D86EA9EE00E94955D80E062
:2022E0000E941B5D80E090E00E94BA5D84E60E947D5D84E60E94655D80E00E94715E10E0C6
:20230000C0E0D0E0812FBE010E948E5E1F5F2C961438C1F7E091B708F091B808E05CFE4F32
:20232000108281E00E94714581E00E945D4581E00E94494580E00E94374580E090E00E942C
:20234000944580E00E94854588E998E00E94274580E00E94DB5F8091210983FF03C060E0E5
:2023600070E002C060EF73E080E00E94695F8091210983FF03C060E070E002C060EF73E06B
:2023800081E00E94695F8091210983FF03C060E070E002C060EF73E082E00E94695F81E0D1
:2023A0000E94710280E00E94540210E00E94416F812F61E00E94916B812F64E60E94EB6BED
:2023C000812F60E043E00E943A59812F61E044E00E943A59812F62E041E00E943A59812F73
:2023E00063E043E00E943A59812F64E043E00E943A59812F65E043E00E943A59812F66E0B3
:2024000040E00E943A59812F67E040E00E943A59812F60E04AE00E944E56812F61E04AE0A0
:202420000E944E56812F62E040E00E944E56812F63E040E00E944E56812F64E04AE00E94E5
:202440004E56812F65E040E00E944E56812F66E040E00E944E56812F67E040E00E944E56C4
:20246000812F6FE00E942957812F6FE00E945857812F64E10E948757812F64E10E94764821
:20248000812F63E20E945E48812F68E00E944648812F60E50E942E48812F60E50E941648D5
:2024A000812F68E20E94FE47812F60E50E94E647812F60E00E94CE4700E0812F602F40E889
:2024C0000E94C43A0F5F0930C1F7812F64E040E50E94C43A812F60E40E94B647812F64E1BC
:2024E0000E948647812F66E00E949E47812F63E20E946E47812F60E50E945647812F60E47C
:202500000E943E47812F60E00E942447812F6EE10E940C47812F63E20E94F446812F68E0DA
:202520000E94DC46812F60E50E94C446812F60E50E94AC46812F68E20E949446812F60E542
:202540000E947C46812F60E00E94644600E0812F602F40E80E94723C0F5F0930C1F7812F35
:2025600064E040E50E94723C812F60E40E944C46812F64E10E941C46812F66E00E9434466F
:20258000812F60E40E94DB3C812F63E20E940446812F60E50E94EC45812F60E40E94D44536
:2025A000812F60E00E94BC45812F68E00E94A445812F68E20E943F44812F6EE10E942744DA
:2025C000812F68E00E940F44812F65E00E94F743812F60E50E94DF43812F6CE30E94C743D9
:2025E000812F60E00E94AD43812F60E00E949343812F60E00E947943812F60E00E945F436F
:20260000812F60E80E944743812F60E40E942F43812F68E00E941743812F64E10E94FD42C4
:20262000812F64E10E94E342812F68E20E94C942812F61E00E94A43F812F60E00E940340EC
:20264000812F60E070E00E943340812F60E070E00E946740812F60E070E00E94AA40812F20
:2026600060E070E00E94ED40812F60E00E943041812F60E070E00E946041812F60E070E035
:202680000E94A141812F60E070E00E94E241812F60E070E00E942342812F60E042E00E94B6
:2026A000B05F812F61E042E00E94B05F812F62E042E00E94B05F812F60E044E00E9411605B
:2026C000812F61E044E00E941160812F62E042E00E9411601F5F133009F068CE0E94356F75
:2026E000DF91CF911F910F91089587E18093200BE0E2FBE020E030E083812827822F8295AF
:202700008227082E869586958025082E869580258770022E232F869507948795302D282712
:20272000069487953025282731968CE0E736F80719F73093220B2093210B0E942C6F80E272
:202740009BE06DE571E04AE451E00E94BF750E94356F0895CF93DF93682F833008F054C019
:20276000A82FB0E083E790E0A89FF001A99FF00DB89FF00D1124EE5DF64F87E1808383E7AD
:20278000689FE0011124CE018E5D964FFC01319620E030E0AC014F585F4F82812827822FA4
:2027A00082958227082E869586958025082E869580258770022E232F869507948795302DAA
:2027C000282706948795302528273196E417F50721F783E790E0A89FF001A99FF00DB89FCC
:2027E000F00D1124EE5DF64F328321830E942C6FBE016C5F7F4FCE018E5D964F43E750E030
:202800000E94BF750E94356FDF91CF91089580E00E94AA1381E00E94AA1382E00E94AA13EF
:202820000895DF92EF92FF920F931F93CF93DF93D82EC82FD0E083E790E0C89F7001C99F89
:20284000F00CD89FF00C112487010E5D164F045A1F4FF801619171918F01C701805A9F4FA3
:202860000E94B975F801619171918F01C7018E599F4F0E94B9750E94416FF801619171915F
:202880008F01C7018C599F4F0E94B975F80160817181C7018A599F4F0E94B9750E94416FB6
:2028A0000D5F1F4FF801619171918F01C70187599F4F0E94B975F801619171918F01C70116
:2028C00085599F4F0E94B9750E94416FF801619171918F01C70183599F4F0E94B975F80132
:2028E00060817181C70181599F4F0E94B9750E94416F83E7D89EC00111248E5D964FFC01B0
:20290000319660E070E09C012F583F4F82816827862F82958627082E869586958025082E5C
:20292000869580258770062E672F869507948795702D682706948795702568273196E2177E
:20294000F30721F783E790E09C01C29FC001C39F900DD29F900D1124FC01EE5DF64F728308
:2029600061838B5F9F4F0E94B975DF91CF911F910F91FF90EF90DF9008950E942C6F80E2F2
:202980009BE06DE571E04AE451E00E949B750E94356F089582E299E064E070E049E551E055
:2029A0000E949B750895CF93DF931092B6081092B5081092C00810921C0883E090E00E9490
:2029C000AB75809321090E94BD1480E29BE09093B8088093B70882E299E064E070E049E5F6
:2029E00051E00E949B758091B7089091B8080E94B707882379F0C2E2D9E0CE010E945E0A99
:202A0000882341F0CD58DF4F8AE0CB37D807A9F781E001C080E0DF91CF910895CF93DF93D9
:202A200023E7829F900111242E5D364F3093BF082093BE0880937F0AC0E0D0E0E091BE086F
:202A4000F091BF08EC0FFD1F80917F0A6C2F45810E943A592196C830D10581F7E091BE08B3
:202A6000F091BF08E059FF4F80917F0A60E040810E941160E091BE08F091BF08EF58FF4FC5
:202A800080917F0A61E040810E941160E091BE08F091BF08EE58FF4F80917F0A62E04081D7
:202AA0000E9411600E94AF440E946442DF91CF91089584EA8093BC0020E030E007C0223350
:202AC000310511F480E008952F5F3F4F8091BC0087FFF5CF9091B900987F983011F481E06C
:202AE000089580E0903109F481E00895FF920F931F931092B90081E18093B8000CEB10E0C9
:202B000084E0F801808384E9F82EF0820E945915F801F0821F910F91FF9008950E94591549
:202B2000089584E98093BC0008958093BB0084E88093BC0020E030E008C083E0283E380736
:202B400011F480E008952F5F3F4F8091BC0087FFF4CF9091B900987F983239F0983129F07B
:202B600080E0903419F481E0089581E008950F931F93182F04E9812F90E00E9459158823C5
:202B8000D1F3812F0E949515882319F40093BC00F2CF1F910F910895FC010097D1F084ECFB
:202BA0008093BC0020E030E006C083E0283E380781F02F5F3F4F8091BC0087FFF6CF8091B2
:202BC000B900887F803529F48091BB00808381E0089580E00895FC0184E88093BC0020E061
:202BE00030E006C083E0283E380781F02F5F3F4F8091BC0087FFF6CF8091B900887F8835C4
:202C000029F48091BB00808381E0089580E00895DF93CF93CDB7DEB728970FB6F894DEBF33
:202C20000FBECDBF9E012F5F3F4F0E948E6969817A8180E00E94025C6B817C8181E00E94B6
:202C4000025C6D817E8182E00E94025C80912009882329F08091350B8178813829F06F81BD
:202C6000788583E00E94025C28960FB6F894DEBF0FBECDBFCF91DF9108952F923F924F920F
:202C80005F926F927F928F929F92AF92BF92CF92DF92EF92FF920F931F93DF93CF93CDB7BD
:202CA000DEB7CD54D0400FB6F894DEBF0FBECDBF1A8219821C821B821E821D8218861F8217
:202CC0000E94CD70182F78940E94FE6F80E090E00E94197080E090E00E942170012F10E095
:202CE00003FF03C082E00E94436F9801247030702C963FAF2EAF2C9702FF05C000FD03C0B6
:202D000083E00E94436F84E190E80E94046D89EB98E066E278E040E50E94B86E8CEC9CEC93
:202D20000E9421700E942F108093ED07A8014170507059A348A300FF07C0803229F085E081
:202D40000E94436F1BA602C051E05BA70E94D314882341F488A199A1892B09F01BA681E0CE
:202D60000E94436F8091210987FF04C086E00E94436F1BA68091210983FF0DC00E94761548
:202D8000C80185709070892B31F08091210981FF02C00E942F028091210983FD0AC0057056
:202DA0001070012B31F081FF04C00E9476150E942F028091210983FD0DC0A8A1B9A1AB2B01
:202DC00031F082FF02C082E003C081E001C080E00E945A690E94526297FF08C084E00E94C9
:202DE000436FE8A1F9A1EF2B09F01BA60E94416F28A139A1232BA9F010E08FE493EC0197D4
:202E0000F1F700C000000E94416F1F5F1436A9F70E94BB60882341F484E00E94436F1BA63A
:202E200003C00E945F601FC00E94416F10E017C02FE738E341E0215030404040E1F700C02B
:202E400000000E94416F8FE798E3A1E081509040A040E1F700C000000E94416F1F5F8091B4
:202E6000340B181728F31092EE070E94C55A0E94EE59882311F41BA607C09BA5992321F043
:202E80008AEA9AEA0E9421700E94AF440E94644210921F0910921E091092830A1092820A3A
:202EA0001092960A1092950A1092C4081092C308A09108012D96AFAF2D97B09109012E9686
:202EC000BFAF2E972A961FAE2A9729961FAE299728961FAE289727961FAE279726961FAE0A
:202EE0001EAE269724961FAE1EAE24972224332422961FAE1EAE22971FAE1EAE1DAE1CAE66
:202F00001BAE1AAE19AE18AE1FAA1EAA1DAA1CAA1BAA1AAA19AA18AA1FA61EA6E1E0EAA78C
:202F2000E9A718A61FA21EA21DA2662477241CA21BA21AA20E94416F8091990A8823D1F332
:202F400020918400309185003DA72CA7CE01479661E041E021E00E949160892B01F139A519
:202F6000332329F028961FAE289719A657C028964FAD2897423328F44F5F28964FAF28978F
:202F80004DC058A5552309F049C08FEF9FEF0E94197080E00E94516981E088A73FC099A5ED
:202FA000992321F428961FAE289712C02896AFAD2897A43128F4AF5F2896AFAF289708C0A9
:202FC000B8A5BB2329F080E090E00E94197018A68091B5089091B6082B8D3C8D820F931F73
:202FE0009093B6088093B508442737FD4095542F8091DB0A9091DC0AA091DD0AB091DE0AEB
:20300000820F931FA41FB51F8093DB0A9093DC0AA093DD0AB093DE0AE1E0E9A7FBA5FF237D
:2030200009F465C48091EE07882379F580916A0C853058F128A139A1232B51F080E00E9492
:20304000665981E00E94665984E00E94665902C00E94D45983E060E041E00E94EA58229639
:203060009FAF8EAF22970E9497070E940E1530917F0A2A963FAF2A970E94455E8FEF9FEFFD
:203080000E94217081E08093EE0727964FAD2797842E9924C40183709070892B09F058C031
:2030A0008091EE078823B9F084E061E041E00E94EA589BAF8AAF85E060E041E00E94EA58DF
:2030C00099AF88AF82E060E041E00E94EA5822243324281A390AE091BE08F091BF08878919
:2030E0006AAD7BAD4EA55FA50E94DB57B82EA92E58A5552391F46AAD7BADAE01495E5F4FCC
:2031000091010091660CE8ACF9AC17E0C12ED12CCC0EDD1E0E9496480AC06EA97FA94CA9AB
:203120005DA991018E01095F1F4F0E949E388091C008882321F080911C08882321F48F8180
:2031400098850E94ED5D8B2D9A2D9C013FA72EA7BFE04B2E512C4820592081E04816510405
:2031600009F071C08091EE07882309F447C080E061E041E00E94EA5826969FAF8EAF2697C6
:2031800081E061E041E00E94EA5824969FAF8EAF249782E060E041E00E94EA582224332444
:2031A000281A390A83E060E041E00E94EA5822969FAF8EAF229785E060E041E00E94EA583C
:2031C00099AF88AF80912009882351F42D962FAD2D972E963FAD2E97C9019FAF8EAF0CC04D
:2031E00086E060E040E00E94EA589FAF8EAF87E060E040E00E94EA589DAF8CAFE091BE0831
:20320000F091BF08858926966EAD7FAD26974AA95BA90E9433589FAB8EABE091BE08F09139
:20322000BF08868924966EAD7FAD249748A959A90E9407589DAB8CABAEA9BFA9BBABAAAB0F
:2032400099AB88AB76C0B2E04B16510411F5E8A5EE23D9F48EA99FA926966EAD7FAD2697C9
:20326000A1012091660C08AD19ADA7E1EA2EF12CEC0EFD1E6E010894C11CD11CF5EBAF2EAA
:20328000F8E0BF2E0E94D6516CC22EA93FA93A83298333E04316510451F548A5442309F5F1
:2032A0008CA99DA924966EAD7FAD2497A1012091660C08AD19ADE7E1EE2EF12CEC0EFD1E81
:2032C00033E0C32ED12CCC0EDD1EB5E0AB2EB12CAC0EBD1EA5EB8A2EA8E09A2E0E94AD4E03
:2032E00040C28CA99DA99C838B833E822D8295E049165104F1F4E091BE08F091BF08838124
:20330000882391F0A981BA81BFABAEABEB81FC81FDABECABCD01BF01AE014F5F5F4F9E01F9
:203320002D5F3F4F0E940E6CCE0109960E94696018C2F6E04F16510409F013C29091C0085D
:20334000992321F080911C08882391F56B817C814D815E8189819A819E01215F3F4F0E9430
:203360008E696F85788980E00E94025C69897A8981E00E94025C6B897C8982E00E94025C50
:2033800080912009882351F08091350B8178813829F48CAD9DAD0E94AF5C05C06D897E89F5
:2033A00083E00E94025C8EAD9FAD0E94CF5C65C020911C0930911D09913049F56091970AE3
:2033C0007091980A4091800A5091810AC9019E01215F3F4F0E948E696F85788980E00E947C
:2033E000025C69897A8981E00E94025C6B897C8982E00E94025C80912009882329F08091AF
:20340000350B81788138F1F06D897E8924C080E0B9010E94025C6091970A7091980A81E048
:203420000E94025C6091800A7091810A82E00E94025C80912009882351F08091350B8178B3
:20344000813829F48CAD9DAD0E94AF5C07C06091C5087091C60883E00E94025C8EAD9FAD28
:203460000E94CF5C8091850A9091860A0E94ED5D80911C08815080931C082AA5222309F4F4
:20348000F6C08091EE07882351F48091C008882309F4EDC080912009882309F0E8C00E942A
:2034A000D25A48A159A1452B09F4DEC08091C008882309F0D9C080917D0980FD08C08091EF
:2034C000F00980FD04C08091630A80FF2AC082E060E041E00E94EA5822243324281A390A02
:2034E000C10181579E4F8F519340D8F481E08093DD0280917D0980FF04C010927F091092CD
:203500007E098091F00980FF04C01092F2091092F1098091630A80FF04C01092650A10922A
:20352000640A8090DD02992498C00E94416F8FE097E20197F1F700C0000082E060E041E0DC
:203540000E94EA58CC24DD24C81AD90A80912009882339F42D96AFAC2D972E96BFAC2E97E9
:2035600006C086E060E040E00E94EA585C01AFE0B0E0EA0EFB1E015F1F4FC701B801A60158
:203580000E940816C5010E94CF5CB3E0003C1B0761F6EE24FF240E94416FEFE0F7E2319799
:2035A000F1F700C000002FE030E0E20EF31E0F501040C701B801A6010E9408160115110580
:2035C00051F7F0ECEF2EF3E0FF2E0E94416F8FE097E20197F1F700C00000A1EFBFEFEA0EFA
:2035E000FB1E0F501040C701B801A6010E940816BCEF00341B0749F7EE24FF240E94416F53
:20360000EFE0F7E23197F1F700C0000021EF3FEFE20EF31E015F1F4FC701B801A6010E94BB
:20362000081630E4E3163CEFF30641F7882089F0992079F410E00E94416F8FE79AE1A6E003
:2036400081509040A040E1F700C000001F5F1A3091F7939492E0991639F0E0E4EE2EECEFD5
:20366000FE2E00E010E061CF0E94D85A1AA68091EE07882309F475C022968EAD9FAD2297AF
:203680000E949707182F2A96AFAD2A97A81769F022968EAD9FAD22970E9497072A968FAF78
:2036A0002A9729961FAE29975CC02996BFAD2997B93128F4BF5F2996BFAF299752C08091C2
:2036C0007F0A2A96EFAD2A97E81709F44AC08E2F0E940E158091DD02823028F0F2E0F093AD
:2036E000DD026624772428A139A1232B31F42C964EAD5FAD2C97452B51F18091680C282F96
:2037000030E080FF24C08091210981FF20C0113059F0113018F01230B9F40EC03695279584
:20372000522F51705FA310C03695279536952795822F81708FA308C053E0369527955A9522
:20374000E1F7922F91709FA3AFA1AA2349F48091840A823021F41FA2B1E0BEA301C01FA298
:203760001DA2E7E04E16510409F04AC0FEA1FF2311F01092840A8091840A823061F0809162
:20378000EE07882341F08091DD02833021F08FEF9FEF0E9421702FA1222321F48091840A9C
:2037A000823069F53DA1332319F031503DA327C04091690C4DA38091210983FF0CC08091A4
:2037C000680C90E044E0969587954A95E1F781700E941F030BC08091680C90E034E096952F
:2037E00087953A95E1F781700E9492078091DD02833021F08EEE9EEE0E9421701FA21EA26A
:2038000027965FAD2797852F90E08F7090700997029760F08BE04816510441F09EE0491649
:20382000510421F0AFE04A165104F9F48091840A8230D9F48091690CBDA1B817B1F480916A
:20384000210983FF10C08091680C90E024E0969587952A95E1F781700E94A7050E945205DD
:203860000E94150302C00E9452054114510469F48091840090918500ECA5FDA58E1B9F0B0B
:203880009093C4088093C30832C0F2E04F16510469F480918400909185002CA53DA5821BF5
:2038A000930B9093960A8093950A21C035E04316510469F480918400909185004CA55DA5C6
:2038C000841B950B9093830A8093820A10C056E04516510461F48091840090918500ACA5C3
:2038E000BDA58A1B9B0B90931F0980931E092796BFAD2797BD3069F41AE002C00E94AC3328
:2039000011501F3F09F463C10E941E6D90FFF6CF5EC12796EFAD2797EE3009F058C1E0916F
:20392000B708F091B808EE5BFE4F808191818101081B190B9091DD02992309F4A3C0913038
:2039400071F4FCEF003E1F070CF09AC00894611C711C25E66216710408F494C08EC0E091B0
:20396000BE08F091BF08E55AFF4F808180FF8AC0923008F487C0943020F0943009F082C00A
:203980004BC0923031F4053611053CF46114710461F14EEF0137140744F12696AEADBFAD30
:2039A0002697AB2B11F52496EEADFFAD2497EF2BE1F42AAD3BAD232BC1F40894611C711C5B
:2039C000923009F05FC03DE2631631E0730608F459C043E04093DD028AEF9AEF0E942170CC
:2039E0006624772451E05CA34DC08CEF013E180724F494E09093DD0203C0A2E0A093DD02A7
:203A00008091840A823019F48EEE9EEE02C08FEF9FEF0E94217034C0BCEF013E1B076CF5DE
:203A200026968EAD9FAD26978C599F4F893C910520F524968EAD9FAD24978C599F4F893CAF
:203A40009105D8F48AAD9BAD8C599F4F893C9105A0F40894611C711CECA1EE2399F0FDE217
:203A60006F16F1E07F0670F080917F0A0E94111422E02093DD021CA205C032E03093DD02DF
:203A800066247724E091BE08F091BF08EC59FF4F808180FF9CC0015E1C4F0CF096C026963B
:203AA0008EAD9FAD26978C599F4F893C910508F08CC024968EAD9FAD24978C599F4F893CBC
:203AC000910508F082C08AAD9BAD8C599F4F893C910508F07AC08AA19BA101969BA38AA3CE
:203AE0008159914008F473C00E94416FE090BE08F090BF08E5E6F0E0EE0EFF1ED7018D9074
:203B00009D907D0180917F0AC82EDD24E3E7F0E0CE9E8001CF9E100DDE9E100D1124C801C1
:203B200087599F4F0E94B3755C01C80185599F4F0E94B375D7012D913C91E9E9FFEFEE0E12
:203B4000FF1E2817390721F410E08A149B0409F011E023E730E0C29EC001C39E900DD29EF4
:203B6000900D112483599F4F0E94B37549E650E0E40EF51ED7012D913C91E7E9FFEFEE0E5E
:203B8000FF1E2817390709F011E023E730E0C29EC001C39E900DD29E900D112481599F4F5C
:203BA0000E94B3754BE650E0E40EF51ED7012D913C912817390709F011E00E94416F112383
:203BC00021F080917F0A0E9411141BA21AA22796BFAD2797BF5F2796BFAF2797B03119F41E
:203BE00027961FAE27971092990AA4C90F931F93CF93DF93FC01E801009789F10115110580
:203C000071F12083223089F0233028F4222351F0213021F507C0243061F0243030F0253043
:203C2000E9F412C0418382E00DC05183428383E009C0872F9927AA27BB2781836283538335
:203C4000448385E088830BC0872F9927AA27BB278183628353834483288301C01882DF913D
:203C6000CF911F910F9108950F931F9390E0FC013697E63CF10540F4E85CFF4FEE0FFF1F70
:203C80000590F491E02D099480E041C290E0011511052105310509F091E0862F692F0E94AC
:203CA000916B35C2862F602F0E94EB6B30C2862F642F402F0E943A592AC2862F642F402F54
:203CC0000E944E5624C2862F602F0E9429571FC2862F602F0E9458571AC2862F602F0E941A
:203CE000875715C2862F602F0E94764810C2862F602F0E945E480BC2862F602F0E944648CC
:203D000006C2862F602F0E942E4801C2862F602F0E941648FCC1862F602F0E94FE47F7C1D8
:203D2000862F602F0E94E647F2C1862F602F0E94CE47EDC1862F642F402F0E94C43AE7C115
:203D4000862F602F0E949E47E2C1862F602F0E94B647DDC1862F602F0E948647D8C1862F73
:203D6000602F0E942447D3C1862F602F0E946E47CEC1862F602F0E945647C9C1862F602F98
:203D80000E943E47C4C1862F602F0E940C47BFC1862F602F0E94F446BAC1862F602F0E943D
:203DA000DC46B5C1862F602F0E94C446B0C1862F602F0E94AC46ABC1862F602F0E94944606
:203DC000A6C1862F602F0E947C46A1C1862F602F0E9464469CC1862F642F402F0E94723C7E
:203DE00096C1862F602F0E944C4691C1862F602F0E941C468CC1862F602F0E94344687C165
:203E0000862F602F0E94DB3C82C1862F602F0E9404467DC1862F602F0E94EC4578C1862FEF
:203E2000602F0E94D44573C1862F602F0E94BC456EC1862F602F0E94A44569C1862F602FB1
:203E40000E943F4464C1862F602F0E9427445FC1862F602F0E940F445AC1862F602F0E946D
:203E6000F74355C1862F602F0E94DF4350C1862F602F0E94C7434BC1862F602F0E94AD4307
:203E800046C1862F602F0E94934341C1862F602F0E9479433CC1862F602F0E945F4337C13E
:203EA000862F602F0E94474332C1862F602F0E942F432DC1862F602F0E94174328C1862F7B
:203EC000602F0E94FD4223C1862F602F0E94E3421EC1862F602F0E94C94219C1862F602F95
:203EE0000E94034014C1862FB8010E9433400FC1862FB8010E9467400AC1862FB8010E9423
:203F0000AA4005C1862FB8010E94ED4000C1862F602F0E943041FBC0862FB8010E94604130
:203F2000F6C0862FB8010E94A141F1C0862FB8010E94E241ECC0862FB8010E942342E7C02D
:203F400090E0011511052105310509F091E0862F692F0E94A43FDBC0862F642F402F0E9439
:203F6000B05FD5C0862F642F402F0E941160CFC0802F0E94B86ACBC0842F602F0E94D06A28
:203F8000C6C0842F602F0E94F36AC1C0842F602F0E94166BBCC0802F0E94546BB8C0802FC1
:203FA0000E94796BB4C0802F0E94016CB0C0802F0E947158ACC0802F0E948A58A8C0C801EF
:203FC0000E94A358A4C0C8010E94C258A0C0C8010E946F5B9CC0802F0E945F5898C060E0CA
:203FE000011511052105310509F061E0842F0E942F5B8DC0842F602F0E94905B88C0842F09
:20400000602F0E94B15B83C0842FB8010E94D25B7EC080E0011511052105310509F081E065
:204020000E94714574C080E0011511052105310509F081E00E945D456AC0802F0E94DB5FB9
:2040400066C0C8010E94385D62C080E0011511052105310509F081E00E941B5D58C0802FF5
:204060000E94655D54C0802F0E947D5D50C0C8010E94955D4CC0C8010E94BA5D48C0802FEB
:204080000E94D95D44C080E0011511052105310509F081E00E9449453AC0802F0E9437450B
:2040A00036C0C8010E94944532C0802F0E9485452EC0C8010E9427452AC080E0011511057E
:2040C0002105310509F081E00E94715E20C0842FB8010E948E5E1BC0802F0E94540217C086
:2040E000802F0E94710213C0C901B8010E94E63F0EC0802F0E940D1081E009C0C8010E940E
:204100006B1081E004C0802F0E94071081E01F910F9108951F93182F8A57823030F48BE727
:204120000E943B6D812F805801C0812F0E943B6D1F910895FF920F931F93CF93DF93EC01FF
:20414000162FF42EFC01962F00E00BC08191082728E08CE800FB06950EF408272A95D1F780
:204160009150992399F704C089910E948A2011501123D1F7FF2019F0802F0E948A208AE7F7
:204180000E943B6DDF91CF911F910F91FF900895DF93CF930F92CDB7DEB78AEA8983CE01AC
:2041A000019661E040E00E949A200F90CF91DF9108959F92AF92BF92CF92DF92EF92FF92F8
:2041C0000F931F93DF93CF9300D000D000D0CDB7DEB70E942C6F8091EE07882319F480E0D3
:2041E00090E005C080E061E041E00E94EA580E94EE56192F89839A83892F0E948A209924CC
:20420000912688E09CE890FA96940EF499268A95D1F71981812F0E948A20912688E09CE866
:2042200090FA96940EF499268A95D1F78091EE07882319F480E090E005C081E061E041E00C
:204240000E94EA580E94EE56192F89839A83892F0E948A20912688E09CE890FA96940EF4C6
:2042600099268A95D1F71981812F0E948A20912688E09CE890FA96940EF499268A95D1F703
:204280008091EE07882319F420E030E009C082E061E041E00E94EA5822273327281B390BB5
:2042A000C9010E94EE56192F89839A83892F0E948A20912688E09CE890FA96940EF49926C1
:2042C0008A95D1F71981812F0E948A20912688E09CE890FA96940EF499268A95D1F7809151
:2042E000EE07882319F480E090E005C083E061E041E00E94EA580E94EE56192F89839A837C
:20430000892F0E948A20912688E09CE890FA96940EF499268A95D1F71981812F0E948A2004
:20432000912688E09CE890FA96940EF499268A95D1F78091EE07882319F480E090E005C02B
:2043400084E061E041E00E94EA580E94EE56192F89839A83892F0E948A20912688E09CE8B5
:2043600090FA96940EF499268A95D1F71981812F0E948A20912688E09CE890FA96940EF4F2
:2043800099268A95D1F78091EE07882319F480E090E005C085E061E041E00E94EA580E94D7
:2043A000EE56192F89839A83892F0E948A20912688E09CE890FA96940EF499268A95D1F745
:2043C0001981812F0E948A20912688E09CE890FA96940EF499268A95D1F710917F0A812F6E
:2043E0000E948A20912688E09CE890FA96940EF499268A95D1F763E0C62ED12CCC0EDD1E69
:2044000055E0A52EB12CAC0EBD1E7E010894E11CF11CC701B601A5010E94FA5E1A81812F93
:204420000E948A20912688E09CE890FA96940EF499268A95D1F71981812F0E948A209126E4
:2044400088E09CE890FA96940EF499268A95D1F71C81812F0E948A20912688E09CE890FA4E
:2044600096940EF499268A95D1F71B81812F0E948A20912688E09CE890FA96940EF49926BA
:204480008A95D1F71E81812F0E948A20912688E09CE890FA96940EF499268A95D1F71D81FD
:2044A000812F0E948A20912688E09CE890FA96940EF499268A95D1F7C701B601A5010E943A
:2044C000105F1A81812F0E948A20912688E09CE890FA96940EF499268A95D1F71981812F8D
:2044E0000E948A20912688E09CE890FA96940EF499268A95D1F71C81812F0E948A20912621
:2045000088E09CE890FA96940EF499268A95D1F71B81812F0E948A20912688E09CE890FA8E
:2045200096940EF499268A95D1F71E81812F0E948A20912688E09CE890FA96940EF49926F6
:204540008A95D1F71D81812F0E948A20912688E09CE890FA96940EF499268A95D1F710913A
:20456000C208812F0E948A20912688E09CE890FA96940EF499268A95D1F71091C108812F5C
:204580000E948A20912688E09CE890FA96940EF499268A95D1F70E94D85E182F0E948A2065
:2045A000912688E09CE890FA96940EF499268A95D1F78091C90A9091CA0A0E94EE56192FF5
:2045C00089839A83892F0E948A20912688E09CE890FA96940EF499268A95D1F71981812F65
:2045E0000E948A20912688E09CE890FA96940EF499268A95D1F78091CB0A9091CC0A0E94F1
:20460000EE56192F89839A83892F0E948A20912688E09CE890FA96940EF499268A95D1F7E2
:204620001981812F0E948A20912688E09CE890FA96940EF499268A95D1F7E090A20AF09049
:20464000A30A0091A40A1091A50A812F9927AA27BB27D82E0E948A209D2488E09CE890FA72
:2046600096940EF499268A95D1F7802F0E948A20902688E09CE890FA96940EF499268A9537
:20468000D1F78F2D0E948A209F2488E09CE890FA96940EF499268A95D1F78E2D0E948A2038
:2046A0009E2488E09CE890FA96940EF499268A95D1F78091CD0A9091CE0A0E94EE56192FE1
:2046C00089839A83892F0E948A20912688E09CE890FA96940EF499268A95D1F71981812F64
:2046E0000E948A20912688E09CE890FA96940EF499268A95D1F78091D10A9091D20A0E94E4
:20470000EE56192F89839A83892F0E948A20912688E09CE890FA96940EF499268A95D1F7E1
:204720001981812F0E948A20912688E09CE890FA96940EF499268A95D1F78091D30A9091D5
:20474000D40A0E94EE56192F89839A83892F0E948A20912688E09CE890FA96940EF4992608
:204760008A95D1F71981812F0E948A20912688E09CE890FA96940EF499268A95D1F78091AC
:20478000D70A9091D80A0E94EE56192F89839A83892F0E948A20912688E09CE890FA969483
:2047A0000EF499268A95D1F71981812F0E948A20912688E09CE890FA96940EF499268A9584
:2047C000D1F71091CF0A812F0E948A20912688E09CE890FA96940EF499268A95D1F780918B
:2047E000D90A9091DA0A0E94EE56192F89839A83892F0E948A20912688E09CE890FA96941F
:204800000EF499268A95D1F71981812F0E948A20912688E09CE890FA96940EF499268A9523
:20482000D1F7E091B708F091B808EA5BFE4F80818570853019F41091A70A02C01091A60A90
:20484000812F0E948A20912688E09CE890FA96940EF499268A95D1F70E94416F80910E0BE1
:2048600090910F0B0E94EE56192F89839A83892F0E948A20912688E09CE890FA96940EF449
:2048800099268A95D1F71981812F0E948A20912688E09CE890FA96940EF499268A95D1F7DD
:2048A0008091100B9091110B0E94EE56192F89839A83892F0E948A20912688E09CE890FA07
:2048C00096940EF499268A95D1F71981812F0E948A20912688E09CE890FA96940EF4992658
:2048E0008A95D1F7E090E70AF090E80A0091E90A1091EA0A812F9927AA27BB27D82E0E941A
:204900008A209D2488E09CE890FA96940EF499268A95D1F7802F0E948A20902688E09CE847
:2049200090FA96940EF499268A95D1F78F2D0E948A209F2488E09CE890FA96940EF49926EF
:204940008A95D1F78E2D0E948A209E2488E09CE890FA96940EF499268A95D1F78091120B31
:204960009091130B0E94EE56192F89839A83892F0E948A20912688E09CE890FA96940EF444
:2049800099268A95D1F71981812F0E948A20912688E09CE890FA96940EF499268A95D1F7DC
:2049A0008091160B9091170B0E94EE56192F89839A83892F0E948A20912688E09CE890FAFA
:2049C00096940EF499268A95D1F71981812F0E948A20912688E09CE890FA96940EF4992657
:2049E0008A95D1F78091180B9091190B0E94EE56192F89839A83892F0E948A20912688E0DD
:204A00009CE890FA96940EF499268A95D1F71981812F0E948A20912688E09CE890FA9694C9
:204A20000EF499268A95D1F71091140B812F0E948A20912688E09CE890FA96940EF49926FA
:204A40008A95D1F780911E0B90911F0B0E94EE56192F89839A83892F0E948A20912688E070
:204A60009CE890FA96940EF499268A95D1F71981812F0E948A20912688E09CE890FA969469
:204A80000EF499268A95D1F7E091B708F091B808EA5BFE4F80818970893019F41091EC0A14
:204AA00002C01091EB0A812F0E948A20912688E09CE890FA96940EF499268A95D1F70E9401
:204AC000416F8091A3089091A4080E94EE56192F89839A83892F0E948A20912688E09CE89F
:204AE00090FA96940EF499268A95D1F71981812F0E948A20912688E09CE890FA96940EF46B
:204B000099268A95D1F78091A5089091A6080E94EE56192F89839A83892F0E948A20912650
:204B200088E09CE890FA96940EF499268A95D1F71981812F0E948A20912688E09CE890FA6A
:204B400096940EF499268A95D1F7E0907E08F0907F080091800810918108812F9927AA2702
:204B6000BB27D82E0E948A209D2488E09CE890FA96940EF499268A95D1F7802F0E948A20FD
:204B8000902688E09CE890FA96940EF499268A95D1F78F2D0E948A209F2488E09CE890FAD6
:204BA00096940EF499268A95D1F78E2D0E948A209E2488E09CE890FA96940EF499268A95DA
:204BC000D1F78091A7089091A8080E94EE56192F89839A83892F0E948A20912688E09CE87E
:204BE00090FA96940EF499268A95D1F71981812F0E948A20912688E09CE890FA96940EF46A
:204C000099268A95D1F78091A9089091AA080E94EE56192F89839A83892F0E948A20912647
:204C200088E09CE890FA96940EF499268A95D1F71981812F0E948A20912688E09CE890FA69
:204C400096940EF499268A95D1F78091AB089091AC080E94EE56192F89839A83892F0E9438
:204C60008A20912688E09CE890FA96940EF499268A95D1F71981812F0E948A20912688E0D6
:204C80009CE890FA96940EF499268A95D1F78091B1089091B2080E94EE56192F89839A8338
:204CA000892F0E948A20912688E09CE890FA96940EF499268A95D1F71981812F0E948A205B
:204CC000912688E09CE890FA96940EF499268A95D1F78091AD089091AE080E94EE56192F0A
:204CE00089839A83892F0E948A20912688E09CE890FA96940EF499268A95D1F71981812F3E
:204D00000E948A20912688E09CE890FA96940EF499268A95D1F78091AF089091B0080E9405
:204D2000EE56192F89839A83892F0E948A20912688E09CE890FA96940EF499268A95D1F7BB
:204D40001981812F0E948A20912688E09CE890FA96940EF499268A95D1F78091B3089091D1
:204D6000B4080E94EE56192F89839A83892F0E948A20912688E09CE890FA96940EF4992604
:204D80008A95D1F71981812F0E948A20912688E09CE890FA96940EF499268A95D1F7E09126
:204DA000B708F091B808EA5BFE4F80818370833019F41091830802C010918208812F0E9442
:204DC0008A20912688E09CE890FA96940EF499268A95D1F70E94416F80E00E94C65C0E9412
:204DE000EE56192F89839A83892F0E948A20912688E09CE890FA96940EF499268A95D1F7FB
:204E00001981812F0E948A20912688E09CE890FA96940EF499268A95D1F781E00E94C65CD8
:204E20000E94EE56192F89839A83892F0E948A20912688E09CE890FA96940EF499268A95E0
:204E4000D1F71981812F0E948A20912688E09CE890FA96940EF499268A95D1F782E00E94F1
:204E6000C65C0E94EE56192F89839A83892F0E948A20912688E09CE890FA96940EF499269D
:204E80008A95D1F71981812F0E948A20912688E09CE890FA96940EF499268A95D1F783E033
:204EA0000E94C65C0E94EE56192F89839A83892F0E948A20912688E09CE890FA96940EF47A
:204EC00099268A95D1F71981812F0E948A20912688E09CE890FA96940EF499268A95D1F797
:204EE0000E946C5E0E94EE56192F89839A83892F0E948A20912688E09CE890FA96940EF492
:204F000099268A95D1F71981812F0E948A20892D812798E02CE880FB86950EF482279A95FB
:204F2000D1F70E948A208AE70E943B6D0E94356F26960FB6F894DEBF0FBECDBFCF91DF9189
:204F40001F910F91FF90EF90DF90CF90BF90AF909F9008951F93DF93CF930F92CDB7DEB78B
:204F600085E589831AE011501F3F21F00E941E6D90FFF9CF81E080930001CE01019660E052
:204F800040E00E949A200F90CF91DF911F910895CF92DF92EF92FF920F931F93DF93CF93CD
:204FA000CDB7DEB762970FB6F894DEBF0FBECDBF6C01DC018C9190E0FC01B097E231F10574
:204FC00010F00C948833E250FF4FEE0FFF1F0590F491E02D0994F601218180E093E28927F9
:204FE00038E09CE880FB86950EF489273A95D1F7822738E09CE880FB86950EF489273A95DA
:20500000D1F7D60112969C91981711F00C9488331C821B821E821D82E22FF0E0E532F105A9
:2050200010F00C948833E05FFE4FEE0FFF1F0590F491E02D099480E029C080E061E041E09F
:205040000E94EA580E94EE569C838B83A1C081E01DC081E0F3CF82E061E041E00E94EA58EF
:20506000909581959F4FF0CF82E061E041E00E94EA58909581959F4FE5CF83E007C083E036
:20508000DDCF84E003C084E0D9CF85E061E041E00E94EA58D9CF85E0D1CF80E00BC080E04E
:2050A0000DC081E007C081E009C082E003C082E005C083E00E94C65CC7CF83E00E94C65CA1
:2050C000C1CF0E946C5EC0CF0E946C5EBBCF80E001C081E00E94265F9C838B83AC0166273F
:2050E00057FD6095762F59C082E0F4CF8091C3089091C40804C08091950A9091960A9E8365
:205100008D8336C08091820A9091830AF8CF80911E0990911F09F3CF40917B0A50917C0A77
:2051200060917D0A70917E0A1AC04091870A5091880A6091890A70918A0A11C040918B0A6F
:2051400050918C0A60918D0A70918E0A08C04091C7085091C8086091C9087091CA0824E005
:205160000C948B33CE0105960E947E028D819E81AC0160E070E023E00C948B3380E001C059
:2051800081E0BE016D5F7F4F0E94555F8B819C81AC01662757FD6095762F22E00C948B334E
:2051A00082E0EFCFF601348520E09CE00AC08191282748E08CE820FB26950EF428274A95D6
:2051C000D1F79150A0F7321711F00C948833D60111969C9111979093C00812968C9112973E
:2051E00080931D0913968C91139780931C0914968C9114978093980A15968C911597809320
:20520000970A16968C9116978093810A17968C9117978093800A18968C9118978093C60869
:2052200019968C9119978093C5081A968C911A978093860A1B968C918093850A992321F4B0
:2052400010921C080C94853382E380931C080C948533F601338120E093E00AC081912827F3
:2052600048E08CE820FB26950EF428274A95D1F79150A0F7321711F00C948833D601119629
:205280008C91119712964C9187FD08C0242F2295269526952370642F6F7302C0642F20E09B
:2052A0001D821B821A86198618861F821B861C861D861E8690E0FC013697E63CF10510F058
:2052C0000C948833EB5CFE4FEE0FFF1F0590F491E02D0994822FBE016E5F7F4F0E94B56B33
:2052E000382F8A81482F50E060E070E021E0D0C5822FBE016B5F7F4F0E94D26B382F8D8113
:20530000482F50E060E070E021E0C2C5822FAE014B5F5F4F0E943156382F8D81482F50E0D1
:2053200060E070E021E0B4C5822FAE014B5F5F4F0E946856382F8D81482F50E060E070E09F
:2053400021E0A6C5822FBE016B5F7F4F0E943F57382F8D81482F50E060E070E021E098C597
:20536000822FBE016B5F7F4F0E946E57382F8D81482F50E060E070E021E08AC5822FBE0152
:205380006B5F7F4F0E949D57382F8D81482F50E060E070E021E07CC5822FBE016B5F7F4FE9
:2053A0000E94FC39382F8D81482F50E060E070E021E06EC5822FBE016B5F7F4F0E94153A3D
:2053C000382F8D81482F50E060E070E021E060C5822FBE016B5F7F4F0E942E3A382F8D8174
:2053E000482F50E060E070E021E052C5822FBE016B5F7F4F0E94473A382F8D81482F50E017
:2054000060E070E021E044C5822FBE016B5F7F4F0E94603A382F8D81482F50E060E070E002
:2054200021E036C5822FBE016B5F7F4F0E94793A382F8D81482F50E060E070E021E028C579
:20544000822FBE016B5F7F4F0E94923A382F8D81482F50E060E070E021E01AC5822FBE01DA
:205460006B5F7F4F0E94AB3A382F8D81482F50E060E070E021E00CC5822FAE014B5F5F4FD7
:205480000E94DE3A382F8D81482F50E060E070E021E0FEC4822FBE016B5F7F4F0E94FB3A04
:2054A000382F8D81482F50E060E070E021E0F0C4822FBE016B5F7F4F0E942D3B382F8D8104
:2054C000482F50E060E070E021E0E2C4822FBE016B5F7F4F0E94143B382F8D81482F50E0D9
:2054E00060E070E021E0D4C4822FBE016D5F7F4F0E94913B382F8B81482F552747FD50957C
:20550000652F752F20E0C4C4822FBE016B5F7F4F0E94463B382F8D81482F50E060E070E0F4
:2055200021E0B6C4822FBE016B5F7F4F0E945F3B382F8D81482F50E060E070E021E0A8C493
:20554000822FBE016B5F7F4F0E94783B382F8D81482F50E060E070E021E09AC4822FBE0173
:205560006B5F7F4F0E94AA3B382F8D81482F50E060E070E021E08CC4822FBE016B5F7F4F07
:205580000E94C33B382F8D81482F50E060E070E021E07EC4822FBE016B5F7F4F0E94DC3BBB
:2055A000382F8D81482F50E060E070E021E070C4822FBE016B5F7F4F0E94F53B382F8D81BB
:2055C000482F50E060E070E021E062C4822FBE016B5F7F4F0E940E3C382F8D81482F50E05D
:2055E00060E070E021E054C4822FBE016B5F7F4F0E94273C382F8D81482F50E060E070E049
:2056000021E046C4822FBE016B5F7F4F0E94403C382F8D81482F50E060E070E021E038C4B0
:20562000822FBE016B5F7F4F0E94593C382F8D81482F50E060E070E021E02AC4822FAE0130
:205640004B5F5F4F0E948C3C382F8D81482F50E060E070E021E01CC4822FBE016B5F7F4FF3
:205660000E94A93C382F8D81482F50E060E070E021E00EC4822FBE016B5F7F4F0E940A3D33
:20568000382F8D81482F50E060E070E021E000C4822FBE016B5F7F4F0E94C23C382F8D817C
:2056A000482F50E060E070E021E0F2C3822FBE016B5F7F4F0E94F13C382F8D81482F50E00A
:2056C00060E070E021E0E4C3822FBE016B5F7F4F0E94233D382F8D81482F50E060E070E0DC
:2056E00021E0D6C3822FBE016B5F7F4F0E943C3D382F8D81482F50E060E070E021E0C8C3B5
:20570000822FBE016B5F7F4F0E94553D382F8D81482F50E060E070E021E0BAC3822FBE01B3
:205720006B5F7F4F0E946E3D382F8D81482F50E060E070E021E0ACC3822FBE016B5F7F4F60
:205740000E94873D382F8D81482F50E060E070E021E09EC3822FBE016B5F7F4F0E94A03D4E
:20576000382F8D81482F50E060E070E021E090C3822FBE016B5F7F4F0E94B93D382F8D8114
:20578000482F50E060E070E021E082C3822FBE016B5F7F4F0E94D23D382F8D81482F50E0B7
:2057A00060E070E021E074C3822FBE016B5F7F4F0E94EB3D382F8D81482F50E060E070E0A3
:2057C00021E066C3822FBE016B5F7F4F0E94043E382F8D81482F50E060E070E021E058C3EB
:2057E000822FBE016B5F7F4F0E941D3E382F8D81482F50E060E070E021E04AC3822FBE017A
:205800006D5F7F4F0E94363E382F8B81482F552747FD5095652F752F20E03AC3822FBE01A4
:205820006D5F7F4F0E944F3E382F8B81482F552747FD5095652F752F20E02AC3822FBE017B
:205840006D5F7F4F0E94683E382F8B81482F552747FD5095652F752F20E01AC3822FBE0152
:205860006D5F7F4F0E94813E382F8B81482F552747FD5095652F752F20E00AC3822FBE0129
:205880006B5F7F4F0E949A3E382F8D81482F50E060E070E021E0FCC2822FBE016B5F7F4F83
:2058A0000E94B33E382F8D81482F50E060E070E021E0EEC2822FBE016B5F7F4F0E94CC3E44
:2058C000382F8D81482F50E060E070E021E0E0C2822FBE016D5F7F4F0E94E53E382F8B8137
:2058E000482F552747FD5095652F752F20E0D0C2822FBE016D5F7F4F0E94FE3E382F8B8167
:20590000482F552747FD5095652F752F20E0C0C2822FBE016D5F7F4F0E94173F382F8B813C
:20592000482F552747FD5095652F752F20E0B0C2822FBE016B5F7F4F0E941A40382F8D8128
:20594000482F50E060E070E021E0A2C2822FBE01675F7F4F0E944C40382F89859A85AC0138
:2059600060E070E023E094C2822FBE01695F7F4F0E948740382F8F819885AC01662757FDAD
:205980006095762F22E084C2822FBE01695F7F4F0E94CA40382F8F819885AC01662757FD51
:2059A0006095762F22E074C2822FBE01695F7F4F0E940D41382F8F819885AC01662757FDFD
:2059C0006095762F22E064C2822FBE016B5F7F4F0E944741382F8D81482F50E060E070E027
:2059E00021E056C2822FBE01695F7F4F0E947E41382F8F819885AC01662757FD6095762F6B
:205A000022E046C2822FBE01695F7F4F0E94BF41382F8F819885AC01662757FD6095762F18
:205A200022E036C2822FBE01695F7F4F0E940042382F8F819885AC01662757FD6095762FC6
:205A400022E026C2822FBE01695F7F4F0E944142382F8F819885AC01662757FD6095762F75
:205A600022E016C2822FBE016E5F7F4F0E94C83F382F8A81482F50E060E070E021E008C224
:205A8000822FAE014B5F5F4F0E94915F382F8D81482F50E060E070E021E0FAC1822FAE01F4
:205AA0004B5F5F4F0E94E95F382F8D81482F50E060E070E021E0ECC1CE0105960E94C36A11
:205AC000382F8D81482F50E060E070E021E0E0C1862FBE016D5F7F4F0E94E16A382F8B810A
:205AE000482F552747FD5095652F752F20E0D0C1862FBE016D5F7F4F0E94046B382F8B812F
:205B0000482F552747FD5095652F752F20E0C0C1862FBE016D5F7F4F0E94276B382F8B81FB
:205B2000482F552747FD5095652F752F20E0B0C1CE0105960E945F6B382F8D81482F50E0AE
:205B400060E070E021E0A4C1CE0105960E946C6B382F8D81482F50E060E070E021E098C166
:205B6000CE0105960E94846B382F8D81482F50E060E070E021E08CC1CE0105960E947D584F
:205B8000382F8D81482F50E060E070E021E080C1CE0105960E949658382F8D81482F50E001
:205BA00060E070E021E074C1CE0107960E94B358382F8F819885AC01662757FD6095762F4A
:205BC00022E066C1CE0107960E94D258382F8F819885AC01662757FD6095762F22E058C18D
:205BE000CE0109960E94815B382F89859A85AC0160E070E023E04CC1CE0105960E9467580D
:205C0000382F8D81482F50E060E070E021E040C1862FBE016E5F7F4F0E94535B382F8A8105
:205C2000482F50E060E070E021E032C1862FBE016B5F7F4F0E949F5B382F8D81482F50E075
:205C400060E070E021E024C1862FBE016B5F7F4F0E94C05B382F8D81482F50E060E070E059
:205C600021E016C1862FBE01695F7F4F0E94EB5B382F8F819885AC01662757FD6095762F9E
:205C800022E006C1CE0102960E944C3F382F8A81482F50E060E070E021E0FAC0CE010296DC
:205CA0000E94603F382F8A81482F50E060E070E021E0EEC0CE0105960E94CC5F382F8D819F
:205CC000482F50E060E070E021E0E2C0CE0109960E94565D382F89859A85AC0160E070E056
:205CE00023E0D6C0CE0102960E94275D382F8A81482F50E060E070E021E0CAC0CE010596E0
:205D00000E94705D382F8D81482F50E060E070E021E0BEC0CE0105960E94885D382F8D8183
:205D2000482F50E060E070E021E0B2C0CE0109960E94AB5D382F89859A85AC0160E070E0D0
:205D400023E0A6C0CE0107960E94CA5D382F8F819885AC01662757FD6095762F22E098C08F
:205D6000CE0105960E94E05D382F8D81482F50E060E070E021E08CC0CE0102960E94743F25
:205D8000382F8A81482F50E060E070E021E080C0CE0105960E94883F382F8D81482F50E02A
:205DA00060E070E021E074C0CE0107960E94303F382F8F819885AC01662757FD6095762FE5
:205DC00022E066C0CE0105960E943D3F382F8D81482F50E060E070E021E05AC0CE010996DE
:205DE0000E94973F382F89859A85AC0160E070E023E04EC0CE0102960E947D5E382F8A81F3
:205E0000482F50E060E070E021E042C0862FBE01675F7F4F0E94A45E382F89859A85AC015B
:205E200060E070E023E034C0CE0105960E944502382F8D81482F50E060E070E021E028C0F3
:205E4000CE0105960E946202382F8D81482F50E060E070E021E01CC0CE010B960E94F03F08
:205E6000382F4B855C856D857E8524E011C00E942F1007C00E9471109A87898779C90E9460
:205E80002A108D83482F50E060E070E021E043C4332309F43DC43FC418861F821A861986A4
:205EA0001B861C861D861E861F86188A198A1A8AC114D10409F42CC4F601F1804281F7FC15
:205EC00007C0642F62956695669563704F7301C060E0D60113968C91823009F44BC08330DB
:205EE00030F4882371F0813009F012C427C0843009F48CC0843008F464C0853009F008C4C0
:205F0000B3C0F6010481B58175E050E00CC0F60181916F01582788E09CE850FB56950EF4EF
:205F200059278A95D1F7715090F7B51709F0F0C3112707FD1095212F312FF9C3D60114966C
:205F40000C9114971596BC9175E050E00CC0F60181916F01582788E09CE850FB56950EF494
:205F600059278A95D1F7715090F7B51709F0D0C310E049C0D60114968C9114978A8715961C
:205F80008C911597898716963C9126E090E00CC0F60181916F01982788E05CE890FB9695D3
:205FA0000EF495278A95D1F7215090F7391709F0AFC389859A858C01222717FD2095322F5C
:205FC000B6C3D60114968C911497888715968C9115978F8316963C9126E090E00CC0F601B8
:205FE00081916F01982788E05CE890FB96950EF495278A95D1F7215090F7391709F088C3CD
:206000008F8198858C0120E030E091C3FE013F96D60114968C911497838315968C911597CB
:20602000828316968C911697818317968C9117978F8718963C9128E090E00CC0F60181918B
:206040006F01982788E05CE890FB96950EF495278A95D1F7215090F7391709F059C30F8519
:20606000188929893A8963C3FE013B96D60114968C911497838315968C91159782831696A0
:206080008C911697818317968C9117978B8718963C9128E090E00CC0F60181916F019827B1
:2060A00088E05CE890FB96950EF495278A95D1F7215090F7391709F02BC30B851C852D85C7
:2060C0003E8535C30E94CF04882319F00E94C82002C00E94AA278091210983FF2EC381E00E
:2060E0000E94CB022AC38091210983FF0FC00E94A004882309F40CC381E00E9483048823C6
:2061000009F406C380E00E94CB0203C080E00E948304882309F4FCC28FEE97E06DE203C32F
:2061200080E098E2892728E09CE880FB86950EF489272A95D1F7D60111969C91981709F027
:20614000E7C20E9475130E940714DFC280E099E2892728E09CE880FB86950EF489272A95F0
:20616000D1F7F6019181981709F0D2C20E94BC5E0E947610CAC280E09AE2892728E09CE88A
:2061800080FB86950EF489272A95D1F7D60111969C91981709F0BCC20E94D920CEC280E0D4
:2061A0009BE2892728E09CE880FB86950EF489272A95D1F7F6019181981709F0A9C28FECC0
:2061C000D6018C938CE211968C93119780E312968C93129784ED13968C9313978CEF149612
:2061E0008C93149715961C92159784E016968C93169717961C928091C00A9091C10AA091A1
:20620000C20AB091C30AB095A095909581959F4FAF4FBF4F8B2F9927AA27BB27F6018087CA
:206220008091C00A9091C10AA091C20AB091C30AB095A095909581959F4FAF4FBF4FA187B5
:206240008091C00A9091C10AA091C20AB091C30AB095A095909581959F4FAF4FBF4F9287A4
:206260008091C00A819583878091C00A9091C10AA091C20AB091C30A8B2F9927AA27BB2724
:2062800084878091C20A85878091C10A86878091C00A87878091050B9091060BA091070BA2
:2062A000B091080BB095A095909581959F4FAF4FBF4F8B2F9927AA27BB27808B8091050B82
:2062C0009091060BA091070BB091080BB095A095909581959F4FAF4FBF4FA18B8091050BF9
:2062E0009091060BA091070BB091080BB095A095909581959F4FAF4FBF4F928B8091050BE8
:206300008195838B8091050B9091060BA091070BB091080B8B2F9927AA27BB27848B809122
:20632000070B858B8091060B868B8091050B878B80919E0890919F08A091A008B091A10893
:20634000B095A095909581959F4FAF4FBF4F8B2F9927AA27BB27808F80919E0890919F08D3
:20636000A091A008B091A108B095A095909581959F4FAF4FBF4FA18F80919E0890919F08FC
:20638000A091A008B091A108B095A095909581959F4FAF4FBF4F928F80919E088195838F8B
:2063A00080919E0890919F08A091A008B091A1088B2F9927AA27BB27848F8091A008858F8E
:2063C00080919F08D6015E968C935E9780919E085F968C930091080110910901C8010E94AB
:2063E000EE56F60190A3C8010E94EE56D60191968C9300910A0110910B01C8010E94EE566B
:20640000F60192A3C8010E94EE56D60193968C9384E28983C60164E286C180E09CE289272E
:2064200028E09CE880FB86950EF489272A95D1F7F6019181981709F06BC10E943910D60162
:206440008C930E943410F6018183C60162E06BC180E09DE2892728E09CE880FB86950EF454
:2064600089272A95D1F7D60111969C91981709F04FC10E94131049C180E09EE2892728E01B
:206480009CE880FB86950EF489272A95D1F7F6019181981709F03CC10E94191036C180E0D9
:2064A0009FE2892728E09CE880FB86950EF489272A95D1F7D60111969C91981709F028C114
:2064C0000E94C8200E94BC5E0E944D1000E010E00E94416FEFE4F3EC3197F1F700C0000033
:2064E0000F5F1F4F083C110599F70E94356FFFCF80E090E3892728E09CE880FB86950EF41B
:2065000089272A95D1F7D60111969C91981709F0FFC00E942F10F601808381E0818387E08B
:2065200082831382E091B708F091B8088081D60114968C930E947110F60195838683C601AD
:2065400067E0F1C0D60115963C91F60120E095E00AC08191282748E08CE820FB26950EF4E9
:2065600028274A95D1F79150A0F7321709F0D0C0F60111810281F380E4800E942C6F8BE24E
:206580000E943B6D8FEB94EDA1E081509040A040E1F700C000008BE20E943B6D8FEB94ED6A
:2065A000A1E081509040A040E1F700C000008BE20E943B6D8FEF98E0ADE381509040A04083
:2065C000E1F700C0000081E40E943B6D8FEB94EDA1E081509040A040E1F700C0000084E576
:2065E0000E943B6D8FEB94EDA1E081509040A040E1F700C0000080E50E943B6D8FEB94ED12
:20660000A1E081509040A040E1F700C000008DE30E943B6D8FEB94EDA1E081509040A04029
:20662000E1F700C00000812F805D0E943B6D8FEB94EDA1E081509040A040E1F700C0000056
:20664000802F805D0E943B6D8FEB94EDA1E081509040A040E1F700C000008F2D805D0E9494
:206660003B6D8FEB94EDA1E081509040A040E1F700C000008E2D805D0E943B6D8FEB94ED00
:20668000A1E081509040A040E1F700C000008DE00E943B6D8FE79FE4A2E181509040A040AC
:2066A000E1F700C0000081E40E943B6D8FEB94EDA1E081509040A040E1F700C0000084E595
:2066C0000E943B6D8FEB94EDA1E081509040A040E1F700C000008FE40E943B6D8FEB94ED23
:2066E000A1E081509040A040E1F700C000008DE00E943B6D8FE79FE4A2E181509040A0404C
:20670000E1F700C000000E94356F0E94C82015C00E94AA2712C0C6018E010F5F1F4F0E9423
:20672000F61DC601698141E00E949A2006C08F2D0E94341E882361F3E8CF62960FB6F894A3
:20674000DEBF0FBECDBFCF91DF911F910F91FF90EF90DF90CF900895682F80910001813050
:2067600021F0823009F043C030C06A3731F06B3711F582E080930001089589EB98E06AE7B0
:206780000E940D6F4091DE024F5F4093DE0289EB98E06BEC78E00E94EF6E882331F08BECEC
:2067A00098E06091DE020E94C82781E0809300011092DE02089589EB98E00E940D6F809150
:2067C000DE028F5F8093DE020895262F20586A5F623068F489EB98E0622F0E940D6F80912B
:2067E000DE028F5F8093DE0281E08093000108951F93CF93DF93EC012889222349F41EA260
:206800001FA218A619A61AA61BA61CA61DA67BC06AA17BA1882777FD8095982F59E0660F25
:20682000771F881F991F5A95D1F730E040E050E00E942775C901DA013E8920E0AC01BD0137
:20684000639FD001439FC001A20BB20B539F900DA11DB21F7303B00D112446E0B595A79526
:20686000979587954A95D1F78EA39FA3A8A7B9A7855D9D4AA040B04044F084ED9DEAA0E0C2
:20688000B0E08EA39FA3A8A7B9A76AA17BA1882777FD8095982F39E0660F771F881F991F9D
:2068A0003A95D1F7288930E040E050E00E942775C901DA013F8920E0AC01BD01639FD00147
:2068C000439FC001A20BB20B539F900DA11DB21F7303B00D112426E0B595A7959795879551
:2068E0002A95D1F78AA79BA7ACA7BDA7855D9D4AA040B04044F084ED9DEAA0E0B0E08AA7E1
:206900009BA7ACA7BDA7EA89E03829F480E090E0A0E0B0E021C06EA17FA1F8A519A5EE237A
:2069200021F4CB01AF2FB12F17C088EE93E08E9F9001442755279E9F300D411D112487E0DF
:2069400056954795379527958A95D1F78F2F912F0E942775C901DA01888F998FAA8FBB8FDE
:20696000DF91CF911F9108952F923F924F925F926F927F928F929F92AF92BF92CF92DF92CE
:20698000EF92FF920F931F93DF93CF9300D000D0CDB7DEB76C017A8369831A01922E38019A
:2069A000FC82EB828091210990E038E0E32EF12CE822F92283FF15C080E029E98601382F1F
:2069C00088279927029FB0011203930B700D811D931F112420E031E040E050E00E94497580
:2069E0006901860102191309AB81BC811E968C911E97882319F01D966C9103C0EB81FC8170
:206A00006485EF28A9F480E0F82FAA27BB27069FC0011603BF0B900DA11DBF1F112425E0E3
:206A2000B595A795979587952A95D1F75C0122C080E044275527069F90011603580B300D8C
:206A4000411D581F11246DE0062F182F409FC001209FB001810B910B309F700D811D911F91
:206A60005003900D112420E031E040E050E00E9449755901AB81BC811F962C911F9780E0E5
:206A8000850166277727029FA0011203780B500D611D781F112497E075956795579547957F
:206AA0009A95D1F790964D905C909197C201AA2797FDA095BA2F84179507A607B7077CF074
:206AC0005094419451085394C201AA2797FDA095BA2F481759076A077B070CF02A019920E5
:206AE000E1F0EB81FC8180859185A285B385181619061A061B0624F41A141B043CF00DC076
:206B00000097A105B10549F0B7FE07C0AB81BC81D1968D909C90D29714C2EB81FC81808983
:206B2000882339F410861186128613868824992408C2EB81FC81E084F18402851385828108
:206B400093818C199D0997FF03C0909581959F4F9093D60A8093D50A2B813C81215C3F4FEB
:206B6000D9012D913C911197DF97BC83AB8380910A0190910B010A97281739071CF01A1482
:206B80001B0464F180910801909109010A968217930714F0B7FC22C0EB81FC8186A5853007
:206BA00021F4C50164E070E005C0181674F4C50162E070E00E941475882777FD8095982F89
:206BC000E60EF71E081F191F09C0C501AA2797FDA095BA2FE80EF91E0A1F1B1FEB81FC81E2
:206BE00086A197A1A0A5B1A58E159F05A007B1072CF480879187A287B3871BC022273327D5
:206C0000A901281B390B4A0B5B0BE216F306040715074CF4AB81BC8118962D933D934D93A9
:206C20005C931B9706C0EB81FC81E086F18602871387AB81BC8112968D919C9113978C1959
:206C40009D0997FF03C0909581959F4F8930910564F09601D7FE04C0222733272C193D090B
:206C6000293C310514F08AE022C0049794F0AB81BC819E968C91853064F4C601D7FE04C0E3
:206C8000882799278C199D098536910514F085E00EC0AB81BC819E968C919E97181624F47D
:206CA00081509E968C9306C0882321F08F5FEB81FC8186A7AB81BC8118962D913D914D91A9
:206CC0005C911B9750966C91509780E0469F8001269F7001080B180B369FF00C011D181FF3
:206CE0005603100D112489E015950795F794E7948A95D1F792968D909C909397C401AA271C
:206D000097FDA095BA2F8E159F05A007B1077CF09094819491089394C401AA2797FDA09557
:206D2000BA2FE816F9060A071B070CF04701EB81FC818389882329F4E08CF18C028D138D21
:206D400083C0C301FEE16F16FBEF7F0614F48EE19BEF04E0833E900714F082EE94E0F2EE54
:206D6000EF2EF4E0FF2EE80EF91EC70169E371E00E941475462F4F5F493048F0AB81BC811B
:206D80005896ED90FD900D911C915B975DC0EB81FC8124893589F901E60FF11D1081C701F7
:206DA00069E371E00E941475240F311DD9012C91211B30E0AC01882799272403830B930B38
:206DC000B0015202930B700D811D931F112429E331E040E050E00E944975E22FE10FAB8114
:206DE000BC81D596EC93D597D6961C92D697E03809F4A7C096966C91969797967C9197973F
:206E00009896FC91989799961C91EE2321F4CB01AF2FB12F17C088EE93E08E9F9001442713
:206E200055279E9F300D411D1124E7E05695479537952795EA95D1F78F2F912F0E942775B0
:206E4000C901DA017C018D01E114F1040105110509F477C0EB81FC81208531854285538565
:206E6000878957FF36C0882319F186E990E0680E791E9DE2691691E07906D0F082A593A508
:206E8000A4A5B5A58E0D9F1DA01FB11FB095A095909581959F4FAF4FBF4F82179307A407DC
:206EA000B50708F44EC02E0D3F1D401F511F2FC088279927DC018E199F09A00BB10B82171C
:206EC0009307A407B50750F12E0D3F1D401F511F30C08823F1F0E6E9F0E06E0E7F1EFDE2F7
:206EE0006F16F1E07F06A8F0EB81FC8182A593A5A4A5B5A58E0D9F1DA01FB11F28173907CF
:206F00004A075B07F0F02E193F09400B510BDF0112C02E153F054007510738F4EB81FC81BB
:206F200010861186128613860CC02E193F09400B510BAB81BC8118962D933D934D935C937B
:206F40001B97EB81FC816189662309F495C08481958109811A81081B190B9801442737FD12
:206F60004095542FDA01C9010396A11DB11D0797A105B10528F420E030E040E050E011C0A8
:206F80002D3F1FEF31071FEF41071FEF51072CF42C5F3F4F4F4F5F4F04C0245030404040D6
:206FA000504080E0469F8001269F7001080B180B369FF00C011D181F5603100D1124AB8112
:206FC000BC81D3964D915C91D4975C962D913C915D9788279927821B930B481759073CF4CB
:206FE000240F351FD4963C932E93D39710C0241735073CF4421B530BEB81FC8154AB43AB9E
:2070000006C0AB81BC81D4961C921E92D397A801970162E055954795379527956A95D1F777
:20702000EB81FC8183A994A9AA2797FDA095BA2F280F391F4A1F5B1F64A175A1CB01AA2751
:2070400097FDA095BA2F82179307A407B50774F0709561957F4FCB01AA2797FDA095BA2F68
:20706000281739074A075B070CF0B901AB81BC819E968C91882311F460E070E0EB81FC8145
:2070800031822082D382C28209811A8115830483B782A682C401840D951D860F971F5C01AD
:2070A000CC24B7FCC094DC2C80910A0190910B019C01442737FD4095542F2A153B054C0524
:2070C0005D0594F080910801909109017C010027F7FC0095102FA6019501AE14BF04C00692
:2070E000D10614F4A8019701AB81BC81D0965C924E929F97D2969C928E92D197D4967C9306
:207100006E93D397D8963C932E93D797C9010F900F900F900F90CF91DF911F910F91FF90A3
:20712000EF90DF90CF90BF90AF909F908F907F906F905F904F903F902F900895AF92BF928D
:20714000CF92DF92EF92FF920F931F93CF93DF935C0169017801E091BE08F091BF08EB5A1F
:20716000FF4F1081E555F040112319F460E070E01CC09B0177FF03C0309521953F4F80E0DB
:20718000682FAA27BB271203A60BB60BC0013102B60B900DA11DB61F112407E0B595A79597
:2071A000979587950A95D1F7BC017093AE086093AD08C091B708D091B808CF5BDE4F0881F1
:2071C000C154D140013019F4709561957F4FEA5AFF4F1081E655F040112319F440E050E063
:2071E0001CC09A0157FF03C0309521953F4F80E0482FAA27BB271203A40BB40BC0013102F5
:20720000B40B900DA11DB41F112417E0B595A795979587951A95D1F7AC015093B0084093F5
:20722000AF08013019F4509541955F4FE95AFF4F1081112319F420E030E022C0CE5BDE4F45
:20724000888199819601281B390B37FF03C0309521953F4F80E0E82FAA27BB271203AE0BF3
:20726000BE0BC0013102BE0B900DA11DBE1F1124E7E0B595A79597958795EA95D1F79C01A2
:20728000013019F4309521953F4F3093B2082093B108CB018A0D9B1D840F951F820F931F19
:2072A000F7019183808320910A0130910B012817390744F0209108013091090182179307CB
:2072C0001CF4F70131832083DF91CF911F910F91FF90EF90DF90CF90BF90AF900895EF92A7
:2072E000FF920F931F93CF93DF93EC012C89222329F418A619A61AA61BA63DC06CA17DA1AB
:20730000882777FD8095982F3AE0660F771F881F991F3A95D1F730E040E050E00E942775B5
:20732000C901DA013F8920E0AC01BD01639FD001439FC001A20BB20B539F900DA11DB21F77
:207340007303B00D112426E0B595A795979587952A95D1F788A799A7AAA7BBA781529B4C8E
:20736000A040B04044F080E29BECA0E0B0E088A799A7AAA7BBA76E89603829F4188E198EF5
:207380001A8E1B8E24C0E8A4F9A40AA51BA5662329F4E88EF98E0A8F1B8F19C080EA9FE078
:2073A000869F900144275527969F300D411D112487E056954795379527958A95D1F7C801C5
:2073C000B7010E942775288F398F4A8F5B8F68A579A58AA59BA52EE330E040E050E00E94C8
:2073E00027752C8F3D8F4E8F5F8FDF91CF911F910F91FF90EF900895DB018330A0F461153B
:20740000710589F0282F30E083E790E0289FF001299FF00D389FF00D1124EE5DF64F808D19
:207420008C9381E0089580E00895DB018330A0F46115710589F0282F30E083E790E0289FA2
:20744000F001299FF00D389FF00D1124EE5DF64F818D8C9381E0089580E00895DB01833026
:20746000A0F46115710589F0282F30E083E790E0289FF001299FF00D389FF00D1124EE5D01
:20748000F64F828D8C9381E0089580E00895DB018330A0F46115710589F0282F30E083E725
:2074A00090E0289FF001299FF00D389FF00D1124EE5DF64F838D8C9381E0089580E008951C
:2074C000DB018330A0F46115710589F0282F30E083E790E0289FF001299FF00D389FF00D92
:2074E0001124EE5DF64F848D8C9381E0089580E00895DB018330A0F46115710589F0282FBD
:2075000030E083E790E0289FF001299FF00D389FF00D1124EE5DF64F858D8C9381E008953C
:2075200080E00895DB018330A0F46115710589F0282F30E083E790E0289FF001299FF00D08
:20754000389FF00D1124EE5DF64F868D8C9381E0089580E00895DB018330A0F46115710556
:2075600089F0282F30E083E790E0289FF001299FF00D389FF00D1124EE5DF64F878D8C9308
:2075800081E0089580E008958330B0F46930A0F4413890F4282F30E083E790E0289FF00176
:2075A000299FF00D389FF00D1124EE5DF64FE60FF11D40A381E0089580E00895DA018330FE
:2075C000C0F46930B0F44115510599F0282F30E083E790E0289FF001299FF00D389FF00DF3
:2075E0001124EE5DF64FE60FF11D80A18C9381E0089580E00895DB018330A0F46115710579
:2076000089F0282F30E083E790E0289FF001299FF00D389FF00D1124EE5DF64F81A58C9355
:2076200081E0089580E00895DB018330A0F46115710589F0282F30E083E790E0289FF001CE
:20764000299FF00D389FF00D1124EE5DF64F82A58C9381E0089580E00895DB018330A0F468
:207660006115710589F0282F30E083E790E0289FF001299FF00D389FF00D1124EE5DF64F4E
:2076800083A58C9381E0089580E00895DB018330A0F46115710589F0282F30E083E790E0DF
:2076A000289FF001299FF00D389FF00D1124EE5DF64F84A58C9381E0089580E00895DB0195
:2076C0008330A0F46115710589F0282F30E083E790E0289FF001299FF00D389FF00D112437
:2076E000EE5DF64F85A58C9381E0089580E00895DB018330A0F46115710589F0282F30E0C7
:2077000083E790E0289FF001299FF00D389FF00D1124EE5DF64F86A58C9381E0089580E0D1
:207720000895DB018330A0F46115710589F0282F30E083E790E0289FF001299FF00D389F8F
:20774000F00D1124EE5DF64F87A58C9381E0089580E00895DB018330A0F46115710589F099
:20776000282F30E083E790E0289FF001299FF00D389FF00D1124EE5DF64F80A98C9381E009
:20778000089580E00895DB018330A0F46115710589F0282F30E083E790E0289FF001299F06
:2077A000F00D389FF00D1124EE5DF64F81A98C9381E0089580E00895DB018330A0F4611556
:2077C000710589F0282F30E083E790E0289FF001299FF00D389FF00D1124EE5DF64F82A938
:2077E0008C9381E0089580E00895DB018330A0F46115710589F0282F30E083E790E0289FDF
:20780000F001299FF00D389FF00D1124EE5DF64F83A98C9381E0089580E00895DB01833044
:20782000A0F46115710589F0282F30E083E790E0289FF001299FF00D389FF00D1124EE5D3D
:20784000F64F84A98C9381E0089580E00895DB018330A0F46115710589F0282F30E083E743
:2078600090E0289FF001299FF00D389FF00D1124EE5DF64F85A98C9381E0089580E008953A
:20788000DB018330A0F46115710589F0282F30E083E790E0289FF001299FF00D389FF00DCE
:2078A0001124EE5DF64F86A98C9381E0089580E00895DB018330A0F46115710589F0282FDB
:2078C00030E083E790E0289FF001299FF00D389FF00D1124EE5DF64F87A98C9381E008955B
:2078E00080E008958330B0F46930A0F4413890F4282F30E083E790E0289FF001299FF00D4C
:20790000389FF00D1124EE5DF64FE60FF11D40AF81E0089580E00895DA018330C0F4693006
:20792000B0F44115510599F0282F30E083E790E0289FF001299FF00D389FF00D1124EE5D5C
:20794000F64FE60FF11D80AD8C9381E0089580E00895DB018330A0F46115710589F0282FB9
:2079600030E083E790E0289FF001299FF00D389FF00D1124ED59F64F80818C9381E00895EE
:2079800080E00895DB018330A0F46115710589F0282F30E083E790E0289FF001299FF00DA4
:2079A000389FF00D1124EC59F64F80818C9381E0089580E00895833090F4613880F4282F7E
:2079C00030E083E790E0289FF001299FF00D389FF00D1124EB59F64F608381E0089580E06D
:2079E0000895DB018330A0F46115710589F0282F30E083E790E0289FF001299FF00D389FCD
:207A0000F00D1124EB59F64F80818C9381E0089580E00895DB018330A0F46115710589F008
:207A2000282F30E083E790E0289FF001299FF00D389FF00D1124EA59F64F80818C9381E076
:207A4000089580E00895DB018330A0F46115710589F0282F30E083E790E0289FF001299F43
:207A6000F00D389FF00D1124E959F64F80818C9381E0089580E00895DB018330A0F46115C5
:207A8000710589F0282F30E083E790E0289FF001299FF00D389FF00D1124E859F64F8081A9
:207AA0008C9381E0089580E00895DB018330A0F46115710589F0282F30E083E790E0289F1C
:207AC000F001299FF00D389FF00D1124E759F64F80818C9381E0089580E00895DB018330B8
:207AE000A0F46115710589F0282F30E083E790E0289FF001299FF00D389FF00D1124E55889
:207B0000F64F80818C9381E0089580E00895DB018330A0F46115710589F0282F30E083E7AC
:207B200090E0289FF001299FF00D389FF00D1124E458F64F80818C9381E0089580E00895B3
:207B4000DB018330A0F46115710589F0282F30E083E790E0289FF001299FF00D389FF00D0B
:207B60001124E659F64F80818C9381E0089580E00895DB018330A0F46115710589F0282F52
:207B800030E083E790E0289FF001299FF00D389FF00D1124E559F64F80818C9381E00895D4
:207BA00080E00895DB018330A0F46115710589F0282F30E083E790E0289FF001299FF00D82
:207BC000389FF00D1124E459F64F80818C9381E0089580E00895DB018330A0F461157105F0
:207BE00089F0282F30E083E790E0289FF001299FF00D389FF00D1124E359F64F80818C93A4
:207C000081E0089580E00895DB018330A0F46115710589F0282F30E083E790E0289FF001E8
:207C2000299FF00D389FF00D1124E259F64F80818C9381E0089580E00895DB018330A0F4B8
:207C40006115710589F0282F30E083E790E0289FF001299FF00D389FF00D1124E159F64F79
:207C600080818C9381E0089580E00895DB018330A0F46115710589F0282F30E083E790E020
:207C8000289FF001299FF00D389FF00D1124E059F64F80818C9381E0089580E00895DB01E9
:207CA0008330A0F46115710589F0282F30E083E790E0289FF001299FF00D389FF00D112451
:207CC000EF58F64F80818C9381E0089580E00895DB018330A0F46115710589F0282F30E00E
:207CE00083E790E0289FF001299FF00D389FF00D1124EE58F64F80818C9381E0089580E01B
:207D00000895DB018330A0F46115710589F0282F30E083E790E0289FF001299FF00D389FA9
:207D2000F00D1124ED58F64F80818C9381E0089580E00895DB018330A0F46115710589F0E4
:207D4000282F30E083E790E0289FF001299FF00D389FF00D1124EC58F64F80818C9381E052
:207D6000089580E00895DB018330A0F46115710589F0282F30E083E790E0289FF001299F20
:207D8000F00D389FF00D1124EB58F64F80818C9381E0089580E00895DB018330A0F46115A1
:207DA000710589F0282F30E083E790E0289FF001299FF00D389FF00D1124EA58F64F808185
:207DC0008C9381E0089580E00895DB018330A0F46115710589F0282F30E083E790E0289FF9
:207DE000F001299FF00D389FF00D1124E958F64F80818C9381E0089580E00895DB01833094
:207E0000A0F46115710589F0282F30E083E790E0289FF001299FF00D389FF00D1124E85862
:207E2000F64F80818C9381E0089580E00895DB018330A0F46115710589F0282F30E083E789
:207E400090E0289FF001299FF00D389FF00D1124E758F64F80818C9381E0089580E008958D
:207E6000FC01009711F480E008958091620C9091630C9183808381E00895DC01009711F4CF
:207E800080E00895E091B708F091B808EF5BFE4F80818C9381E00895DC01009711F480E0E6
:207EA0000895E091B708F091B808E05CFE4F808180FF03C081E08C9308951C9281E008951F
:207EC000DC01009711F480E00895E091B708F091B808E05CFE4F808181FF03C081E08C936E
:207EE00008951C9281E00895DC01009711F480E00895E091B708F091B808E05CFE4F8081C8
:207F000082FF03C081E08C9308951C9281E00895DC01009711F480E00895E091B708F0912D
:207F2000B808EA5BFE4F80818C9381E00895FC01009711F480E008958091640C9091650C28
:207F40009183808381E00895833010F080E00895282F30E0662371F083E790E0289FF00179
:207F6000299FF00D389FF00D1124E658F64F81E08083089583E790E0289FF001299FF00D58
:207F8000389FF00D1124E658F64F108281E00895DB018330C8F461157105B1F0282F30E086
:207FA00083E790E0289FF001299FF00D389FF00D1124E658F64F8081882319F41C9281E016
:207FC000089581E08C93089580E008956093DB0A7093DC0A8093DD0A9093DE0A81E0089526
:207FE000FC01009711F480E008958091DB0A9091DC0AA091DD0AB091DE0A80839183A28371
:20800000B38381E00895282F833090F4862F8E7F79F430E083E790E0289FF001299FF00D08
:20802000389FF00D1124E358F64F608381E0089580E00895DB018330A0F46115710589F051
:20804000282F30E083E790E0289FF001299FF00D389FF00D1124E358F64F80818C9381E058
:20806000089580E008958330A8F497E0613D790788F4282F30E083E790E0289FF001299F45
:20808000F00D389FF00D1124E258F64F7183608381E0089580E00895DB018330B0F46115E0
:2080A000710599F0282F30E083E790E0289FF001299FF00D389FF00D1124E258F64F80817A
:2080C00091818D939C9381E0089580E00895282F8330D8F4CB0188539F4F81599140A8F492
:2080E00030E083E790E0289FF001299FF00D389FF00D1124E058F64F44E0660F771F4A9585
:20810000E1F77183608381E0089580E00895CF93DF93EB018330D0F461157105B9F0282F92
:2081200030E083E790E0289FF001299FF00D389FF00D1124E058F64F8081918160E170E0AE
:208140000E9414757983688381E001C080E0DF91CF910895282F8330D8F4CB0188539F4FB3
:2081600081599140A8F430E083E790E0289FF001299FF00D389FF00D1124EE57F64F54E08A
:20818000660F771F5A95E1F77183608381E0089580E00895CF93DF93EB018330D0F461158E
:2081A0007105B9F0282F30E083E790E0289FF001299FF00D389FF00D1124EE57F64F80814E
:2081C000918160E170E00E9414757983688381E001C080E0DF91CF910895282F8330D8F425
:2081E000CB018C509E4F895E9340A8F430E083E790E0289FF001299FF00D389FF00D112424
:20820000EC57F64FA4E0660F771FAA95E1F77183608381E0089580E00895CF93DF93EB019E
:208220008330D0F461157105B9F0282F30E083E790E0289FF001299FF00D389FF00D11246B
:20824000EC57F64F8081918160E170E00E9414757983688381E001C080E0DF91CF910895F1
:20826000282F833090F4862F8E7F79F430E083E790E0289FF001299FF00D389FF00D1124D1
:20828000EA57F64F608381E0089580E00895DB018330A0F46115710589F0282F30E083E721
:2082A00090E0289FF001299FF00D389FF00D1124EA57F64F80818C9381E0089580E0089527
:2082C000282F8330C8F4CB014E96CD97A8F430E083E790E0289FF001299FF00D389FF00DED
:2082E0001124E957F64F7695762F6627779567957183608381E0089580E00895CF93DF93D9
:20830000EB018330D0F461157105B9F0282F30E083E790E0289FF001299FF00D389FF00DD3
:208320001124E957F64F8081918160E870E00E9414757983688381E001C080E0DF91CF9174
:208340000895282F8330C8F4CB014E96CD97A8F430E083E790E0289FF001299FF00D389FCC
:20836000F00D1124E757F64F7695762F6627779567957183608381E0089580E00895CF93CF
:20838000DF93EB018330D0F461157105B9F0282F30E083E790E0289FF001299FF00D389FDE
:2083A000F00D1124E757F64F8081918160E870E00E9414757983688381E001C080E0DF9159
:2083C000CF910895282F8330C8F4CB014E96CD97A8F430E083E790E0289FF001299FF00DC3
:2083E000389FF00D1124E557F64F7695762F6627779567957183608381E0089580E00895DC
:20840000CF93DF93EB018330D0F461157105B9F0282F30E083E790E0289FF001299FF00DD2
:20842000389FF00D1124E557F64F8081918160E870E00E9414757983688381E001C080E073
:20844000DF91CF910895282F8330C8F4CB014E96CD97A8F430E083E790E0289FF001299FCF
:20846000F00D389FF00D1124E357F64F7695762F6627779567957183608381E0089580E0FD
:208480000895CF93DF93EB018330D0F461157105B9F0282F30E083E790E0289FF001299FB2
:2084A000F00D389FF00D1124E357F64F8081918160E870E00E9414757983688381E001C058
:2084C00080E0DF91CF9108951F93E091BE08F091BF08E35BFF4F819161917191A191B081A9
:2084E00039973191419150813896919121911081109277081092760810927D0810927C0886
:20850000809382081092840884E6809383086093850870938608A0938708B093880830931F
:20852000890840938A0850938B0890938C0820938D0884ED90E30E940B5790939908809311
:20854000980884ED90E30E940B5790939B0880939A0880E197E20E940B5790939D0880935F
:208560009C081092A208212F2695820F911D612F70E00E94147570939708609396081092E1
:20858000A8081092A70886E798E00E946F391F9108958330B0F46338A4F06E3794F4282F54
:2085A00030E083E790E0289FF001299FF00D389FF00D1124E758F64F60830E94644281E03B
:2085C000089580E008958330B0F46338A4F06E3794F4282F30E083E790E0289FF001299F8D
:2085E000F00D389FF00D1124E858F64F60830E94644281E0089580E008958330B0F46338D8
:20860000A4F06E3794F4282F30E083E790E0289FF001299FF00D389FF00D1124E958F64F4C
:2086200060830E94644281E0089580E008958330A0F4613290F4282F30E083E790E0289FAE
:20864000F001299FF00D389FF00D1124EA58F64F60830E94644281E0089580E008958330FB
:20866000A0F4613890F4282F30E083E790E0289FF001299FF00D389FF00D1124EB58F64FFA
:2086800060830E94644281E0089580E008958330A0F4613890F4282F30E083E790E0289F48
:2086A000F001299FF00D389FF00D1124EC58F64F60830E94644281E0089580E00895833099
:2086C000B0F4603FA4F0613194F4282F30E083E790E0289FF001299FF00D389FF00D1124E2
:2086E000ED58F64F60830E94644281E0089580E008958330B0F4603FA4F0613194F4282FCF
:2087000030E083E790E0289FF001299FF00D389FF00D1124EE58F64F60830E94644281E0D2
:20872000089580E008958330B0F4603FA4F0613194F4282F30E083E790E0289FF001299F3A
:20874000F00D389FF00D1124EF58F64F60830E94644281E0089580E008958330B0F4603F6B
:20876000A4F0613194F4282F30E083E790E0289FF001299FF00D389FF00D1124E059F64F06
:2087800060830E94644281E0089580E008958330A0F4613890F4282F30E083E790E0289F47
:2087A000F001299FF00D389FF00D1124E159F64F60830E94644281E0089580E008958330A2
:2087C000A0F4613890F4282F30E083E790E0289FF001299FF00D389FF00D1124E259F64FA1
:2087E00060830E94644281E0089580E008958330A0F4613890F4282F30E083E790E0289FE7
:20880000F001299FF00D389FF00D1124E359F64F60830E94644281E0089580E0089583303F
:20882000A0F4613890F4282F30E083E790E0289FF001299FF00D389FF00D1124E459F64F3E
:2088400060830E94644281E0089580E008958330A0F4613890F4282F30E083E790E0289F86
:20886000F001299FF00D389FF00D1124E559F64F60830E94644281E0089580E008958330DD
:20888000A0F4613890F4282F30E083E790E0289FF001299FF00D389FF00D1124E659F64FDC
:2088A00060830E94644281E0089580E008956F927F928F92AF92CF92DF92EF920F931F9377
:2088C000DF93CF93CDB7DEB71E856F847888F30111821082178216828487168684E68587AE
:2088E0006787408B218B028BE38AD58AC48AA68A878A84ED90E30E940B57F30191A380A3F8
:2089000084ED90E30E940B57F30193A382A380E197E20E940B57F30195A384A316A6212FE3
:208920002695880F991F820F911D612F70E00E941475758F648F14AA13AA828985AB16AA76
:20894000C3010E94F833CF91DF911F910F91EF90DF90CF90AF908F907F906F9008958F92EF
:208960009F92AF92CF92DF92EF920F931F93CF93DF93E091BE08F091BF0800D00F92DF013A
:20898000909682A5CDB7DEB789838AE99AE09B838A83858D608D418D228D068DE78C6D015D
:2089A000A1A483A40E945744E091BE08F091BF08DF01AF5BBF4F54E4852E912C8E0E9F1E96
:2089C000EE5BFF4F8081E254F040CDB7DEB789838FED9AE09B838A8385A960A941A922A967
:2089E00006A9E7A8F8966F01AC90F40180800E945744E091BE08F091BF08E65AFF4F10812F
:208A0000829180931F080F900F900F9080E197E20E940B579093230880932208880F991F74
:208A2000212F2695820F911D612F70E00E9414757093210860932008DF91CF911F910F917A
:208A4000EF90DF90CF90AF909F908F9008959C01885E9340815A9F4010F080E008953093CF
:208A6000650C2093640C0E94AF4481E00895982F807F11F080E00895E091B708F091B8089A
:208A8000EA5BFE4F90830E9464420E94AF4481E00895E091B708F091B808882329F0E05CE5
:208AA000FE4F8081846004C0E05CFE4F80818B7F80830E94AF4481E00895E091B708F091E5
:208AC000B808882329F0E05CFE4F8081826004C0E05CFE4F80818D7F80830E94AF4481E053
:208AE0000895E091B708F091B808882329F0E05CFE4F8081816004C0E05CFE4F80818E7FDE
:208B000080830E94AF4481E00895823010F080E00895E091B708F091B808EF5BFE4F808305
:208B20000E94AF4481E008959C01865E994F85539C4010F080E008953093630C2093620C35
:208B40000E94AF4481E008958330A0F4613290F4282F30E083E790E0289FF001299FF00D66
:208B6000389FF00D1124E458F64F60830E94AF4481E0089580E008958330A0F4613890F494
:208B8000282F30E083E790E0289FF001299FF00D389FF00D1124E558F64F60830E94AF4414
:208BA00081E0089580E008958330A0F4613890F4282F30E083E790E0289FF001299FF00D98
:208BC000389FF00D1124E759F64F60830E94AF4481E0089580E008958330A0F4613890F430
:208BE000282F30E083E790E0289FF001299FF00D389FF00D1124E859F64F60830E94AF44B0
:208C000081E0089580E008958330A0F4613890F4282F30E083E790E0289FF001299FF00D37
:208C2000389FF00D1124E959F64F60830E94AF4481E0089580E008958330A0F4613890F4CD
:208C4000282F30E083E790E0289FF001299FF00D389FF00D1124EA59F64F60830E94AF444D
:208C600081E0089580E008958330A0F4613290F4282F30E083E790E0289FF001299FF00DDD
:208C8000389FF00D1124EC59F64F60830E94AF4481E0089580E008958330A0F4613890F46A
:208CA000282F30E083E790E0289FF001299FF00D389FF00D1124ED59F64F60830E94AF44EA
:208CC00081E0089580E008958330A0F4623090F4282F30E083E790E0289FF001299FF00D7E
:208CE000389FF00D1124EE5DF64F67AB0E94AF4481E0089580E008958330A0F4613890F4D5
:208D0000282F30E083E790E0289FF001299FF00D389FF00D1124EE5DF64F66AB0E94AF4456
:208D200081E0089580E008958330A0F4613890F4282F30E083E790E0289FF001299FF00D16
:208D4000389FF00D1124EE5DF64F65AB0E94AF4481E0089580E008958330A0F4613890F476
:208D6000282F30E083E790E0289FF001299FF00D389FF00D1124EE5DF64F64AB0E94AF44F8
:208D800081E0089580E008958330A0F4613890F4282F30E083E790E0289FF001299FF00DB6
:208DA000389FF00D1124EE5DF64F63AB0E94AF4481E0089580E008958330A0F4613890F418
:208DC000282F30E083E790E0289FF001299FF00D389FF00D1124EE5DF64F62AB0E94AF449A
:208DE00081E0089580E008958330A0F4613890F4282F30E083E790E0289FF001299FF00D56
:208E0000389FF00D1124EE5DF64F61AB0E94AF4481E0089580E008958330A0F4613890F4B9
:208E2000282F30E083E790E0289FF001299FF00D389FF00D1124EE5DF64F60AB0E94AF443B
:208E400081E0089580E008958330B0F46338A4F06E3794F4282F30E083E790E0289FF0016B
:208E6000299FF00D389FF00D1124EE5DF64F67A70E94AF4481E0089580E008958330A0F4AF
:208E8000613890F4282F30E083E790E0289FF001299FF00D389FF00D1124EE5DF64F66A751
:208EA0000E94AF4481E0089580E008958330A0F4613890F4282F30E083E790E0289FF001C5
:208EC000299FF00D389FF00D1124EE5DF64F65A70E94AF4481E0089580E008958330A0F451
:208EE000613890F4282F30E083E790E0289FF001299FF00D389FF00D1124EE5DF64F64A7F3
:208F00000E94AF4481E0089580E008958330A0F4613890F4282F30E083E790E0289FF00164
:208F2000299FF00D389FF00D1124EE5DF64F63A70E94AF4481E0089580E008958330A0F4F2
:208F4000613290F4282F30E083E790E0289FF001299FF00D389FF00D1124EE5DF64F62A79A
:208F60000E94AF4481E0089580E008958330A0F4613890F4282F30E083E790E0289FF00104
:208F8000299FF00D389FF00D1124EE5DF64F61A70E94AF4481E0089580E008958330A0F494
:208FA000623090F4282F30E083E790E0289FF001299FF00D389FF00D1124EE5DF64F678F4E
:208FC0000E94AF4481E0089580E008958330A0F4613890F4282F30E083E790E0289FF001A4
:208FE000299FF00D389FF00D1124EE5DF64F668F0E94AF4481E0089580E008958330A0F447
:20900000613890F4282F30E083E790E0289FF001299FF00D389FF00D1124EE5DF64F658FE8
:209020000E94AF4481E0089580E008958330A0F4613890F4282F30E083E790E0289FF00143
:20904000299FF00D389FF00D1124EE5DF64F648F0E94AF4481E0089580E008958330A0F4E8
:20906000613890F4282F30E083E790E0289FF001299FF00D389FF00D1124EE5DF64F638F8A
:209080000E94AF4481E0089580E008958330A0F4613890F4282F30E083E790E0289FF001E3
:2090A000299FF00D389FF00D1124EE5DF64F628F0E94AF4481E0089580E008958330A0F48A
:2090C000613890F4282F30E083E790E0289FF001299FF00D389FF00D1124EE5DF64F618F2C
:2090E0000E94AF4481E0089580E008958330A0F4613890F4282F30E083E790E0289FF00183
:20910000299FF00D389FF00D1124EE5DF64F608F0E94AF4481E0089580E008950E94EE568C
:2091200060E870E00E941475862F08952F923F924F925F926F927F928F929F92AF92BF92C0
:20914000CF92DF92EF92FF920F931F93DF93CF93CDB7DEB72E970FB6F894DEBF0FBECDBFDE
:209160005C014B015E874D873901DC86CB86452B09F4DAC50370033051F581E080938408A8
:20918000C7010E948E48282F332727FD309580918208280F311D2138310514F020E830E02A
:2091A00037FF02C020E030E0809183086901C81AD108C601D7FE03C0909581959F4F0397C4
:2091C00034F02093830886E798E00E946F39E091BE08F091BF08E45BFF4F608180E085012B
:2091E00044275527069F90011603580B300D411D581F1124B7E05595479537952795BA955B
:20920000D1F7398728878401EE24FF24069F60011603F80AD00CE11CF81E1124A7E0F59408
:20922000E794D794C794AA95D1F7DF82CE824291EB54F040E42EFF2437FF03C0E759FF4F37
:2092400002C0E559FF4F8081918160E870E00E941475E60EF71EF7FC03C0460F498301C049
:20926000198280E068857985098144275527609F90017003580B300D411D581F112476E094
:2092800055954795379527957A95D1F740900A0150900B01421653064CF0809108019091BA
:2092A00009012901281739070CF42C015092AC084092AB08E091BE08F091BF08EB5AFF4FA1
:2092C0004081442319F41D821C8220C02091D90A3091DA0A37FF03C0309521953F4F80E0A1
:2092E000182FAA27BB274203A10BB10BC0013402B10B900DA11DB11F112467E0B595A795E7
:20930000979587956A95D1F79D838C832C813D813093AE082093AD08E091B708F091B80852
:20932000EF5BFE4F8081813029F4309521953F4F3D832C83E091BE08F091BF08EA5AFF4F3E
:209340004081442319F41B821A8220C020911E0B30911F0B37FF03C0309521953F4F80E098
:20936000582FAA27BB274203A50BB50BC0013402B50B900DA11DB51F112457E0B595A79526
:20938000979587955A95D1F79B838A836A817B817093B0086093AF08A091B708B091B80866
:2093A000AF5BBE4F5C91A154B140513029F4709561957F4F7B836A83E091BE08F091BF08F2
:2093C000E95AFF4F4081442319F42224332422C0AE5BBE4F8D919C919301281B390B37FF96
:2093E00003C0309521953F4F80E0782FAA27BB274203A70BB70BC0013402B70B900DA11D1A
:20940000B71F112447E0B595A795979587954A95D1F71C01513021F4309421943108339479
:209420003092B2082092B108AD85BE8514960D911C911597E091B708F091B808E05CFE4F35
:20944000808182FF03C0109501951F4FED85FE85F085FA878091210990E038E0E32EF12C42
:20946000E822F92283FD03C08884998416C080E02EEB48855985A82F88279927429FB00189
:2094800052039A0B700D811D9A1F112420E031E040E050E00E9449754901B401601B710B12
:2094A00080918408882319F08091830802C080918208A82FB0E0EFEF003C1E071CF4E0E0EC
:2094C00021E007C00134110514F0E1E001C0E0E020E0CB0177FF04C088279927861B970B7B
:2094E0008134910504F197FE10C010161106ECF0C4018054904008171907BCF0C401805CB9
:209500009F4F80179107A4F00EC017FD0EC0C401805C9F4F8017910744F0C401805490408F
:20952000081719072CF050E001C051E040E002C050E041E0222319F420E030E006C0809142
:209540008508282F332727FD3095EE2339F080918608992787FD9095280F391F442339F083
:2095600080918708992787FD9095280F391F552339F080918808992787FD9095280F391F19
:20958000C9018A0F9B1F97FF03C020E030E007C0813891051CF020E830E001C09C01EF2896
:2095A000C9F480E0F82F7303D001629FC0017203BF0B900DA11DBF1F639F900DA11DBF1FAB
:2095C000112425E0B595A795979587952A95D1F75C012AC040E0AA27BB27629FC0017203AB
:2095E000B40B900DA11DB41F11242DE030E06C017D01D39EC001C29EB001D29E700D811D73
:20960000941FC39E700D811D941FE29E800D911DF29E900DE39E900D112420E031E040E0FC
:2096200050E00E94497559012091890880E0A501EE24FF24429F60015203F80AD00CE11C51
:20964000F81E1124F5E0F594E794D794C794FA95D1F76090980870909908C301AA2797FD6F
:20966000A095BA2F8C159D05AE05BF057CF07094619471087394C301AA2797FDA095BA2FE6
:20968000C816D906EA06FB060CF0360180918A08882359F410927E0810927F0810928008D3
:2096A000109281081E861D8644C15A855523C1F080917E0890917F08A0918008B091810869
:2096C000181619061A061B062CF41A141B040CF460C006C00097A105B10511F0B7FC59C0E9
:2096E000C0907E08D0907F08E0908008F09081088091A2088B3024F0C50168E070E005C0FF
:2097000018165CF4C50164E070E00E941475CB01AA2797FDA095BA2F05C0C501AA2797FD07
:20972000A095BA2F8C0D9D1DAE1DBF1DC0909E08D0909F08E090A008F090A108C816D90616
:20974000EA06FB064CF4C0927E08D0927F08E0928008F09281081DC022273327A9012C19A3
:209760003D094E095F0982179307A407B5074CF420937E0830937F084093800850938108C0
:2097800008C080937E0890937F08A0938008B093810880917808909179088819990997FF2B
:2097A00003C0909581959F4F893091052CF08114910411F084E114C004974CF08091A2085C
:2097C0008A302CF48114910411F08AE009C08091A208181614F4815003C0882319F08F5F2A
:2097E0008093A20840917E0850917F08609180087091810820918A0880E0629F7001429FF4
:209800006001E80AF80A529FD00CE11CF81E7203F00C1124E9E0F594E794D794C794EA955B
:20982000D1F780919A0890919B089E878D87FC01CF01AA2797FDA095BA2F8C159D05AE056A
:20984000BF058CF0F095E195FF4FFE87ED87CF01AA2797FDA095BA2FC816D906EA06FB0685
:2098600014F0DE86CD86FA85FF2311F1141615061606170624F41A141B048CF019C04115FC
:20988000510561057105A1F0B7FE12C0C0909208D0909308E0909408F090950817C0809188
:2098A000920890919308A0919408B091950827C080918C088038E9F177FF19C0C0908E0854
:2098C000D0908F08E0909008F090910888279927DC018C199D09AE09BF0984179507A60776
:2098E000B70790F04C0D5D1D6E1D7F1D1AC080918E0890918F08A0919008B09191084817F5
:2099000059076A077B0748F410927E0810927F0810928008109281080CC0481B590B6A0B0A
:209920007B0B40937E0850937F08609380087093810860918B08662319F460E070E08AC0E3
:2099400080917A0890917B08CE80DF80C81AD90A9601442737FD4095542FDA01C901039692
:20996000A11DB11D0797A105B10528F420E030E040E050E011C02D3F7FEF37077FEF470740
:209980007FEF57072CF42C5F3F4F4F4F5F4F04C0245030404040504080E0469F7001269F43
:2099A0006001E80AF80A369FD00CE11CF81E5603F00C1124E091A708F091A8086091960824
:2099C0007091970888279927861B970BE817F9073CF46E0F7F1F7093A8086093A7080EC0C8
:2099E0006E177F073CF4E61BF70BF093A808E093A70804C01092A8081092A708F594E79469
:209A0000D794C7948091A7089091A808AA2797FDA095BA2FC80ED91EEA1EFB1E60919C08E9
:209A200070919D08CB01AA2797FDA095BA2F8C159D05AE05BF0574F0709561957F4FCB017E
:209A4000AA2797FDA095BA2FC816D906EA06FB060CF0B6011093770800937608909279084C
:209A6000809278088E819F8190937B0880937A08B0927D08A0927C082D853E85260D371D71
:209A8000260F371F7092A4086092A308AD85BE85B093A608A093A5087093A8086093A70855
:209AA0003093AA082093A908E091BE08F091BF08EE59FF4F8081918160E170E00E941475EA
:209AC000640D751DEC81FD816E0F7F1FCA80DB806C0D7D1D620D731D620F731FAB85BC8552
:209AE00011967C936E9380910A0190910B01861797071CF48D939C930BC0809108019091C6
:209B000009016817790724F4EB85FC8591838083AB85BC858D919C919093B4088093B308B3
:209B20008091DD02833009F05EC08091A5089091A608BFEF88339B071CF00333110554F037
:209B4000E091BE08F091BF08EE59FF4F80819181059731C0EFEF863F9E071CF003301105B4
:209B600054F0E091BE08F091BF08EE59FF4F80819181019720C0893C910524F4FFEF0E3C57
:209B80001F0754F4E091BE08F091BF08EE59FF4F8081918105960FC00B9724F42FEF0E3FA1
:209BA00012075CF4E091BE08F091BF08EE59FF4F80819181019691838083E091BE08F091AF
:209BC000BF08EE59FF4F808191813FE1813493071CF080E49FE105C0805C904E24F480ECB4
:209BE00090EE91838083E091BE08F091BF08EC59FF4F8081E456F040882309F495C0C8018D
:209C000017FF03C0909581959F4F853691050CF48BC068857985645D7E4F54F4AB85BC8574
:209C20008D919C91E759FF4F841595059CF40EC0088519850D52114094F0AB85BC858D91CC
:209C40009C91E559FF4F4816590624F480819181019603C080819181019791838083B9810D
:209C60002B2F30E0E091BE08F091BF08E759FF4F8081918160E870E00E941475620F731F94
:209C800077FF0BC080E890E06C01E980CE9CC001DE9C900D112491838083E091BE08F0918F
:209CA000BF08E759FF4F8081918101EF803090071CF480E091EF05C081509F4024F080E02C
:209CC0009FE091838083E091BE08F091BF08E559FF4F8081918160E870E00E941475260FD8
:209CE000371F37FF0BC080E890E09C014981249FC001349F900D112491838083E091BE0857
:209D0000F091BF08E559FF4F8081918151EF803095071CF480E091EF05C081509F4024F057
:209D200080E09FE0918380832E960FB6F894DEBF0FBECDBFCF91DF911F910F91FF90EF90F4
:209D4000DF90CF90BF90AF909F908F907F906F905F904F903F902F9008952F923F924F92DF
:209D60005F926F927F928F929F92AF92BF92CF92DF92EF92FF920F931F93DF93CF93CDB76C
:209D8000DEB727970FB6F894DEBF0FBECDBF3C012B011A01922EFD82EC82DF82CE826501E1
:209DA000EF2809F4EAC2C8010E948E489091EB0A282F332727FD3095290F311D37FF02C074
:209DC00090E006C02138310514F090E801C0980F19E091229116C9F481E08093ED0A292F07
:209DE000332727FD30958091EC0A281B310937FF03C0309521953F4F2330310534F09093CA
:209E0000EC0A8FED9AE00E94F833E091BE08F091BF0834A920E0A301AA27BB27439FC00133
:209E20005303B20B900DA11DB21F112417E0B595A795979587951A95D1F79B838A83B20194
:209E400088249924639F30017303920A700C811C921E112443A9E959FF4F8081918160E87F
:209E600070E00E941475CB01840F911D97FF02C0198202C0460F498380E06A817B811981A3
:209E800044275527619F90017103580B300D411D581F112476E055954795379527957A9579
:209EA000D1F740900A0150900B01421653064CF080910801909109012901281739070CF438
:209EC0002C015092190B4092180B60911F08662321F4D6012D923C92BEC080911D0890916B
:209EE0001E08F101E81BF90B9F01442737FD4095542FDA01C9018796A11DB11D8F34910505
:209F0000A105B10528F420E030E040E050E011C0293DFFEF3F07FFEF4F07FFEF5F072CF446
:209F2000285D3F4F4F4F5F4F04C0285230404040504080E0469F8001269F7001080B180BD2
:209F4000369FF00C011D181F5603100D1124409124085091250820912008309121088827B3
:209F60009927821B930B481759073CF4240F351F30932508209324080EC0241735073CF42C
:209F8000421B530B509325084093240804C01092250810922408A801970163E0559547954C
:209FA000379527956A95D1F78091240890912508AA2797FDA095BA2F280F391F4A1F5B1FD2
:209FC0006091220870912308CB01AA2797FDA095BA2F82179307A407B50724F4D6016D9362
:209FE0007C9315C0EE27FF27E61BF70BCF01AA2797FDA095BA2F281739074A075B0724F4A2
:20A00000D601ED93FC9303C0F60131832083D6018D919C91119790932508809324088D91D2
:20A020009C911197820D931D11969C938E9320910A0130910B01281739071CF42D933C936E
:20A040000AC02091080130910901821793071CF4F6013183208330921E0820921D08AC8134
:20A06000BD811296AD90BC901397E091B708F091B808E05CFE4F808181FF04C0B094A1940F
:20A08000B108B39447E095948794779467944A95D1F78A819B81B301A501EC81FD81278194
:20A0A00081013FEDE32E3AE0F32ECC24C3940E94B4347C01E091BE08F091BF08E05AFF4F51
:20A0C000008111817D974081442319F4E0E0F0E040C0E091B708F091B808EE5BFE4F0190FC
:20A0E000F081E02DE219F309F7FF08C02FEFEA36F2075CF49F012A563F4F09C0E739F10519
:20A1000024F09F012659304002C020E030E080E0582F88279927249FB0013403950B700DAC
:20A12000811D951F112420E031E040E050E00E944975E0910A01F0910B01E217F3074CF09F
:20A140008091080190910901F901281739070CF4FC01F0931B0BE0931A0BC80160E170E0A9
:20A160000E941475640D751D6E0D7F1D6E0F7F1FAE81BF8111967C936E9380910A0190911C
:20A180000B01861797074CF080910801909109016817790724F4AE81BF818D939C93AE81F3
:20A1A000BF818D919C9190931F0B80931E0B8091DD02833009F073C08091100B9091110B53
:20A1C0008E0F9F1FBFEF88339B0724F0E3E3AE16B10454F0E091BE08F091BF08E05AFF4F7B
:20A1E00080819181059734C0FFEF863F9F0724F013E0A116B10454F0E091BE08F091BF082D
:20A20000E05AFF4F80819181019722C0893C91052CF42EECA2162FEFB20654F4E091BE0887
:20A22000F091BF08E05AFF4F80819181059610C00B972CF43EEFA3163FEFB3065CF4E09180
:20A24000BE08F091BF08E05AFF4F80819181019691838083E091BE08F091BF08E45AFF4F9C
:20A260008081918147E0803D940718F4019691838083E091BE08F091BF08E05AFF4F80818A
:20A2800091815CE0813895071CF080E89CE005C08058934F24F480E893EF91838083E09122
:20A2A000BE08F091BF08EC59FF4F8081E456F040882309F462C0A501B7FE03C050954195EF
:20A2C0005F4F453651050CF458C08A819B81845D9E4F54F4AE81BF818D919C91E959FF4F60
:20A2E000841595059CF40EC02A813B812D52314094F0AE81BF818D919C91E959FF4F48164A
:20A30000590624F480819181019603C080819181019791838083E091BE08F091BF08E959D6
:20A32000FF4F8081918160E870E00E941475B9816B0F711D77FF0BC080E890E09C014B2F87
:20A34000249FC001349F900D112491838083E091BE08F091BF08E959FF4F8081918151EF5B
:20A36000803095071CF480E091EF05C081509F4024F080E09FE09183808327960FB6F89414
:20A38000DEBF0FBECDBFCF91DF911F910F91FF90EF90DF90CF90BF90AF909F908F907F90E0
:20A3A0006F905F904F903F902F9008952F923F924F925F926F927F928F929F92AF92BF924B
:20A3C000CF92DF92EF92FF920F931F93DF93CF93CDB7DEB763970FB6F894DEBF0FBECDBF17
:20A3E0009A8389837C836B835E834D832F8319870887FB86EA86DD86CC86EF2809F4F8C241
:20A40000E091BE08F091BF08E85AFF4F8081882309F4F4C0C090B508D090B608E091B70875
:20A42000F091B808EC5BFE4FE080F180A6E0F594E794AA95E1F7C601B7010E9414758B019F
:20A440003497808182FD03C0109501951F4FC601B7010E9414759093B6088093B508C80121
:20A460000E9429702C01C8010E94A1709B8B8A8B40911A0B50911B0B20E032E010E0530368
:20A48000C001429FB0015203910B700D811D911F439F700D811D911F1124E091BE08F09113
:20A4A000BF0821A930E040E050E00E94497579018A018091A20A9091A30AA091A40AB0919B
:20A4C000A50A9C01AD016A897B89E0E073036001269F5001369FB00CC11CDE1E7203DE0A17
:20A4E000B00CC11CDE1E469FC00CD11C569FD00C479FD00C11242091E70A3091E80A40913B
:20A50000E90A5091EA0A2E0D3F1D401F511F2E873F87488B598BB20173034001269F30017B
:20A52000369F700C811C9E1E72039E0A700C811C9E1E469F800C911C569F900C479F900C4E
:20A5400011249C01AD0173032001269F1001369F300C411C5E1E72035E0A300C411C5E1E32
:20A56000469F400C511C569F500C479F500C11242E853F85488959896A897B897303D0010D
:20A58000269FC001369F900DA11DBE1F7203BE0B900DA11DBE1F469FA00DB11D569FB00DA0
:20A5A000479FB00D1124A618B708C808D908FDE0D594C794B794A794FA95D1F7A092A20A39
:20A5C000B092A30AC092A40AD092A50A820D931DA41DB51DEDE0B595A79597958795EA958F
:20A5E000D1F78E199F09A00BB10B8093E70A9093E80AA093E90AB093EA0A04C01092B60843
:20A600001092B508888599850E948E489091A60A282F332727FD3095290F311D37FF02C04F
:20A6200090E006C02138310514F090E801C0980F7F8175707530C9F481E08093A80A292FAC
:20A64000332727FD30958091A70A281B310937FF03C0309521953F4F2330310534F09093A6
:20A66000A70A8AE99AE00E94F833E091BE08F091BF08348D20E049815A8100271127439F49
:20A6800070015303120BF00C011D121F112477E015950795F794E7947A95D1F737016B81B8
:20A6A0007C8144245524639F10017303520A300C411C521E1124438DEB59FF4F8081918124
:20A6C00060E870E00E941475CB01840F911D97FF02C0DD2402C0D42ED60E80E0B3011D2D4B
:20A6E00044275527619F90017103580B300D411D581F112466E055954795379527956A9531
:20A70000D1F780900A0190900B01821693064CF080910801909109014901281739070CF4AF
:20A720004C019092D40A8092D30AE091BE08F091BF0887A5882319F41B8A1A8A22C00E94AD
:20A740006C5EE091BE08F091BF0837A520E0AC01AA27BB273403A20BB20BC0015302B20B00
:20A76000900DA11DB21F112457E0B595A795979587955A95D1F766277727681B790B7B8B84
:20A780006A8B8A899B899093D80A8093D70AAA85BB85AD90BC90E091B708F091B808E05CEF
:20A7A000FE4F808180FF04C0B094A194B108B39447E055944794379427944A95D1F7C301B3
:20A7C000B101A501EA85FB8526810D811E813AE9E32E3AE0F32ECC240E94B4349C01E09167
:20A7E000BE08F091BF08E25AFF4F8081918160E170E00E941475680D791D4A895B89640FBD
:20A80000751F620F731FAC85BD8511967C936E9380910A0190910B01861797071CF48D93C3
:20A820009C930BC080910801909109016817790724F4EC85FD8591838083AC85BD858D9127
:20A840009C919093DA0A8093D90A8091DD02833009F062C08091CB0A9091CC0ABFEF8833CA
:20A860009B0724F0E3E3AE16B10454F0E091BE08F091BF08E25AFF4F80819181059734C0F3
:20A88000FFEF863F9F0724F013E0A116B10454F0E091BE08F091BF08E25AFF4F808191818C
:20A8A000019722C0893C91052CF42EECA2162FEFB20654F4E091BE08F091BF08E25AFF4FAA
:20A8C00080819181059610C00B972CF43EEFA3163FEFB3065CF4E091BE08F091BF08E25A60
:20A8E000FF4F80819181019691838083E091BE08F091BF08E25AFF4F808191814CE0813848
:20A9000094071CF080E89CE005C08058934F24F480E893EF91838083E091BE08F091BF0895
:20A92000EC59FF4F8081E456F040882309F460C0A501B7FE03C0509541955F4F45365105F9
:20A940000CF456C064ED66166EEF760654F4AC85BD858D919C91EB59FF4F881599059CF4D8
:20A960000EC0BDE26B16B1E07B0694F0AC85BD858D919C91EB59FF4F8816990624F48081AD
:20A980009181019603C080819181019791838083E091BE08F091BF08EB59FF4F8081918165
:20A9A00060E870E00E9414756D0D711D77FF0AC080E890E09C012D9DC0013D9D900D1124E0
:20A9C00091838083E091BE08F091BF08EB59FF4F8081918131EF803093071CF480E091EFE2
:20A9E00005C081509F4024F080E09FE09183808363960FB6F894DEBF0FBECDBFCF91DF91C8
:20AA00001F910F91FF90EF90DF90CF90BF90AF909F908F907F906F905F904F903F902F90C4
:20AA200008951F920F920FB60F9211240F931F932F933F934F935F936F937F938F939F9368
:20AA4000AF93BF93EF93FF93809120099091E202882309F45DC0992309F0F0C04F9BEEC04D
:20AA600020918400309185007894409107014830D0F5A42FB0E0AA0FBB1FFD01E45BFB4FBC
:20AA800080819181B901681B790BCB0177E28131970760F030934D0420934C04463090F10F
:20AAA00080916A0C8F5F80936A0C2CC0A45CBB4F11969C938E93E42FEF5FE0930701E830B7
:20AAC00041F0F0E0EE0FFF1FE45BFB4F318320831BC030934D0420934C0480916A0C8F5F13
:20AAE00080936A0C11C080914C0490914D04A901481B590BCA0130934D0420934C04815104
:20AB0000974210F010920701F8941092E20296C08091E30291110C941856939509B10C7F37
:20AB200020918400309185007894102F182712FF12C002FF05C020934C0430934D040BC085
:20AB4000A90160914C0470914D04461B570B40933C0450933D0413FF12C003FF05C0209360
:20AB60004E0430934F040BC0A90160914E0470914F04461B570B40933E0450933F0414FF50
:20AB800012C004FF05C020935004309351040BC0A9016091500470915104461B570B409356
:20ABA00040045093410415FF13C005FF05C020935204309353040CC0A90160915204709198
:20ABC0005304461B570B4093420450934304E39516FF12C006FF05C02093540430935504C8
:20ABE0000BC0A9016091540470915504461B570B409344045093450417FF12C007FF05C080
:20AC000020935604309357040BC0A9016091560470915704461B570B4093460450934704DF
:20AC2000802FF89409B10C7F80130C949055912D8093E3029093E202E0936A0CFF91EF91C6
:20AC4000BF91AF919F918F917F916F915F914F913F912F911F910F910F900FBE0F901F909A
:20AC60001895DA018330C0F46830B0F44115510599F0282F30E083E790E0289FF001299FB3
:20AC8000F00D389FF00D1124EE5DF64FE60FF11D85818C9381E0089580E008958330B0F4A4
:20ACA0006830A0F4413890F4282F30E083E790E0289FF001299FF00D389FF00D1124EE5D59
:20ACC000F64FE60FF11D458781E0089580E00895DA018330C0F46830B0F44115510599F0B2
:20ACE000282F30E083E790E0289FF001299FF00D389FF00D1124EE5DF64FE60FF11D8585F0
:20AD00008C9381E0089580E00895E82F809120098823C9F18091350B81FF11C0E43009F4B0
:20AD200046C0E53030F4E230F1F1E33009F048C03CC0E530F1F1E63009F042C03CC082FF4B
:20AD400010C0E330B1F1E43028F4E130A1F1E230B0F533C0E53049F1E53048F1E63081F5C8
:20AD600022C083FF2DC0E33001F1E43028F4E13011F1E230C0F421C0E530D9F0E530B8F0F8
:20AD8000E630F1F41CC0E23091F0E33028F4EE2351F0E130A9F40DC0E43079F0E43058F074
:20ADA000E53071F40CC0E5E00BC0E6E009C0E3E007C0E4E005C0E2E003C0E1E001C0E0E054
:20ADC000F0E0EE0FFF1FE45CFB4F8FB7F894208131818FBF265A3E40C901089533E0880F7C
:20ADE000991F3A95E1F7AA2797FDA095BA2FBC01CD010E94937220E030E040EA51E40E942E
:20AE0000E77120E030E040EA51E40E94ED700E94F172CB010895AA2797FDA095BA2FBC01BE
:20AE2000CD010E94937220E030E040EA51E40E94ED7020E030E040EA51E40E94E77120E0C6
:20AE400030E040E05EE30E94ED700E94F172CB010895833090F4613880F4282F30E083E7FF
:20AE600090E0289FF001299FF00D389FF00D1124EE5DF64F658B81E0089580E00895DB0185
:20AE80008330A0F46115710589F0282F30E083E790E0289FF001299FF00D389FF00D11243F
:20AEA000EE5DF64F85898C9381E0089580E00895833090F4613880F4282F30E083E790E055
:20AEC000289FF001299FF00D389FF00D1124EE5DF64F668B81E0089580E00895DB018330E1
:20AEE000A0F46115710589F0282F30E083E790E0289FF001299FF00D389FF00D1124EE5D47
:20AF0000F64F86898C9381E0089580E00895833090F4613880F4282F30E083E790E0289F77
:20AF2000F001299FF00D389FF00D1124EE5DF64F678B81E0089580E00895DB018330A0F4B2
:20AF40006115710589F0282F30E083E790E0289FF001299FF00D389FF00D1124EE5DF64F35
:20AF600087898C9381E0089580E008958823A9F0CA01821B930B97FF03C0909581959F4FDB
:20AF80006817790750F44217530724F4A901461B570B03C0A901460F571F86E04B315807BD
:20AFA00014F04AE156E089EF463E580714F446EE59EFCA010895CF93DF93E82F9B01EA0173
:20AFC0008091DF028E17B9F0EE2349F0E03839F486E090E090930201809301010AC08DE05A
:20AFE00093E06E2F70E00E9414757093020160930101E093DF0260910101709102018E2FC3
:20B00000A9019E010E94B657DF91CF910895CF93DF93E82F9B01EA018091E0028E17B9F018
:20B02000EE2349F0E03839F489E190E090930401809303010AC084E39CE06E2F70E00E942C
:20B0400014757093040160930301E093E00260910301709104018E2FA9019E010E94B65763
:20B06000DF91CF910895CF93DF93E82F9B01EA018091E1028E17B9F0EE2349F0E03839F420
:20B0800089E190E090930601809305010AC084E39CE06E2F70E00E941475709306016093D1
:20B0A0000501E093E10260910501709106018E2FA9019E010E94B657DF91CF91089581385A
:20B0C00010F080E008958093340B81E00895FC01009711F480E008958091340B808381E0D9
:20B0E0000895982F887F11F080E00895E091B708F091B808938B81E00895DC01009711F4E1
:20B1000080E00895E091B708F091B80883898C9381E00895982F807711F080E00895E0916B
:20B12000B708F091B808958B81E00895DC01009711F480E00895E091B708F091B8088589FC
:20B140008C9381E008959C01865E994F85539C4010F080E00895E091B708F091B808378B85
:20B16000268B81E00895DC01009711F480E00895E091B708F091B808868997898D939C93BB
:20B1800081E008959C01865E994F85539C4010F080E00895E091B708F091B808318F208FB7
:20B1A00081E00895DC01009711F480E00895E091B708F091B808808D918D8D939C9381E0CF
:20B1C000089599E0899FC00111248C509C4F0E94F56D0895FF920F931F93182FF62E042F50
:20B1E0000E948556BC0186E06B31780714F06AE176E09B0199EF663E790714F426EE39EF63
:20B20000002351F089E0189FC00111248C509C4FB9010E94F56D9C01FF2051F0E12FF0E052
:20B22000EE0FFF1FEC51FD4F80819181281B390BE091BE08F091BF08E10FF11D8585682FB2
:20B2400070E0621773072CF4C901861B970BBC010CC088279927861B970B281739071CF0B8
:20B2600060E070E002C0620F731FCB011F910F91FF9008950F931F93162F042F833010F5AD
:20B28000683000F54530F0F4282F30E083E790E0289FF001299FF00D389FF00D1124EE5DB6
:20B2A000F64FE60FF11D4583862F0E948556AC0189E0189FC00111248C509C4F602F0E9491
:20B2C000B76D01C080E01F910F910895CF92DF92EF92FF920F931F93D82E67E0681708F43C
:20B2E0005BC00E9485568FE798E3A1E081509040A040E1F700C00000CC24EE24FF2487017E
:20B300008D2D0E948556AA2797FDA095BA2FE80EF91E0A1F1B1F0E94416F8FE798E3A1E03F
:20B3200081509040A040E1F700C00000C39490E1C91631F7A801970164E05595479537950E
:20B3400027956A95D1F7DA01C90188539F4FAF4FBF4F81599140A040B040F0F4ED2DF0E0A7
:20B36000EE0FFF1FEC51FD4F3183208381E0D81649F0D81620F094E0D91679F40AC087EA41
:20B3800092E002C089EA92E0B9010E94D77581E004C08BEA92E0F8CF80E01F910F91FF90DA
:20B3A000EF90DF90CF90089587EA92E00E94B3759093E5028093E40289EA92E00E94B37544
:20B3C0009093E7028093E6028BEA92E00E94B3759093ED028093EC0281E008950F931F9350
:20B3E000CF93DF9310926A0C80E090E0FC01E45BFB4F11821082FC01EC51FD4F118210823B
:20B4000002968031910591F7C4EFD3E004EF12E0CE0164E040E198010E946C6D882361F135
:20B420002996005E1F4F84E0CC33D80789F78091350B80FF0EC081E0809320094F9A5798AC
:20B440008091680088608093680080917300806810C01092200989B18C6F89B98AB1837064
:20B460008AB980916800886080936800809173008C6F8093730081E0DF91CF911F910F9127
:20B4800008951F920F920FB60F9211248F93EF93FF9381E08093990AE3EBF0E080818D5356
:20B4A0008083FF91EF918F910F900FBE0F901F9018951F920F920FB60F9211248F939F93B1
:20B4C000AF93BF938091840090918500179B06C01798A0917504B091760405C0179AA0916A
:20B4E0007704B0917804A80FB91FB0938B00A0938A00BF91AF919F918F910F900FBE0F900F
:20B500001F9018951F920F920FB60F9211242F933F934F935F938F939F93EF93FF93409141
:20B5200084005091850020910C0128B930915C04E32FF0E0EE0FFF1FE759FB4F80819181C7
:20B54000840F951F90938900809388003F5F30935C04220F20930C01353011F4169A08C0C9
:20B56000363031F4169810925C0484E080930C01FF91EF919F918F915F914F913F912F914C
:20B580000F900FBE0F901F9018951092800092E0909381001092B00084E08093B10090936F
:20B5A00070000895EFE6F0E08081826080830895EFE6F0E08081846080830895CF93DF9358
:20B5C000EB016091690470916A0440916B0450916C0420916D0430916E04460F571F420FB0
:20B5E000531F20916F0430917004420F531F2091710430917204A82FBB27A7FDB095FD01C0
:20B60000EE0FFF1FE759FB4F808191812C0F3D1F281B390B240F351FE091B708F091B8085C
:20B62000428D538DCA01C2972817390718F022E330E004C0CA01821B930B9C018FB7F89462
:20B64000AA0FBB1FA759BB4F1196DC93CE9330937404209373048FBFDF91CF910895282F5F
:20B66000843010F080E00895E091B708F091B808662361F081E090E002C0880F991F2A952D
:20B68000E2F7248D282B248F81E0089581E090E002C0880F991F2A95E2F78095248D282391
:20B6A000248F81E00895282FDB018430B0F46115710599F0E091B708F091B808848D90E0E7
:20B6C00002C0959587952A95E2F780FF03C081E08C9308951C9281E0089580E0089523ECB3
:20B6E0008035920731F021E6883A920711F080E00895E091B708F091B808938F828F81E076
:20B700000895DC01009711F480E00895E091B708F091B808828D938D8D939C9381E0089529
:20B72000843058F46E3748F4E091B708F091B808E80FF11D658F81E0089580E00895DB01E7
:20B74000843068F46115710551F0E091B708F091B808E80FF11D858D8C9381E0089580E0A7
:20B760000895843058F46E3748F4E091B708F091B808E80FF11D61A381E0089580E00895D6
:20B78000DB01843068F46115710551F0E091B708F091B808E80FF11D81A18C9381E00895DB
:20B7A00080E008958430A8F49EEF6C3079078CF091E0653F79076CF4E091B708F091B808B1
:20B7C00090E0880F991FE80FF91F76A365A381E0089580E00895DB01843090F4611571057F
:20B7E00079F0E091B708F091B80890E0880F991FE80FF91F85A196A18D939C9381E00895F7
:20B8000080E008959F92AF92BF92CF92DF92EF92FF920F931F93CF93DF93982ECB0126E0C4
:20B820006B31720714F08AE196E09C0149EF863E940714F426EE39EFA92CBB24F501EE0FEF
:20B84000FF1FDF01A35ABB4F2D933C93C090B708D090B808EC0DFD1D85A196A1820F931F72
:20B860007C010027F7FC0095102FF601EA0DFB1D1816190614F4258D01C021A130E040E09D
:20B8800050E0C801B7010E94E17457E095958795779567955A95D1F7EB01D6015C968C91F2
:20B8A00090E002C095958795AA94E2F780FF03C0D095C195DF4FF60187A98823F1F18E018B
:20B8C000D7FF04C0002711270C1B1D0BC8016CE070E00E941475862F8F5F843870F5E62FB7
:20B8E000F0E07C96EE0FFF1FEC0DFD1D0190F081E02D90E04C96880F991FC80ED91ED601E4
:20B900002D913C912E1B3F0BC8016CE070E00E941475AC01249FC001259F900D349F900D77
:20B9200011246CE070E00E9400756E0F7F1FD7FF05C0709561957F4F01C0BE016A55714FA1
:20B94000892D0E94DE5ADF91CF911F910F91FF90EF90DF90CF90BF90AF909F900895BC0144
:20B9600086E06B31780714F06AE176E089EF663E780714F466EE79EF70936404609363047D
:20B980006A55714F83E00E94DE5A0895E82FF0E0EE0FFF1FE35AFB4F80819181089526E00F
:20B9A0008B31920714F08AE196E029EF863E920714F486EE99EF9093680480936704BC010A
:20B9C0006A55714F2091690430916A0440916B0450916C0480916D0490916E04420F531F32
:20B9E000480F591F80916F0490917004480F591F460F571FE091B708F091B808228D338DE5
:20BA0000C901C2974817590718F022E330E002C0241B350B8FB7F894709372046093710433
:20BA200030937404209373048FBF089580916704909168040895E091B708F091B8088823F4
:20BA400019F081E080AB01C010AA81E00895DC01009711F480E00895E091B708F091B808F1
:20BA600080A9813011F48C9308951C9281E0089523EC8035920791F021E6883A920771F0DE
:20BA800027E28031920751F022E28234920731F02DE18C34920711F080E00895E091B70809
:20BAA000F091B80897A786A781E00895DC01009711F480E00895E091B708F091B80886A5CA
:20BAC00097A58D939C9381E008958E3710F080E00895E091B708F091B80881AB81E0089580
:20BAE000DC01009711F480E00895E091B708F091B80881A98C9381E008958E3710F080E0F3
:20BB00000895E091B708F091B80882AB81E00895DC01009711F480E00895E091B708F091C5
:20BB2000B80882A98C9381E008952EE0863A920751F029E08830920731F027E08C36920778
:20BB400011F080E00895E091B708F091B80894AB83AB81E00895DC01009711F480E0089595
:20BB6000E091B708F091B80883A994A98D939C9381E008959C018C509E4F895E934010F07E
:20BB800080E00895E091B708F091B80836AB25AB81E00895DC01009711F480E00895E091A1
:20BBA000B708F091B80885A996A98D939C9381E00895E091B708F091B80885A781E0089530
:20BBC000DC01009711F480E00895E091B708F091B80885A58C9381E00895EF92FF920F9383
:20BBE0001F93CF93DF9326E08B31920714F08AE196E09C0189EF263E380714F426EE39EF83
:20BC00003093660420936504C091B708D091B8088DA99EA9820F931F7C010027F7FC0095BE
:20BC2000102F1816190614F429A901C02AA930E040E050E0C801B7010E94E174E7E0959541
:20BC4000879577956795EA95D1F788A9882319F0709561957F4F8BA99CA9860F971F2EA534
:20BC60003FA5281B390B4FB7F894909378048093770430937604209375044FBFDF91CF9153
:20BC80001F910F91FF90EF90089580E060E070E00E94025C81E060E070E00E94025C82E066
:20BCA00060E070E00E94025C83E060E070E00E94025C86EE99EF0E94CF5C80E090E00E94C6
:20BCC000ED5D88B1837088B987B18C6F87B917980F9A16980E9A08958091650490916604EA
:20BCE0000895E091B708F091B808882319F081E087AB01C017AA81E00895DC01009711F4F6
:20BD000080E00895E091B708F091B80887A9813011F48C9308951C9281E00895843890F427
:20BD200096E06532790770F4E091B708F091B80890E04C96880F991FE80FF91F718360831A
:20BD400081E0089580E00895DB01843898F46115710581F0E091B708F091B80890E04C96A4
:20BD6000880F991FE80FF91F808191818D939C9381E0089580E0089502C00E94416F88B1BB
:20BD80008C73D9F71699F9CFF89480916F008D7F80936F00789402C00E94416F1799FCCF28
:20BDA000F89480916F008B7F80936F007894089580918504089580938504089521E030E0C1
:20BDC00002C0220F331F8A95E2F780918504822380938504811181E0089521E030E002C0E8
:20BDE000220F331F8A95E2F780918504822B809385040895FC01DB018091790490917A0442
:20BE00009183808380917B0490917C048D939C9380917D0490917E04FA01918380830895A7
:20BE2000FC01DB0180917F04909180049183808380918104909182048D939C9380918304B5
:20BE400090918404FA01918380830895833048F5813079F0813018F0823019F51DC0E091B9
:20BE6000B708F091B808E95BFE4F808180FF0AC00EC0E091B708F091B808E95BFE4F808116
:20BE800080FF05C02091790430917A040CC020917B0430917C0407C020917D0430917E0478
:20BEA00002C02FEF3FEFC9010895DB01833078F46115710561F0E82FF0E0EE0FFF1FE1579B
:20BEC000F54F808191818D939C9381E0089580E00895E82F833018F58091210990E0AC0192
:20BEE0004870507083FF03C021E03CEF02C020E030E0621773079CF0452B19F080E094E0BB
:20BF000002C08FEF97E0861797074CF0F0E0EE0FFF1FE157F54F7183608381E0089580E057
:20BF20000895DA018330D0F46330C0F441155105A9F0282F30E083E790E0289FF001299FC5
:20BF4000F00D389FF00D1124EE5DF64FE60FF11DE359FF4F80818C9381E0089580E00895A3
:20BF60008330C0F46330B0F44138A0F4282F30E083E790E0289FF001299FF00D389FF00D84
:20BF80001124EE5DF64FE60FF11DE359FF4F408381E0089580E00895DC01009711F480E0B8
:20BFA0000895E091B708F091B808E95BFE4F80818C9381E00895982F887F11F080E00895F8
:20BFC000E091B708F091B808E95BFE4F908381E00895DA018330D0F46330C0F44115510509
:20BFE000A9F0282F30E083E790E0289FF001299FF00D389FF00D1124EE5DF64FE60FF11D4E
:20C00000E059FF4F80818C9381E0089580E0089599E0899FC00111248A57984F0E94F56D1B
:20C020000895742F833008F048C0633008F045C0483008F042C0282F30E083E790E0289F03
:20C04000F001299FF00D389FF00D1124EE5DF64FE60FF11DE059FF4F4083662319F0613021
:20C06000F1F40AC0E091B708F091B808E95BFE4F808180FF0AC00EC0E091B708F091B80886
:20C08000E95BFE4F808180FF05C04091790450917A0409C040917B0450917C0404C040910E
:20C0A0007D0450917E0489E0689FC00111248A57984F672F0E94B76D089580E008958FE801
:20C0C0009AE06DEA72E046E050E00E949B7581E00895CF93DF93EC010097E9F080912109CB
:20C0E00083FF19C085FF17C0CE010E9412639C01888199819093800480937F048A819B8180
:20C1000090938204809381048C819D81909384048093830402C02FEF3FEFC901DF91CF91C6
:20C120000895CF93DF93EC01009719F42FEF3FEF1EC08091210983FD04C0CE010E94E96694
:20C1400003C0CE010E94F3639C018881998190937A04809379048A819B8190937C04809387
:20C160007B048C819D8190937E0480937D04C901DF91CF9108952F923F924F925F926F9240
:20C180007F928F929F92AF92BF92CF92DF92EF92FF920F931F93DF93CF93CDB7DEB761978D
:20C1A0000FB6F894DEBF0FBECDBF8FE89AE06DEA72E046E050E00E949B751B861A864CC148
:20C1C00087EA91E60197F1F700C000000E94416FCE01019660E040E020E00E949160DC01AF
:20C1E000E091B708F091B808E95BFE4F808129813A814B815C8180FF05C0C901BC01CA0198
:20C200009C0104C0C9019C01CA01BC014D815E81B7FF0CC020918F0A3091900A6091910A6E
:20C220007091920A4091930A5091940A80918F0A9091900A998B888B281B390BC901AA27B6
:20C2400097FDA095BA2FE80EF91E0A1F1B1F2091910A3091920A3F872E87621B730BCB01D1
:20C26000AA2797FDA095BA2FA80EB91ECA1EDB1E8091930A9091940A9D878C87481B590B62
:20C28000CA01AA2797FDA095BA2F280E391E4A1E5B1E0894811C911C90E0891694E09906DA
:20C2A00009F08ECF17FD05C060E072E080E090E004C060E07EEF8FEF9FEF6E0D7F1D801FBA
:20C2C000911F20E034E040E050E00E94497539014A01D7FC05C060E072E080E090E004C0A7
:20C2E00060E07EEF8FEF9FEF6A0D7B1D8C1D9D1D20E034E040E050E00E94497559016A018A
:20C3000057FC05C060E072E080E090E004C060E07EEF8FEF9FEF620D731D841D951D20E0D4
:20C3200034E040E050E00E94497579018A01D401C30197FE07C088279927DC0186199709B4
:20C34000A809B9090297A105B1050CF064C0D601C501D7FE07C088279927DC018A199B0989
:20C36000AC09BD090297A105B1050CF054C0D801C70117FF07C088279927DC018E199F0924
:20C38000A00BB10B0297A105B1050CF044C08091210990E09C012870307083FF03C080E01C
:20C3A00090E002C080EF93E048895989481B590BCA0189589F4F8F3E910568F52115310529
:20C3C00019F080E090E002C080EF93E04E855F85481B590BCA0189589F4F8F3E9105D8F499
:20C3E000232B19F080E090E002C080EF93E02C853D85281B390BC90189589F4F8F3E91057C
:20C4000050F48FE89AE06DEA72E046E050E00E94BF7581E02EC048895989460D571D509366
:20C42000900A40938F0A8E859F858A0D9B1D9093920A8093910A2C853D852E0D3F1D309336
:20C44000940A2093930A4A855B854F5F5F4F5B874A874830510561F0AA24BB2465012224B8
:20C460003324210188249924EE24FF248701A8CE80E061960FB6F894DEBF0FBECDBFCF91A9
:20C48000DF911F910F91FF90EF90DF90CF90BF90AF909F908F907F906F905F904F903F9079
:20C4A0002F9008950F931F93CF93DF9310928504C6E8D7E006E814E0CE0167E040E89801AF
:20C4C0000E946C6D882319F42FEF3FEF11C0299600501F4F87E0C13AD80771F780912109AB
:20C4E00083FD03C00E94C86802C00E94DF659C01C901DF91CF911F910F9108951F93182F62
:20C500000E945915882351F40E9491150E945915882321F40E945915882361F080ED0E94E8
:20C520009515882339F0812F0E949515882319F081E001C080E01F9108950E947E628823D1
:20C5400089F00E948E15882331F40E9491150E948E15882339F081ED0E949515882319F07E
:20C5600081E0089580E008951F93162F0E947E62882329F0812F0E949515882319F480E06F
:20C580001F9108950E94911581E0FACFDF93CF930F92CDB7DEB78091210985FD02C080E06F
:20C5A00001C085E719820E949D62882341F0CE0101960E94EB15882311F00E949115898130
:20C5C0000F90CF91DF9108951F93CF93DF93EC01162F0097A1F417C0123040F0209799F0E2
:20C5E000CE010E94CC15882399F007C0209759F0CE010E94EB15882379F01150219611231D
:20C6000059F781E001C080E0DF91CF911F910895CE010E94CC1503C0CE010E94EB158823FA
:20C6200091F3EBCFEF92FF920F931F93DF93CF93CDB7DEB72C970FB6F894DEBF0FBECDBF5F
:20C640008C01009709F4BFC08091210985FFBBC080E00E94DB5E8BE30E949D62882351F0CA
:20C66000CE01079666E00E94E462882319F00E94911512C08091C1089091C20801969093D3
:20C68000C2088093C10880E00E94ED5E81E00E94ED5E82E00E94ED5E888589838F818A83D4
:20C6A0008A858B8389858C838C858D838B858E8389819A8160E170E00E9414757B017A83A4
:20C6C00069838B819C8160E170E00E9414759B017C836B838D819E8160E170E00E94147517
:20C6E0006D837E83E091B708F091B808E95BFE4F8081E754F140482F81FF05C06B837C8331
:20C700003E832D8312C082FF10C088279927821B930B9A8389838D819E819C838B838827A9
:20C7200099278E199F099E838D8329813A818B819C8140FF09C0D80111969C938E931396AA
:20C740003C932E93129708C0D80111963C932E9313969C938E9312978D819E81D801159675
:20C760009C938E931497E05CFE4F8081282F81FD08C08D919C911197909581959F4F8D935B
:20C780009C9320FD08C0F80182819381909581959F4F9383828322FF0CC0D80114968D91A3
:20C7A0009C911597909581959F4F15969C938E9314970E94D85E882319F420E030E005C06C
:20C7C00020E030E802C02FEF3FEFC9012C960FB6F894DEBF0FBECDBFCF91DF911F910F9140
:20C7E000FF90EF900895DF92EF92FF920F931F93DF93CF93CDB7DEB72C970FB6F894DEBF19
:20C800000FBECDBF8C01F62ED42EE22E009719F42FEF3FEFC5C180E00E94DB5E8091210910
:20C8200085FD02C08DE101C083E40E949D62882351F0CE01079666E00E94E462882319F043
:20C840000E94911512C08091C1089091C20801969093C2088093C10880E00E94ED5E81E0EB
:20C860000E94ED5E82E00E94ED5E888589838F818A838A858B8389858C838C858D838B85DB
:20C880008E832B813C8140E82030340719F48FEF9FE704C088279927821B930B9C838B83BF
:20C8A0002D813E8180E82030380719F48FEF9FE704C088279927821B930B9E838D83E091F3
:20C8C000B708F091B808E95BFE4F8081482F81FF09C02B813C818D819E819C838B833E8382
:20C8E0002D830EC082FF0CC089819A812B813C813A8329832D813E813C832B839E838D836B
:20C90000F80116821782108640FF0DC08B819C81815090488E5F9F4F18F081E0F801868333
:20C9200089819A810CC089819A81815090488E5F9F4F18F081E0F80186838B819C818150F8
:20C9400090488E5F9F4F18F081E0F80187838D819E81815090488E5F9F4F18F081E0F801A5
:20C96000808789819A81FFE3883F9F071CF087EF9FE305C08850904C24F488E090EC9A83A6
:20C98000898389819A8197FF02C0089703C0009719F008969A83898389819A8160E170E08F
:20C9A0000E9414757A8369838B819C814FE3883F94071CF087EF9FE305C08850904C24F411
:20C9C00088E090EC9C838B838B819C8197FF02C0089703C0009719F008969C838B838B81EC
:20C9E0009C8160E170E00E9414757C836B832D813E81C90180519048805F9F4718F420514F
:20CA0000304007C0C90101978E5E9F4720F4205F3F4F3E832D838D819E8160E270E00E94B8
:20CA200014757E836D83FF20E1F089819A8120918F0A3091900A821B930B9A8389838B8152
:20CA40009C812091910A3091920A821B930B9C838B838091930A9091940A681B790B7E8333
:20CA60006D83EE20A9F069817A8180E00E9408609A8389836B817C8181E00E9408609C8334
:20CA80008B836D817E8182E00E9408609E838D83DD2009F45FC049815A81E091BE08F09188
:20CAA000BF08E359FF4F8081ED56F040282F30E0241735072CF4421B530B5A8349830EC081
:20CAC00088279927821B930B481759072CF4240F351F3A83298302C01A8219824B815C813B
:20CAE000E259FF4F8081EE56F040282F30E0241735072CF4421B530B5C834B830EC0882755
:20CB00009927821B930B481759072CF4240F351F3C832B8302C01C821B824D815E81E15963
:20CB2000FF4F8081282F30E0241735072CF4421B530B5E834D830EC088279927821B930BC4
:20CB4000481759072CF4240F351F3E832D8302C01E821D82E091B708F091B808E95BFE4FFB
:20CB600080814B815C8129813A8180FF06C0F801518340833383228305C0F8013183208361
:20CB8000538342838D819E81F801958384830E94D85E882319F420E030E002C020E030E83B
:20CBA000C9012C960FB6F894DEBF0FBECDBFCF91DF911F910F91FF90EF90DF900895809157
:20CBC000210985FD20C08DE361E00E94B462882309F454C08EE360E80E94B462882309F48B
:20CBE0004DC08EE361E00E94B462882309F446C00E94416F89E160E00E94B4628823F1F1CF
:20CC000086E162E132C08AE661E00E94B4628823A9F18BE660E80E94B462882379F10E94A2
:20CC2000416F87EA91E60197F1F700C000000E94416F8BE661E00E94B4628823F9F00E942A
:20CC4000416F89E160E00E94B4628823B9F08AE162E00E94B462882389F08BE160E10E9496
:20CC6000B462882359F08CE160E10E94B462882329F00E94416F20E030E002C02FEF3FEF10
:20CC8000C9010895813059F0813018F0823091F40CC0662311F02C9808952C9A08956623A0
:20CCA00011F02B9808952B9A0895662311F02A9808952A9A08950F931F93CF93DF93082F08
:20CCC000833018F0CFEFDFEF17C0662311F018E901C010E941111460802F61E00E944266F1
:20CCE000812F0E9472698AEA9AEA0E947D69EC01802F60E00E944266CE01DF91CF911F9112
:20CD00000F910895EF92FF920F931F93CF93DF93082F7B016115710509F451C0833008F044
:20CD20004EC061E00E94426680E80E9472698AEA9AEA0E947D69EC01802F60E00E944266CF
:20CD4000D7FD32C0D6FD30C0C0FD2EC0209761F10E94416F1AE013C0802F61E00E9442663D
:20CD600080E80E9472698AEA9AEA0E947D69EC01802F60E00E9442660E94416F1150D5FDA3
:20CD80000AC0D7FD08C0D6FD06C0C0FD04C0209711F0112309F79E01D7FD06C0D6FD04C057
:20CDA000C0FD02C0112319F49E0130680AC0CE019F7096958795F7019183808302C02FEF9E
:20CDC0003FEFC901DF91CF911F910F91FF90EF9008953F924F925F926F927F928F929F9289
:20CDE000AF92BF92CF92DF92EF92FF920F931F93DF93CF9300D0CDB7DEB75C01562E342E69
:20CE0000422E009709F47EC11A82198280E00E94DB5E80E00E94DB5E80E060E041E00E94BF
:20CE20005B6697FD04C083FD02C082FD0CC08091C1089091C20801969093C2088093C10827
:20CE400080E00E94ED5E0E94416F81E060E041E00E945B6697FD04C083FD02C082FD0CC029
:20CE60008091C1089091C20801969093C2088093C10881E00E94ED5E0E94416F82E060E04B
:20CE800041E00E945B6697FD04C083FD02C082FD0CC08091C1089091C20801969093C208E0
:20CEA0008093C10882E00E94ED5E0E94416F0E94D85E80E0BE016F5F7F4F0E9482668C014B
:20CEC00097FF10C08091C1089091C20801969093C2088093C10880E00E94ED5E4801CC2441
:20CEE000DD2405C0C980DA80812C50E8952E81E0BE016F5F7F4F0E9482668C0197FF10C0E8
:20CF00008091C1089091C20801969093C2088093C10881E00E94ED5E480100E010E002C0C3
:20CF200009811A8182E0BE016F5F7F4F0E9482663C0197FF10C08091C1089091C208019686
:20CF40009093C2088093C10882E00E94ED5E4301EE24FF2402C0E980FA80F5011682178274
:20CF60001086E091B708F091B808E95BFE4F808180FF13C00115110521F0F7E00F3F1F073E
:20CF800019F481E0F5018683C114D104C1F0FFEFCF16F7E0DF06B1F412C0C114D10429F000
:20CFA000FFEFCF16F7E0DF0619F481E0F50186830115110521F0F7E00F3F1F0719F481E07F
:20CFC000F5018783E114F10429F0FFEFEF16F7E0FF0619F481E0F5018087552091F080910D
:20CFE0008F0A9091900AC81AD90A8091910A9091920A081B190B8091930A9091940AE81AF9
:20D00000F90A442079F080E0B6010E9408606C0181E0B8010E9408608C0182E0B7010E9445
:20D0200008607C01332009F44DC0E091BE08F091BF08E359FF4F8081ED56F040282F30E0CA
:20D040002C153D051CF4C21AD30A0CC088279927821B930BC816D9061CF0CC24DD2402C092
:20D06000C20ED31EE259FF4F8081EE56F040282F30E0201731071CF4021B130B0CC0882755
:20D080009927821B930B081719071CF000E010E002C0020F131FE159FF4F8081282F30E085
:20D0A0002E153F051CF4E21AF30A0CC088279927821B930BE816F9061CF0EE24FF2402C06A
:20D0C000E20EF31EE091B708F091B808E95BFE4F808180FF06C0F50111830083D382C28261
:20D0E00005C0F501D182C08213830283F501F582E4820E94D85E882341F4672819F08824F6
:20D10000992403C088248A94982CC4010F900F90CF91DF911F910F91FF90EF90DF90CF9002
:20D12000BF90AF909F908F907F906F905F904F903F900895FF920F931F93CF93DF93F82EEC
:20D1400082E08F1518F4CFEFDFEF1BC0662311F018EA01C010EA4111146021111260011193
:20D1600011608F2D61E00E944266812F0E9472698AEA9AEA0E947D69EC018F2D60E00E94BF
:20D180004266CE01DF91CF911F910F91FF900895EF92FF920F93CF93DF931092C208109236
:20D1A000C10880E060E040E020E000E00E949A68EC01181619061CF4EE24FF2408C080E0BB
:20D1C0000E94ED5EE12CE0E8FE2EEC2AFD2A0E94416F81E060E040E020E000E00E949A688D
:20D1E000EC011816190644F081E00E94ED5EE12C70E8F72EEC2AFD2A0E94416F82E060E0B8
:20D2000040E020E000E00E949A68EC011816190644F082E00E94ED5EE12C60E8F62EEC2A1E
:20D22000FD2A0E94416F0E94D85E882309F47E01C701DF91CF910F91FF90EF900895809380
:20D24000A107823091F0833028F4882301F18130F1F405C0833079F08430C9F415C08CB589
:20D2600082608CBD8CB58E7F0BC08CB58D7F8CBD8CB5816011C08CB58D7F8CBD8CB5816029
:20D280008CBD8DB581600BC08CB58D7F02C08CB582608CBD8CB58E7F8CBD8DB58E7F8DBDAC
:20D2A0000895982F8091A107981719F0892F0E941F69089594B1906A94B9269895B19C618D
:20D2C00095B994B19C6194B990E49CBD9CB590619CBD9CB598609CBD9CB594609CBD0E9427
:20D2E0001F6908958EBD0DB407FEFDCF08958EBD0DB407FEFDCF8EB508959EBD0DB407FEB1
:20D30000FDCF3EB58EBD0DB407FEFDCF2EB5932F80E030E0282B392BC90108952F923F92AC
:20D320004F925F926F927F928F929F92AF92BF92CF92DF92EF92FF920F931F93DF93CF9319
:20D34000CDB7DEB760970FB6F894DEBF0FBECDBFDC013B016A011901E091B708F091B80867
:20D360008389E82E80FF0AC0882799278A1B9B0BAC01662757FD6095762F05C0AD01662760
:20D3800057FD6095762F3381313019F480E020E802C0218980E0629F5001429F4001A80A23
:20D3A000B80A529F900CA11CB81E7203B00C112489829A82AB82BC82E1FE0AC0882799277B
:20D3C00086199709AC01662757FD6095762F05C0A301662757FD6095762F313019F480E034
:20D3E00020E802C0228980E0629F4001429F3001880A980A529F700C811C981E7203900CFF
:20D400001124E2FE06C0A601662757FD6095762F09C0882799278C199D09AC01662757FDFE
:20D420006095762F313019F480E020E802C0208980E0629F6001429F5001C80AD80A529F78
:20D44000B00CC11CD81E7203D00C1124FE83ED83188A1F865524AD81BE8114968C91149727
:20D4600029813A814B815C81682F64038001620370010509150963031509F00C011D151D4D
:20D480006502100D1124EB86FC860D871E871896EC91940183014E2F4203D0014003C001CC
:20D4A000A509B5094103B509900DA11DB51D4302B00D1124ED81FE814484A6019501642D17
:20D4C00064038001620370010509150963031509F00C011D151D6502100D1124EF82F886EA
:20D4E00009871A87EF85F889E20DF31DEB84FC840D851E858E0D9F1DA01FB11F0F811885D0
:20D5000029853A85800F911FA21FB31F2EE0B595A795979587952A95D1F7918380832D81A4
:20D520003E812F5F3F4F3E832D834F8558894E5F5F4F588B4F874830510509F08CCF6096BE
:20D540000FB6F894DEBF0FBECDBFCF91DF911F910F91FF90EF90DF90CF90BF90AF909F90CB
:20D560008F907F906F905F904F903F902F900895883010F080E00895E091B708F091B8085F
:20D58000838381E00895DC01009711F480E00895E091B708F091B80883818C9381E008957F
:20D5A000843068F463385CF06E374CF4E091B708F091B808E80FF11D648381E0089580E0D4
:20D5C0000895DB01843068F46115710551F0E091B708F091B808E80FF11D84818C9381E09A
:20D5E000089580E00895843068F463385CF06E374CF4E091B708F091B808E80FF11D608758
:20D6000081E0089580E00895DB01843068F46115710551F0E091B708F091B808E80FF11D80
:20D6200080858C9381E0089580E00895843068F463385CF06E374CF4E091B708F091B8087E
:20D64000E80FF11D648781E0089580E00895DB01843068F46115710551F0E091B708F09115
:20D66000B808E80FF11D84858C9381E0089580E008958430B8F46338ACF06E379CF4E09185
:20D68000B708F091B808E80FF11D6483433854F04E3744F4408723382CF02E371CF42487C4
:20D6A00081E0089580E00895813810F080E00895E091B708F091B808808B81E00895DC0162
:20D6C000009711F480E00895E091B708F091B80880898C9381E00895DC01009711F480E041
:20D6E0000895E091B708F091B80881898C9381E00895813810F080E00895E091B708F0918E
:20D70000B808818B81E00895DC01009711F480E00895E091B708F091B80882898C9381E0CD
:20D720000895833010F080E00895282F30E0662371F083E790E0289FF001299FF00D389F1D
:20D74000F00D1124EE5DF64F81E08383089583E790E0289FF001299FF00D389FF00D1124A3
:20D76000EE5DF64F138281E00895DB018330C0F461157105A9F0282F30E083E790E0289FB6
:20D78000F001299FF00D389FF00D1124EE5DF64F8381813011F48C9308951C9281E0089518
:20D7A00080E00895DB018330A0F46115710589F0282F30E083E790E0289FF001299FF00D26
:20D7C000389FF00D1124EE5DF64F84818C9381E0089580E00895833090F4613880F4282FF6
:20D7E00030E083E790E0289FF001299FF00D389FF00D1124EE5DF64F648381E0089580E0E4
:20D800000895813810F080E00895E091B708F091B808828B0E94AF4481E008956F927F9292
:20D820008F929F92AF92BF92DF92EF92FF920F931F93CF93DF93DC01EB014A013901FA0110
:20D8400091838083F90171836083E091BE08F091BF0824818AE998E0829FA00166277727E4
:20D86000929F500D611D11248381882309F468C08D01085F1F4FA4E015950795AA95E1F74F
:20D880002896F4E0D595C795FA95E1F7EBE07695679557954795EA95D1F75A01CC9FC00161
:20D8A000CD9F900DDC9F900D1124009F9001019F300D109F300D1124820F931F0E94A670E9
:20D8C0009C01A816B90608F03BC0DD24A5011503C001049FB00114039D09700D811D9D1DD5
:20D8E000059F700D811D9D1D1124790100E010E0A80197010E94497554E0220F331F5A95E9
:20D90000E1F7F401318320839E01A5013503C001249FB00134039D09700D811D9D1D259FBB
:20D92000700D811D9D1D1124A80197010E94497544E0220F331F4A95E1F7F3013183208393
:20D94000DF91CF911F910F91FF90EF90DF90BF90AF909F908F907F906F9008951F920F9251
:20D960000FB60F9211242F938F939F93EF93FF939091C0002091C600E091E407EF5FEF7180
:20D980008091E507E81711F482E008C0892F8871E093E407F0E0EE53F84F20838093E60752
:20D9A000FF91EF919F918F912F910F900FBE0F901F9018951F920F920FB60F9211248F93D1
:20D9C0009F93EF93FF939091E2078091E307981769F0E091E307EF5FEF71E093E307F0E0BE
:20D9E000EE55F84F80818093C60005C08091C1008F7D8093C100FF91EF919F918F910F904D
:20DA00000FBE0F901F9018959C011092E2071092E3071092E4071092E50797FF04C082E0B3
:20DA20008093C0003F773093C5002093C40088E98093C10086E08093C20008959091E40735
:20DA40008091E507981719F420E031E012C0E091E507EF5FEF71E093E507F0E0EE53F84F68
:20DA600030812091E607922F80E0AC01430F511D9A01C9010895282F9091E2079F5F9F7158
:20DA80008091E3079817E1F3E92FF0E0EE55F84F20839093E2078091C10080628093C1005F
:20DAA0000895CF93DF93EC0103C021960E943B6D88818823D1F7DF91CF910895CF93DF9387
:20DAC000EC0102C00E943B6DFE01219684918823C9F7DF91CF910895DC01F901009709F43F
:20DAE00044C02115310509F440C06830F0F581E090E0062E02C0880F991F0A94E2F7242F5C
:20DB000030E08217930789F51D921D921D921C92139714961C92149715961C92159716962B
:20DB20006C9316971896FC93EE93179740E061E070E00BC0220F331F1796ED91FC91189767
:20DB4000E20FF31F118210824F5F242F30E0CB0116960C90169702C0880F991F0A94E2F743
:20DB6000281739073CF381E0089580E00895EF92FF921F93CF93DF93EC017A01009771F103
:20DB80008E81861758F16D8381E090E002C0880F991F6A95E2F7182F11501C831F5F612F91
:20DBA00070E080E090E09701442737FD4095542F0E94E174688379838A839B8320E080E04D
:20DBC00090E008C0EF81F885E80FF91FF182E0822F5F02962117B0F381E001C080E0DF9149
:20DBE000CF911F91FF90EF900895EF92FF920F931F93CF93DF93EC01009719F460E070E00F
:20DC000052C02D81222309F44EC081E090E002C0880F991F2A95E2F7182F8C818F5F8C8329
:20DC2000811708F01C829B01442737FD4095542F88819981AA81BB81280F391F4A1F5B1F27
:20DC40008C8190E0880F991FEF81F885E80FF91F80819181AA2797FDA095BA2F281B390BDF
:20DC60004A0B5B0B288339834A835B8371836083812F869557FF07C079018A01E81AF10818
:20DC80000109110906C079018A01E80EF11C011D111DC801B7010D8004C095958795779522
:20DCA00067950A94D2F7CB01DF91CF911F910F91FF90EF900895DC01009761F12115310538
:20DCC00049F1423041F0443031F0483021F0403111F04032F9F44617E8F012961C92129744
:20DCE0006C9311964C93119714963C932E93139720E080E090E00AC01396ED91FC9114971A
:20DD0000E80FF91F118210822F5F02962417A0F381E0089580E00895DC019B01009719F4C3
:20DD200020E030E023C08C91882301F112968C91129790E0880F991F1396ED91FC911497AA
:20DD4000E80FF91F408151817183608312962C9112972F5F12962C9312978C9190E030E001
:20DD60002817390714F012961C929A01C9010895FC01009751F06115710539F07183608307
:20DD800042831482138281E0089580E00895DC01009711F113968C9113978823E9F0149684
:20DDA0008C911497ED91FC911197E80FF11DE0818F5F14968C93149712969C911297891702
:20DDC00020F0891B14968C93149713968C911397815013968C9301C0E0E08E2F0895EF92B6
:20DDE000FF921F93CF93DF937C01142F009771F06115710559F0EB0105C0C7010E94C76ECF
:20DE0000899311501123C9F781E001C080E0DF91CF911F91FF90EF900895CF93DF93EC0123
:20DE2000362F0097A9F02B816A81261788F48C8190E0820F911D70E00E941475E881F981E3
:20DE4000E80FF91F30838B818F5F8B8381E001C080E0DF91CF91089588E10FB6F89480933C
:20DE60006000109260000FBE08952BE088E190E00FB6F894A895809360000FBE2093600011
:20DE80000895A8950895833009F456C0843030F48130D1F0823009F058C044C0853031F05E
:20DEA000853000F1863009F050C02AC02FB7F8948FEF9FEF9093E9078093E8072FBF2FB7AC
:20DEC000F89481E091E029C02FB7F8948FEF9FEF9093E9078093E8072FBF2FB7F89485E0A3
:20DEE00095E01BC02FB7F8948FEF9FEF9093E9078093E8072FBF2FB7F89485E195E10DC036
:20DF00002FB7F8948FEF9FEF9093E9078093E8072FBF2FB7F89485E590E09093EB0780930C
:20DF2000EA0708C02FB7F89481E091E09093E9078093E8072FBF08952FB7F89485E095E0F8
:20DF40009093E9078093E8072FBF08951F920F920FB60F9211242F933F938F939F9380913B
:20DF6000E707882309F041C078948091C5019091C60101979093C6018093C501892B91F5AE
:20DF800086E290E09093C6018093C5018091C3019091C401880F991F9093C4018093C3011D
:20DFA000892B31F481E090E09093C4018093C3012091C3013091C4018091E8079091E907EC
:20DFC00082239323892B11F0289801C0289A8091EA079091EB0782239323892B11F0299808
:20DFE00001C0299AF8941092E7079F918F913F912F910F900FBE0F901F9018958FB7F89468
:20E000001092E9071092E8078FBF8FB7F8941092EB071092EA078FBF85B1836085B984B1BC
:20E02000836084B914BC85E085BD81E080936E0008952FB7F8949093E9078093E8072FBF55
:20E0400008952FB7F8949093EB078093EA072FBF08950F931F93CF93DF9360E07AE50E94A4
:20E060001475EC0197FF02C0C050D64A26E1C038D20760F0CE018A559040865A9C4240F40A
:20E0800080E09DE2BC016C1B7D0BEB0140E010C0CE01845B90408C5C924418F4C050DD4282
:20E0A00006C080E09AE59C012C1B3D0BE90141E0CE0160E470E00E941475862F8F5F8B3593
:20E0C00080F0442349F08091C1019091C20166277727681B790B2FC06091C1017091C201E1
:20E0E0002AC0E62FF0E0EE0FFF1FE35FFE4F00811181E82FF0E0EE0FFF1FE35FFE4F208162
:20E100003181201B310BCE0160E470E00E941475BC01269FC001279F900D369F900D1124FB
:20E1200060E470E00E941475600F711F442319F0709561957F4FCB01DF91CF911F910F91FC
:20E1400008958058994E0E9429700895CF93DF93EC012296FE01F695E795229781E090E082
:20E160000DC09F012F5F3F4FCE01BF010E940075260F371FCF01F901F695E7959F01281B31
:20E18000390BC90137FF03C0909581959F4F029744F7CF01DF91CF9108950F931F9304B72F
:20E1A00084B7807E84BF2BE088E190E00FB6F894A895809360000FBE20936000102F03FFDD
:20E1C00002C00E945C1012FF04C010FD02C00E943E10802F1F910F910895A0E2B0E0E3EF5B
:20E1E000F0E70C94647569837A838B839C832D833E834F835887CE010196BE01675F7F4FDE
:20E200000E946974CE010596BE016F5E7F4F0E9469749985923088F089898230C8F09430A4
:20E2200019F4823051F404C0843029F4923081F487EC91E0C6C0923049F420E09A858A8973
:20E24000981321E02A87CE010996BBC0823049F420E09A858A89981321E02A8BCE01419650
:20E26000B0C02D843E844F8458886D887E888F88988CEE24FF248701AA24BB24650140E0E2
:20E2800050E060E070E0E0E0F0E0C10181709070892BE9F0E60CF71C081D191D9A01AB0147
:20E2A0002A0D3B1D4C1D5D1D80E090E0A0E0B0E0E614F7040805190520F481E090E0A0E087
:20E2C000B0E0BA01A901480F591F6A1F7B1FAA0CBB1CCC1CDD1C97FE08C081E090E0A0E03B
:20E2E000B0E0A82AB92ACA2ADB2A3196E032F10549F0660C771C881C991C569447943794EA
:20E300002794C3CFFA85EA892B893C898B859C85280F391F2E5F3F4F17C0CA0181709070D7
:20E32000892B61F016950795F794E79480E090E0A0E0B0E8E82AF92A0A2B1B2B76956795EC
:20E34000579547952F5F3F4F77FDE7CF0CC0440F551F661F771F17FD4160EE0CFF1C001F18
:20E36000111F21503040403090E0590790E0690790E4790760F32B8F3C8FDB01CA018F77F3
:20E380009070A070B07080349105A105B10561F447FD0AC0E114F1040105110529F0405C89
:20E3A0005F4F6F4F7F4F40781A8EFE1711F081E08A8F4D8F5E8F6F8F78A383E0898FCE0107
:20E3C00049960E949473A096E2E10C948075A8E1B0E0EDEEF1E70C946C7569837A838B83E3
:20E3E0009C832D833E834F835887B9E0EB2EF12CEC0EFD1ECE010196B7010E9469748E01CC
:20E400000F5E1F4FCE010596B8010E9469742985223008F47EC03989323010F4B8017CC028
:20E420008A859A8989278A87243011F0223031F4231709F06EC067EC71E06EC0343039F459
:20E440001D861E861F86188A1C861B8604C0323021F484E08987B7015FC02B853C858B89E0
:20E460009C89281B390B3C872B87ED84FE840F851889AD88BE88CF88D88CEA14FB040C050F
:20E480001D0540F4EE0CFF1C001F111F215030403C872B8720E030E040E050E080E090E03C
:20E4A000A0E0B0E460E070E0EA14FB040C051D0540F0282B392B4A2B5B2BEA18FB080C098C
:20E4C0001D09B695A79597958795EE0CFF1C001F111F6F5F7F4F6F31710531F7DA01C90164
:20E4E0008F779070A070B07080349105A105B10561F427FD0AC0E114F1040105110529F0DE
:20E50000205C3F4F4F4F5F4F20782D873E874F87588BBE01675F7F4FCB010E949473689615
:20E52000EAE00C948875A8E0B0E0E9E9F2E70C946D759B01AC0183E08983DA01C901882723
:20E54000B7FD83959927AA27BB27B82E211531054105510519F482E089833AC08823A9F0D5
:20E56000203080E0380780E0480780E8580729F460E070E080E09FEC30C0EE24FF248701F1
:20E58000E21AF30A040B150B02C079018A018EE1C82ED12CDC82CB82ED82FE820F8318875F
:20E5A000C801B7010E94457301971816190684F4082E04C0EE0CFF1C001F111F0A94D2F75E
:20E5C000ED82FE820F831887C81AD90ADC82CB82BA82CE0101960E9494732896E9E00C9439
:20E5E0008975ACE0B0E0E7EFF2E70C94747569837A838B839C83CE010196BE016B5F7F4FF6
:20E600000E9469748D81823061F1823050F1843021F48E81882351F12EC02F81388537FD22
:20E6200020C06E812F3131051CF06623F9F023C08EE190E0821B930B29853A854B855C85DC
:20E6400004C056954795379527958A95D2F76623B1F050954095309521953F4F4F4F5F4F86
:20E660000EC020E030E040E050E009C02FEF3FEF4FEF5FE704C020E030E040E050E8B901ED
:20E68000CA012C96E2E00C949075EF92FF920F931F937B018C0180E0E81680E0F80681E0FA
:20E6A000080780E0180788F48FEFE816F1040105110531F028F088E090E0A0E0B0E017C0CB
:20E6C00080E090E0A0E0B0E012C080E0E81680E0F80680E0080781E0180728F088E190E0EC
:20E6E000A0E0B0E004C080E190E0A0E0B0E020E230E040E050E0281B390B4A0B5B0B04C0FD
:20E7000016950795F794E7948A95D2F7F701E153FE4F8081281B310941095109C9011F91AF
:20E720000F91FF90EF900895DF92EF92FF920F931F93FC01E480F58006811781D180808170
:20E74000823048F480E090E0A0E1B0E0E82AF92A0A2B1B2BA5C0843009F49FC0823021F4FE
:20E76000EE24FF24870105C0E114F1040105110519F4E0E0F0E096C0628173819FEF62381F
:20E7800079070CF05BC022E83FEF261B370B2A3131052CF020E030E040E050E02AC0B80177
:20E7A000A701022E04C076956795579547950A94D2F781E090E0A0E0B0E004C0880F991F93
:20E7C000AA1FBB1F2A95D2F70197A109B1098E219F21A023B1230097A105B10521F081E0A7
:20E7E00090E0A0E0B0E09A01AB01282B392B4A2B5B2BDA01C9018F779070A070B070803411
:20E800009105A105B10539F427FF09C0205C3F4F4F4F5F4F04C0215C3F4F4F4F5F4FE0E0B9
:20E82000F0E02030A0E03A07A0E04A07A0E45A0710F0E1E0F0E079018A0127C060387105B6
:20E8400064F5FB01E158FF4FD801C7018F779070A070B07080349105A105B10539F4E7FE4D
:20E860000DC080E490E0A0E0B0E004C08FE390E0A0E0B0E0E80EF91E0A1F1B1F17FF05C0E6
:20E8800016950795F794E794319687E016950795F794E7948A95D1F705C0EE24FF24870147
:20E8A000EFEFF0E06E2F679566276795902F9F77D794DD24D7948E2F8695492F462B582F94
:20E8C0005D29B701CA011F910F91FF90EF90DF900895FC01DB01408151812281622F6F773F
:20E8E00070E0221F2227221F9381892F880F822B282F30E0991F9927991F11969C931197D8
:20E9000021153105A9F5411551056105710511F482E037C082E89FEF13969C938E9312976D
:20E920009A01AB0167E0220F331F441F551F6A95D1F783E08C930DC0220F331F441F551F7F
:20E9400012968D919C911397019713969C938E931297203080E0380780E0480780E458077F
:20E9600058F314962D933D934D935C93179708952F3F310579F4411551056105710519F452
:20E9800084E08C93089564FF03C081E08C9312C01C9210C02F57304013963C932E93129789
:20E9A00083E08C9387E0440F551F661F771F8A95D1F7706414964D935D936D937C9317979A
:20E9C0000895629FD001739FF001829FE00DF11D649FE00DF11D929FF00D839FF00D749F4B
:20E9E000F00D659FF00D9927729FB00DE11DF91F639FB00DE11DF91FBD01CF011124089540
:20EA0000AA1BBB1B51E107C0AA1FBB1FA617B70710F0A61BB70B881F991F5A95A9F78095BE
:20EA20009095BC01CD01089597FB092E07260AD077FD04D0E5DF06D000201AF470956195AE
:20EA40007F4F0895F6F7909581959F4F0895A1E21A2EAA1BBB1BFD010DC0AA1FBB1FEE1FB7
:20EA6000FF1FA217B307E407F50720F0A21BB30BE40BF50B661F771F881F991F1A9469F71C
:20EA800060957095809590959B01AC01BD01CF01089597FB092E05260ED057FD04D0D7DF1E
:20EAA0000AD0001C38F450954095309521953F4F4F4F5F4F0895F6F7909580957095619566
:20EAC0007F4F8F4F9F4F08952F923F924F925F926F927F928F929F92AF92BF92CF92DF92D3
:20EAE000EF92FF920F931F93CF93DF93CDB7DEB7CA1BDB0B0FB6F894DEBF0FBECDBF099414
:20EB00002A88398848885F846E847D848C849B84AA84B984C884DF80EE80FD800C811B8183
:20EB2000AA81B981CE0FD11D0FB6F894DEBF0FBECDBFED010895DC01CB01FC01F999FECFCE
:20EB400006C0F2BDE1BDF89A319600B40D9241505040B8F70895F999FECF92BD81BDF89A0B
:20EB6000992780B50895A8E1B0E042E050E00C949D750196272F0E94DD750C94DC75DC0137
:20EB8000CB0103C02D910E94CA7541505040D0F70895262FF999FECF1FBA92BD81BD20BDCB
:20EBA0000FB6F894FA9AF99A0FBE019608950E94C975272F0C94CA75262FF999FECF92BDC4
:20EBC00081BDF89A019700B4021639F01FBA20BD0FB6F894FA9AF99A0FBE0895F894FFCFE6
:20EBE0000106001900190008E6F91A060400008E001D01AC013B02C9025803E603740401B3
:20EC0000058E051B06A7063207BD074808D2085B09E3096B0AF10A770BFC0B800C030D86FC
:20EC20000D070E870E050F830F00107B10F5106D11E4115A12CF124213B31323149114FE22
:20EC4000146915D2153A16A01604176717C71726188318DE1837198E19E319361A871AD635
:20EC60001A231B6D1BB61BFC1B411C831CC21C001D3B1D741DAB1DDF1D111E411E6F1E9A73
:20EC80001EC21EE81E0C1F2E1F4C1F691F831F9B1FB01FC21FD31FE01FEC1FF41FFB1FFED2
:20ECA0001F00200100010000000000000000000001020203030303040404040404040405DD
:20ECC000050505050505050505050505050505060606060606060606060606060606060683
:20ECE000060606060606060606060606060606070707070707070707070707070707070743
:20ED0000070707070707070707070707070707070707070707070707070707070707070713
:20ED20000707070707070707070707070707070808080808080808080808080808080808E2
:20ED40000808080808080808080808080808080808080808080808080808080808080808B3
:20ED6000080808080808080808080808080808080808080808080808080808080808080893
:20ED8000080808080808080808080808080808080808080808080808080808080808080873
:20EDA000080808080808080808080808080808002091C3013091C4018091E8079091E907CF
:20EDC00082239323892B11F0289801C0289A8091EA079091EB0782239323892B11F02998FA
:20EDE00001C0299AF8941092E7079F918F913F912F910F900FBE0F901F9018958FB7F8945A
:20EE0000FFFFFFFFFFFFFFFFFFFFFFFFFFFFFFFFFFFFFFFFFFFFFFFFFFFFFFFFFFFFFFFF12
:20EE2000FFFFFFFFFFFFFFFFFFFFFFFFFFFFFFFFFFFFFFFFFFFFFFFFFFFFFFFFFFFFFFFFF2
:20EE4000FFFFFFFFFFFFFFFFFFFFFFFFFFFFFFFFFFFFFFFFFFFFFFFFFFFFFFFFFFFFFFFFD2
:20EE6000FFFFFFFFFFFFFFFFFFFFFFFFFFFFFFFFFFFFFFFFFFFFFFFFFFFFFFFFFFFFFFFFB2
:20FC0000F8940FEF0DBF00E10EBF22243324A89500916000076100936000107F0093600038
:20FC2000589A599A519A41E050EA06E0F101EF01F101019700404899E1F781F1219734965A
:20FC400068F1489BFBCF0F2EC5950694E9F72397269668F7EA35F20550F3F797F695E795CA
:20FC60002F01CAE0ECECFDEF0590002031F079D00016D1F3CA9591F0F5CF06EA8CD071D0BC
:20FC8000E1F70AEA88D06DD0F1F76BD0F1F3F101E8940430F8F061F1063020F42AB82BB811
:20FCA0000C94000031F45DD05CD0672851F331010FC0073059F455D019F453D0005821F010
:20FCC000059000126894F7CF1EF0DBCF07EADACF0BEAD8CFE2EDFDEFC0E0EC0FF21DC49113
:20FCE0000150D8F708EA57D00591C150E0F7C9CFA0E0B1E0ED0135D021F433D00058689445
:20FD000031F0E8940D93A0300FE0B007A1F7AC17BD0731F1A0E0BFE0E050F24F10E832979E
:20FD20001E900E9001E015D01A95C9F7E0301CEFF107A8F403E00DD005E009D0AC17BD078E
:20FD400069F776F0E050F24F09EA25D0D4CF01D001E107BFE89507B700FDFDCF0895B8CF40
:20FD600090CFA895489BFDCF4899FECF18E0C2019695879523D021D006954899006807FDBC
:20FD800064267694679408F4642608F475261A9591F7053A089511D05998149119E000959F
:20FDA00000C000C00AD0069518F40000599802C0599A00C01A95A1F70895C2010497F0F7B3
:20FDC0008D3F18F011F08F3F01F00895506564610000030108030E00041E96090400FC009A
:00000001FF
